:1000000000800020BD01000029CD0200E1CC0200EB
:10001000E1CC0200E1CC0200E1CC0200E1CC020024
:10002000E1CC0200E1CC0200E1CC020029CD0200CB
:1000300029CD0200E1CC020069EF02006DEF020061
:1000400029CD020029CD020029CD020029CD0200D0
:1000500029CD020029CD020029CD020029CD0200C0
:1000600029CD020029CD020029CD020029CD0200B0
:1000700029CD020029CD020029CD020029CD0200A0
:1000800029CD020029CD020029CD020029CD020090
:1000900029CD020029CD020029CD020029CD020080
:1000A00029CD020029CD020029CD020029CD020070
:1000B00029CD020029CD020029CD020029CD020060
:1000C00029CD020029CD020029CD020029CD020050
:1000D00029CD020029CD020029CD020029CD020040
:1000E00029CD020029CD020029CD020029CD020030
:1000F00029CD020019D8020029CD020029CD020025
:1001000029CD02002DDF020029CD020029CD0200F9
:1001100029CD020029CD020029CD020029CD0200FF
:1001200029CD020029CD020029CD020029CD0200EF
:1001300029CD020029CD02004DC3020029CD0200C5
:1001400029CD020029CD020029CD020029CD0200CF
:10015000D9F20200EDF2020001F3020015F30200F1
:1001600029CD02001DE2020029CD020029CD0200A6
:1001700029CD020029CD020029CD020029CD02009F
:1001800029CD020029CD020029CD020029CD02008F
:1001900029CD020029CD020029CD020029CD02007F
:1001A00029CD020029CD020029CD020029CD02006F
:1001B00029CD020029CD020029CD0200564B4CF278
:1001C000205210B51A804DF628121A8000BF00BFC9
:1001D0002CF0AEFD514B4FF010621A60504A9A60FD
:1001E000504ADA60504A136813F4807304D14F49BF
:1001F0000B604FF4A85313604D4B1A78110703D5C9
:100200001A7842F008021A704A4B4B492A221A7097
:100210004A4A4B4B8B4204D252F8040F43F8040B6A
:10022000F8E7484B484900228B4202D243F8042B9E
:10023000FAE74649464A002352F8230041F82300D2
:1002400001336F2BF8D1434B434A802103F8011B44
:100250009342FBD1414B3D4A1A60414B8A221A70AE
:10026000A3F5805324225A70A0221A709A7992071B
:10027000FCD59A79D406FCD43A4A937903F00C035E
:10028000082B384BF9D105221A7143225A719A79F9
:100290009006FCD5334A9179324B4906FBD5324A58
:1002A0004FF0817111600521516020221A709A79F6
:1002B00002F00C020C2AFAD12C4B2D4A1A602D4B5D
:1002C0002D4A1A6000225A60072243F8042C2B4A58
:1002D000C3F80C2D62B62CF06FFE144B1B68DA07C6
:1002E00005D527482CF0C6FD264B274A1A60274B18
:1002F0001B785B0609D5234C234B22689A4204D114
:100300001F482CF0B7FD002323602CF017FD32F0BE
:1003100095F92FF009F8FEE70E20054030800440E3
:10032000823F04000100002B10D0034014D0034092
:1003300002D0074000E00740C892FF1F38A003002A
:100340002087FF1FC892FF1F14A3FF1F0082FF1FFB
:100350000000000000E400E05FE400E008ED00E0E1
:1003600000500640004006404480044004800440A1
:10037000C010050014E000E03F190100000020203B
:10038000AC7413631CE00340A5C3945A00F007400B
:10039000FFFFFFFFFFFFFFFFFFFFFFFFFFFFFFFF6D
:1003A000FFFFFFFFFFFFFFFFFFFFFFFFFFFFFFFF5D
:1003B000FFFFFFFFFFFFFFFFFFFFFFFFFFFFFFFF4D
:1003C000FFFFFFFFFFFFFFFFFFFFFFFFFFFFFFFF3D
:1003D000FFFFFFFFFFFFFFFFFFFFFFFFFFFFFFFF2D
:1003E000FFFFFFFFFFFFFFFFFFFFFFFFFFFFFFFF1D
:1003F000FFFFFFFFFFFFFFFFFFFFFFFFFFFFFFFF0D
:10040000FFFFFFFFFFFFFFFFFFFFFFFFDEF9FFFF23
:1004100010B5054C237833B9044B13B10448AFF33E
:1004200000800123237010BDC892FF1F0000000050
:1004300034A00300084B10B51BB108490848AFF3BE
:1004400000800848036803B910BD074B002BFBD0A0
:10045000BDE81040184700BF00000000CC92FF1F0D
:1004600034A00300C892FF1F000000000020704766
:10047000704700BF036D0BB101207047406D003025
:1004800018BF0120704700BF00690B699842D4BFB4
:1004900000200120704700BF80698B690028B8BF29
:1004A0004042002BB8BF5B429842D4BF00200120DD
:1004B000704700BFF0B586460120DEF85870DEF8C0
:1004C0003030BA6A106079683A680A447A600EF18E
:1004D000300493B15A69002A08DB9A6A10605E689A
:1004E00019683D695A6931445960521B19690A44B7
:1004F0005A6154F8043F002BECD1DEF82430144A42
:10050000DEF81840DEF86C0000211160DB00516855
:1005100003F1804303F5603321440D241961146015
:10052000DA68502122F08002DA60D96000B1F0BDB3
:100530007A68FB689A4200D0F0BDDEF85C30012298
:100540008EF82820002BF7D0BDE8F040184700BFF8
:1005500000800340C36A00F12C0233B10120D96A44
:1005600052F8043F0860002BF9D1704710B50446DB
:10057000806D18B132F0B2F80023A365236D2BB162
:1005800004F11800BDE810402AF068BD636D002B2F
:10059000F6D110BDF0B5002395B01A4605461831C6
:1005A00004A84FF47A74224F8DF804308DF80C3083
:1005B00012931393029400972AF0A4FD129B002B30
:1005C0002BD05C202EF0B8FE04461A4B9DF8040098
:1005D000029A1949236000269DF80C302073A1600F
:1005E000226104A9237504F1180066602AF008FD51
:1005F0006368124AA76001334FF47A71A6652E71C1
:100600002E732C616360A9602A600D4B009304A8CF
:100610002AF024FD284615B0F0BD139B002BD0D145
:10062000064A2B71AC602B732B612A60EDE700BF8B
:10063000B86203000863030070620300DC62030019
:1006400094620300836C13B1184628F083BFC06C1A
:1006500008B126F0C9BD4FF0FF30704700B5836C7C
:1006600083B063B1184601220DF1070128F0A2FE04
:1006700001280CD19DF8070003B05DF804FBC06CA5
:1006800028B101220DF1070126F0DAFCF0E74FF066
:10069000FF30F1E708B52DF0BDFB0028CCBF0320EB
:1006A000002008BD836D012210B55B6880F89020A2
:1006B000044672B60021D0F8800031F0C9FBE16F2A
:1006C000A06731F081FD28B1D4F88830C4F88C30AF
:1006D00062B610BDD4F8883003F10043C4F88C3002
:1006E00062B610BD036D9BB11A7812F0700F00D185
:1006F000704710B504460021184629F04DF8606D8A
:1007000028B100220023BDE8104026F085BD10BDB1
:10071000406D0028ECD090F8313013F0500FE7D046
:100720000022002326F078BD38B5846D0CB1204638
:1007300038BD05464FF4807031F0C8FF0146A8650A
:1007400080B1286D0C7028B14FF480722AF090FAB5
:10075000AC6DECE7686D40B14FF4807228F0CCF8D6
:10076000AC6DE4E7024CAC65E1E70C46DFE700BFA7
:10077000E492FF1F8A79A2F150031B0620D4F0B542
:100780004B79046D0D798E784F780978013385B0F7
:1007900002F26C72DBB244B103918DE8E0002046B6
:1007A000022129F011F905B0F0BD406D0028FAD002
:1007B00003918DE8E000022127F0E8FA05B0F0BDD2
:1007C00000207047D0B5046D8CB1012B08BF002A02
:1007D00001D30020D0BD1146204628F0DDFF0028BF
:1007E000F7D0204629F058F90028F2D0D0BD446D4A
:1007F000002CEED0204626F00FFD0028E9D0204640
:10080000BDE8D04027F070BBF0B5036D83B00C4657
:100810002BB318460DF1060201A928F03FFCD8B110
:10082000BDF80430BDF8062003B9AAB102F01F06D6
:10083000C3F343155912C2F345177600013D01F584
:10084000EA6103F01F03D21226706571A171237152
:100850006770A27003B0F0BD002003B0F0BD406D22
:100860000028F9D00DF1060201A926F089FBD6E790
:10087000F0B5036D83B00C462BB318460DF106029C
:1008800001A928F0FBFBD8B1BDF80430BDF8062063
:1008900003B9AAB102F01F06C3F343155912C2F3FC
:1008A00045177600013D01F5EA6103F01F03D212FE
:1008B00026706571A17123716770A27003B0F0BDDD
:1008C000002003B0F0BD406D0028F9D00DF1060204
:1008D00001A926F045FBD6E7036D13B15869002145
:1008E0007047436D13B193E80300704718461946EB
:1008F000704700BF036D13B1D86900217047436D85
:1009000013B118695969704718461946704700BFF6
:10091000036D13B1184628F04DBD406D08B126F0A7
:100920008FBB4FF0FF307047036D13B1184628F0AE
:1009300011BE406D08B126F057BC4FF0FF30704734
:10094000036D33B11B7813F0700F14BF012000202A
:100950007047406D30B190F8313013F0500F14BF34
:1009600001200020704700BF8A79A2F150031B06C6
:1009700020D4F0B54B79046D0D798E784F780978D5
:10098000013385B002F26C72DBB244B103918DE8A1
:10099000E0002046042129F017F805B0F0BD406DB5
:1009A0000028FAD003918DE8E000042127F0EEF949
:1009B00005B0F0BD00207047036963B11A680749AC
:1009C00092698A4208D1186D08B128F0F7BF586DB6
:1009D00008B127F06FB8704718461047F5090000B6
:1009E000836C13B1184628F0E9BFC06C08B127F03A
:1009F00061B87047036D13B1184628F0DFBF406D32
:100A000008B127F057B8704703697BB110B41C6870
:100A10000B48E46884420ED1186D10B110BC29F067
:100A200077B8586D20B110BC27F0CEBA00207047BF
:100A3000002010BC70471846234610BC184700BF62
:100A4000C90A0000036973B11A68084952698A42E9
:100A500007D1186D08B128F07DBD586D18B126F08A
:100A6000C3BB184610474FF0FF30704729090000FC
:100A7000036923B310B51968124A8C68944282B096
:100A800014D1186D48B101220DF1070128F092FC34
:100A900090B19DF8070002B010BD586D0028F8D045
:100AA00001220DF1070126F0CBFAF1E718460122E9
:100AB0000DF10701A047EBE74FF0FF30EBE74FF0F8
:100AC000FF30704711090000036D13B1184629F07B
:100AD0001FB8406D08B127F077BA7047836C13B127
:100AE000184629F015B8C06C08B127F06DBA7047E8
:100AF00000B5836C83B08DF8071043B1184601220E
:100B00000DF1070129F004F803B05DF804FBC06C97
:100B10000028F9D001220DF1070127F055FA03B0A2
:100B20005DF804FB10B5036982B08DF80710BBB106
:100B30001968104ACC68944215D1186D30B1012261
:100B40000DF1070128F0E4FF02B010BD586D002838
:100B5000FAD001220DF1070127F036FA02B010BDDC
:100B6000184602B010BD184601220DF10701A0473A
:100B700002B010BDC90A0000026D62B1137803F023
:100B8000080303F0FF0003B3D3695069181A48BF84
:100B90006FF000407047416DC1B191F8313003F002
:100BA000080303F0FF0083B1D1E90423D1E9000178
:100BB000101A30B463EB010100256FF000448D4240
:100BC00008BF844200D2204630BC704708467047B8
:100BD000826C62B1137803F0080303F0FF0003B3E3
:100BE000D3695069181A48BF6FF000407047C16C54
:100BF000C1B191F8313003F0080303F0FF0083B175
:100C0000D1E90423D1E90001101A30B463EB0101EA
:100C100000256FF000448D4208BF844200D2204678
:100C200030BC704708467047006970B30368184AC3
:100C30001B6993420ED1026D6AB1137803F0080369
:100C400003F0FF000BB3D3695069181A48BF6FF067
:100C5000004070471847416DC1B191F8313003F041
:100C6000080303F0FF0083B1D1E90423D1E90001B7
:100C7000101A30B463EB010100256FF000448D427F
:100C800008BF844200D2204630BC704708467047F7
:100C9000790B0000D0B4039C16461F4634B1012CDA
:100CA0001ED0022C0DD00020D0BC7047046DDCB1EA
:100CB000012B08BF002AF6D220461146D0BC28F0EE
:100CC0006BBD036DB3B1DA69B61847F10007012FA8
:100CD00008BF002EE7D231461846D0BC28F05CBDD4
:100CE000036D8BB15A69EFE7406D0028DBD0D0BCB3
:100CF00026F092BA406D0028D5D0D0E9042392198D
:100D00007B41D0BC26F088BA406D0028CBD0D0E91A
:100D1000002392197B41EAE738B50446806D0C4BFD
:100D2000236018B131F0DAFC0023A365236D04F1D0
:100D300018054BB128462AF091F9064BA3602846C6
:100D40002AF08CF9204638BD636D002BF2D1F4E710
:100D5000086303009462030038B50446806D0E4BAF
:100D6000236018B131F0BAFC0023A365236D04F1B0
:100D700018056BB128462AF071F9084BA360284684
:100D80002AF06CF920465C212EF0DAFA204638BDB4
:100D9000636D002BEED1F0E708630300946203005B
:100DA00070B50469244B036005461CB16668013EBA
:100DB00066600EB1284670BD2368204ADB6A934204
:100DC0002CD1A06D10B131F089FCA665236D5BB309
:100DD00004F118002AF042F92C69002CEAD02368AB
:100DE000174A5B6893421CD1A06D164B236018B163
:100DF00031F074FC0023A365236D04F11806BBB128
:100E000030462AF02BF9104BA36030462AF026F921
:100E100020465C212EF094FA284670BD2046984763
:100E2000DAE720469847C5E7636D002BD0D1D3E7BA
:100E3000636D002BE4D1E6E7DC6203006D05000082
:100E4000590D0000086303009462030070B5056942
:100E5000284B036004461DB16E68013E6E602EB1E2
:100E6000204614212EF06CFA204670BD2B68224AD1
:100E7000DB6A934230D1A86D10B131F02FFCAE6522
:100E80002B6D7BB305F118002AF0E8F82569002DD9
:100E9000E6D02B68194A5B68934220D1A86D184BA5
:100EA0002B6018B131F01AFC0023AB652B6D05F1F6
:100EB0001806DBB130462AF0D1F8124BAB60304651
:100EC0002AF0CCF828465C212EF03AFA204614216C
:100ED0002EF036FA204670BD28469847D6E72846B9
:100EE0009847BDE76B6D002BCCD1CFE76B6D002B26
:100EF000E0D1E2E7DC6203006D050000590D00005F
:100F00000863030094620300036A8B4210B523D088
:100F1000C369994200D010BD8369002BFBD072B623
:100F2000194AC369846900211160DB00516803F12B
:100F3000804303F5603321440D2419611460DA689D
:100F4000502122F08002DA60D96062B6006903683D
:100F5000BDE810405B6818470446006903689B6859
:100F6000984794F82430002BD5D004F108002EF0D7
:100F700091F90023E06963602BF0D2F9206ABDE8A3
:100F800010402BF0CDB900BF008003408268002ADA
:100F900036D0816D836F2DE9F04104464868D4F85E
:100FA000AC101B1A002BB8BF5B428B423ADBD4F863
:100FB000B0108B4208DBE06F83425CDB936823F068
:100FC00002039360BDE8F081D4F88830002BF5D09F
:100FD0001168324881421FD95068314DB5FBF3F397
:100FE000091A8B420DD2606901680026012503248D
:100FF00096600968D56013609460BDE8F0410847C9
:101000007047591A0025012403209560D4601160AF
:1010100090601360BDE8F0812149B1FBF3F31360E8
:10102000BDE8F081D4E92467D4F8A80000FB03F000
:10103000321847F100031046194630F0CBFE2FF06E
:101040006BF831F0E1F8A2680346D8B1002ABFD1AD
:10105000144B134D1B68B5FBF0F51BB102210120A9
:101060009847A2680020012103239060D160156099
:101070009360BDE8F081C31AD4E92667D4F8A800CC
:10108000013BD3E7002A99D1064B1B68002B95D072
:10109000022101209847A26890E700BF7F3202003A
:1010A0000051250244A0FF1F2DE9F041856FC76F55
:1010B000866D044629463846736831F05DF800288D
:1010C0003BD0284631F0A0F8054694F890300BB19B
:1010D000002D7DD0B368AB422DD0002D3368B4BF56
:1010E0004FF0FF3201229A4215D004F1280101206D
:1010F00008E013685B42012B13600BBF126B536B4C
:101100001360186051F8042F002AF2D1636F03EBCB
:101110004303DB0044D185EAE572A2EBE572A368E4
:1011200022BB002B00F085809A6822F002029A60B0
:10113000B560BDE8F081BDE8F081D4F88C80384618
:10114000414630F07DFD00210746404631F03CF835
:10115000394600282ED0284631F036F800282ED106
:101160002846E06731F050F80546AEE7002B4AD03C
:1011700019683548814224D95868344FB7FBF2F2D8
:10118000091A8A4235D26069002601689E600127EB
:101190000326DF6009681A609E608847A66DC7E76E
:1011A000013BFDD185EAE572A2EBE572A368002A56
:1011B000B7D0DBE7284630F0E9FF0028D0D038462A
:1011C000CFE72249B1FBF2F21A60B560BDE8F081C9
:1011D00004F10C002EF05EF8206AA5602BF0A0F858
:1011E000606A2BF09DF8A36D9D6084F89050BDE877
:1011F000F081511A0027012403209F60DC601960F0
:1012000098601A6094E71249104FD1F80080B7FB3C
:10121000F2F7B8F1000F04D002210120C047A36803
:10122000A66D0020012103229860D9601F609A609A
:101230007EE7074B1B68002B3FF476AF02210120AD
:101240009847A368A66D6FE77F3202000051250220
:1012500044A0FF1F70B5044608460D4632F0F0FA70
:1012600023680246294620465B68BDE8704018475F
:1012700038B50A22002305462EF0B4F80446284665
:101280002EF09CF8204438BD10B509211E482DF0E1
:1012900005FD1E482EF092F8FE211D4825F018FB92
:1012A00018BB0A211A4825F013FB98B909211848E0
:1012B000184C25F00DFB18BB20600C2116482DF0B2
:1012C000EDFC216811482EF0CDF81048BDE8104023
:1012D0002EF074B80F4C11480A23194623602DF0E4
:1012E000DDFC0A482EF06AF8E7E70A4C0C480123B7
:1012F000092123602DF0D2FC04482EF05FF8DCE7D2
:1013000008480923E9E700BFBC6303006488FF1FA6
:10131000709BFF1FFC99FF1FEC630300D463030065
:10132000C8630300E063030070B586B0044603ADF4
:101330000DF11706236820465B699847C3B2042B5A
:1013400002D0FF2B2BD028700135B542F2D103A873
:1013500031F064F904460D46184804212DF09EFC36
:1013600003A832F06DFA014603A82DF097FC14484B
:101370002EF024F8072113482DF090FC0421009151
:1013800022462B460E482EF077F80D482EF016F820
:101390002046294606B070BD23685B6998472368DC
:1013A00020461B69984700282046F5DC03A831F049
:1013B00035F903A831F032F906B070BDFC630300C3
:1013C0006488FF1F0464030001280BD0032806D0A3
:1013D00010B10020054970470548FFF7A5BF054833
:1013E000FFF7A2BF0448FFF79FBF00BF0000F0BF98
:1013F0006488FF1F3C88FF1F2888FF1F013970B5D4
:10140000044603296BD8DFE801F02D201102354D89
:101410006B6D002B53D0012B61D1EB6DA86D00FBE0
:1014200003F030F0BDFC696E064624E02D4D6B6B79
:10143000002B34D0012B52D1EB6BA86B00FB03F0D7
:1014400030F0AEFC696C064615E0264DD5F8B83094
:10145000CBB96B6A286A00FB03F030F0A1FCA96AE3
:10146000064608E01F4D2B69E86800FB03F030F0EA
:1014700097FC69690646204630F09EFD01463046DD
:1014800030F0E6FC70BDD5F8C030D5F8BC0000FBEC
:1014900003F030F085FCD5F8C4100646EBE7AB6BE3
:1014A000E86B00FB03F030F07BFC296C30F0D0FCE3
:1014B0000D490646A86C30F0CBFC0146DBE7EB6D2E
:1014C000A86D00FB03F030F06BFC296E30F0C0FC1F
:1014D00005490646A86E30F0BBFC0146CBE700206C
:1014E00070BD00BFBC96FF1FDB0FC9402DE9F8435C
:1014F000284F3E68804689463046002130F046FE3F
:10150000002843D1244D2C680021204630F03EFEB7
:1015100010B104F100442C603146304630F098FCA4
:1015200021460646204630F093FC0146304630F016
:1015300087FB2FF0E3FF2EF035FD30F02BFB3968F1
:10154000064630F039FD29680446304630F034FD57
:101550000646484630F028FC0146304630F078FC1C
:101560002FF0CCFF2EF092FC30F014FB28604046A8
:1015700030F01AFC214630F06BFC2FF0BFFF2EF04C
:1015800085FC30F007FB3860BDE8F88306F10046C3
:101590003E60B7E78095FF1F189BFF1F38B5334BA0
:1015A0001B68013B0A2B60D8DFE803F026363F5F5B
:1015B0005F060606064F36002D4B2E4D18682E4C42
:1015C000FFF702FF30F09EFA2C4A03462C481168C0
:1015D000C3624C226B6163642BF0FEFA294B2846F0
:1015E000196860222BF0F8FA274B204619686C2204
:1015F000BDE838402BF0F0BA1D4B244C1868FFF7BB
:10160000E3FE30F07FFA224B6061196820467822B1
:10161000BDE838402BF0E0BA154B1E4C1868FFF7B8
:10162000D3FE30F06FFA1C4BEEE7114B1B4C1868E1
:10163000FFF7CAFE30F066FA194B60611968204660
:101640003422BDE838402BF0C7BA094B154C186856
:10165000FFF7BAFE30F056FA134BA0621968204625
:101660007022BDE838402BF0B7BA38BD6C87FF1F39
:101670008087FF1F5C96FF1FE898FF1F7087FF1F82
:10168000CC97FF1F9887FF1F8487FF1FE095FF1FE0
:101690008C87FF1FBC94FF1F5C87FF1FB498FF1F40
:1016A0006487FF1F109AFF1F9087FF1F934B1B68D3
:1016B000013B10B50A2B6DD8DFE803F01121324849
:1016C0006C060606065621008D4C2368013B032B51
:1016D0006CD8DFE813F0C400B800AC006000894BA0
:1016E0001868FFF771FE30F00DFA874A936D013BE1
:1016F0000446032B4ED8DFE803F091887F76814BB8
:101700001868FFF761FE30F0FDF9804A936D042BF5
:1017100061D8DFE813F05F00E000DE00DC00DA00F3
:101720007B4C2368032B00F0D880042B06D1754B2B
:101730001868FFF749FE30F0E5F9E061754B744831
:1017400019683422BDE810402BF046BA724C236869
:10175000013B0D2B1ED8DFE803F0AFA69D8E1D1DAB
:101760001D1D1D1DAFA69D8E6C4C636C012B00F0E2
:10177000BC80022B00F0E680032B00F0EB80042BF2
:1017800000F0F080664B654819687022BDE8104093
:101790002BF022BA10BD5B4B1868FFF715FE30F036
:1017A000B1F9604A604BE063506258655F4B544842
:1017B00019684C222BF010FA5D4B5A4819686022C8
:1017C0002BF00AFA5B4B584819686C22BDE81040B0
:1017D0002BF002BA5061584B4C4819687822BDE88A
:1017E00010402BF0F9B9554B5462474819687822DC
:1017F000BDE810402BF0F0B9504B14624248196814
:101800007822BDE810402BF0E7B94C4BD4613E483C
:1018100019687822BDE810402BF0DEB9474B94617F
:10182000394819687822BDE810402BF0D5B9354BFE
:101830001868FFF7C9FD30F065F93A4A3A4BA063E2
:1018400010621865B2E72F4B1868FFF7BDFD30F046
:1018500059F9344A344B6063D061D864A6E7294B08
:101860001868FFF7B1FD30F04DF92E4A2E4B20637A
:10187000906198649AE7234B1868FFF7A5FD30F054
:1018800041F92F4B2063196823485422BDE81040CA
:101890002BF0A2B91B4B1868FFF796FD30F032F918
:1018A000274B6062EFE7174B1868FFF78DFD30F0AC
:1018B00029F9234BA061E6E7124B1868FFF784FD76
:1018C00030F020F91E4BE060DDE7506283E71062E4
:1018D00081E7D0617FE790617DE70A4B1868FFF7E9
:1018E00073FD30F00FF9A06128E7064B1868FFF789
:1018F0006BFD30F007F9E06244E700BF6C87FF1F23
:10190000CC97FF1F8087FF1FE095FF1FBC94FF1F30
:10191000B498FF1F6487FF1F5894FF1F109AFF1F82
:101920009087FF1F5C96FF1FE898FF1F7087FF1FBF
:101930009887FF1F8487FF1F5C87FF1F8C87FF1F0F
:101940002487FF1F0B4B1868FFF73EFD30F0DAF8D5
:10195000206317E7074B1868FFF736FD30F0D2F821
:1019600060630FE7034B1868FFF72EFD30F0CAF8ED
:10197000A06307E78087FF1F70B5684D2B686A6812
:10198000064602FB03F00C4630F00AFAA96830F074
:101990005FFA2FF0B3FD2EF079FA30F0B3F8611E44
:1019A00004296ED8DFE801F0182E435803005C4C80
:1019B0002368E660012B65D030F0F6F9314630F04F
:1019C000FBFA30F047FCA060564B554819681022CE
:1019D000BDE870402BF000B9534C2368E660012B42
:1019E00000F08C8030F0E0F9314630F0E5FA30F06C
:1019F00031FCA0604D4B4C4819681022BDE8704086
:101A00002BF0EAB84A4C2368E660012B67D030F02F
:101A1000CBF9314630F0D0FA30F01CFCA060454BD9
:101A2000434819681022BDE870402BF0D5B8424CED
:101A30002368E660012B43D030F0B6F9314630F030
:101A4000BBFA30F007FCA0603C4B3B481968102201
:101A5000BDE870402BF0C0B8394C2368E660012B1C
:101A60001FD030F0A1F9314630F0A6FA30F0F2FB89
:101A7000A060344B324819681022BDE870402BF04A
:101A8000ABB870BD30F090F92F490546304630F0C4
:101A900093FA0146284630F0DBF930F0DBFBA0601A
:101AA00092E730F081F928490546304630F084FA53
:101AB0000146284630F0CCF930F0CCFBA060D8E7E6
:101AC00030F072F920490546304630F075FA01468B
:101AD000284630F0BDF930F0BDFBA060B4E730F02F
:101AE00063F919490546304630F066FA0146284642
:101AF00030F0AEF930F0AEFBA06090E730F054F972
:101B000011490546304630F057FA0146284630F074
:101B10009FF930F09FFBA0606CE700BFBC96FF1FF1
:101B2000D89AFF1F5087FF1FB49AFF1F4087FF1FDF
:101B3000EC92FF1F4487FF1F0C93FF1F4887FF1F76
:101B4000C89AFF1F4C87FF1F0000B4432DE9F041E6
:101B5000684CD4F8D830A3F10A021D2A804640F21E
:101B6000898023686068644A6449654E654D00FB5E
:101B700003F0002333600B60136030F011F9A168AB
:101B8000614E30F065F9E96830F016FA07464046D4
:101B900030F00AF90146384630F00EFA2FF0AEFC6C
:101BA0002EF074F92FF0AEFF2B683060013B032B51
:101BB00022D8DFE803F0412C0223636BAD694D4C62
:101BC000002B5CD1A36BE06B504E00FB03F030F0B8
:101BD000E7F8216C30F03CF94D490746A06C30F035
:101BE00037F90146284630F0E7F90146384630F02B
:101BF0002FF930F009FB3060BDE8F081636DAD690D
:101C00003C4C002B51D0012B60D0BDE8F081D4F8C2
:101C1000B830A869374C002B35D1A16A3B4D30F064
:101C2000CBF90646606A30F0BBF80146304630F02A
:101C30000FF90646206A0EE06169A869334D30F05D
:101C4000BBF90646206930F0ABF80146304630F06B
:101C5000FFF80646E06830F0A3F80146304630F061
:101C6000F7F82FF04BFC2EF011F92FF04BFF286006
:101C7000BDE8F081D8B200212BF010F971E7012BFB
:101C80002ED0BDE8F081D4F8C410204D30F094F986
:101C90000646D4F8C00030F083F80146304630F0F4
:101CA000D7F80646D4F8BC00D5E7E36DA06D174E13
:101CB00000FB03F030F074F8216E30F0C9F81449DD
:101CC0000746A06E30F0C4F801468BE7E36DA06DC7
:101CD0000E4E00FB03F030F063F8616E074681E7BB
:101CE000E36BA06B094E00FB03F030F059F8616C18
:101CF000074677E7BC96FF1FB093FF1F5499FF1F5D
:101D00001C93FF1FE898FF1FF89AFF1FB094FF1F56
:101D1000DB0FC940094B1B68012B0BD0032B05D0EF
:101D200003B17047014606482DF022BB0146054825
:101D30002DF01EBB014604482DF01ABB8087FF1F03
:101D40006488FF1F3C88FF1F2888FF1F70B5064668
:101D500088B00D4632B1AC4BD3F8CC40012C00F02A
:101D6000BB800022A94C2368029302992368019347
:101D7000019B5B1A092BF9D9042E27D8DFE806F05E
:101D80003466588A0300002D00F0D2809E4B93F8F1
:101D9000A0100F2081F001012BF080F89C4904A8CD
:101DA0002DF0ACFD002104A8FFF7B4FF04A82DF02E
:101DB00065FD984904A82DF0A1FD04A80021FFF7B6
:101DC000A9FF04A82DF05AFD934B1B6855B122685A
:101DD000924B049204991A6823680393039B5B1A3D
:101DE0009A42F9D808B070BD002D00F0CD80864B26
:101DF00093F89C10042081F001012BF04FF88849E2
:101E000004A82DF07BFD002104A8FFF783FF04A8A0
:101E10002DF034FD7F4904A82DF070FD04A80021A9
:101E2000FFF778FF04A82DF029FD7E4B1B68CDE756
:101E3000002D00F08980744B93F89E10162081F0DD
:101E400001012BF02BF804A87749A9E7002D00F039
:101E5000BB806D4B93F89D100E2081F001012BF09B
:101E60001DF8724904A82DF049FD002104A8FFF7D0
:101E700051FF04A82DF002FD664904A82DF03EFD97
:101E800004A80021FFF746FF04A82DF0F7FC684BDB
:101E90001B689BE76DB35C4B93F89F10112081F09A
:101EA00001012AF0FBFF634904A82DF027FD002162
:101EB00004A8FFF72FFF04A82DF0E0FC554904A863
:101EC0002DF01CFD04A80021FFF724FF04A82DF02D
:101ED000D5FC594B1B6879E7102158482CF0DEFEE1
:101EE000214657482DF0BEFA55482DF067FA224694
:101EF00038E7002AEDD1444B112093F89F102AF0C7
:101F0000CDFF04A84F492DF0F9FC294604A8FFF79E
:101F100001FF04A82DF0B2FC04A83E492DF0EEFC10
:101F200004A82946FFF7F6FE04A82DF0A7FCD0E789
:101F3000002A7FF449AF344B0F2093F8A0102AF009
:101F4000ADFF04A840490AE0002A7FF43DAF2E4BC4
:101F5000162093F89E102AF0A1FF3C4904A82DF00A
:101F6000CDFC294604A8FFF7D5FE04A82DF086FC79
:101F700004A828492DF0C2FC04A82946FFF7CAFE90
:101F800004A82DF07BFC1FE7002A7FF44EAF1E4B08
:101F9000042093F89C102AF081FF04A82C492DF00E
:101FA000ADFC294604A8FFF7B5FE04A82DF066FC99
:101FB00004A818492DF0A2FC04A82946FFF7AAFEA0
:101FC00004A82DF05BFC30E7002A7FF460AF0E4BD5
:101FD0000E2093F89D102AF061FF04A81D492DF0F2
:101FE0008DFC294604A8FFF795FE04A82DF046FCB9
:101FF00004A808492DF082FC04A82946FFF78AFEB0
:1020000004A82DF03BFC42E7BC96FF1F7CA0FF1FFD
:10201000246503004064030090F00F406887FF1FB1
:102020002064030010F00F40A46403006464030004
:10203000D0F00F40E464030050F00F400C64030044
:102040006488FF1F0465030044650300C464030043
:1020500044640300846403002DE9F041A04B1B7825
:1020600084B0002B52D09F4E6C469F499F4FA04D8D
:10207000DFF8B08220462DF041FC00212046FFF71A
:1020800049FE20462DF0FAFB316820462DF036FC43
:1020900000212046FFF73EFE20462DF0EFFB95493C
:1020A00020462DF02BFC00212046FFF733FE204672
:1020B0002DF0E4FB316820462DF020FC0021204665
:1020C000FFF728FE20462DF0D9FB3C6820462FF074
:1020D0006BFE2B680646686800FB03F02FF060FE7D
:1020E000A9682FF0B5FE014630462FF065FF824902
:1020F0002FF0AEFE814BC8F800001B68013B032B9C
:1021000000F2EB80DFE803F0714C2B0A7C4B1D786A
:102110006C46002D00F0A680724EA6E76B6D744CE5
:10212000012B00F2D780774E30682FF03DFE616EB4
:102130002FF08EFEE36D8046A06D00FB03F02FF0C4
:102140002FFE014640462FF037FF04466E4B01221A
:10215000002104201C60FFF7F9FD3C685FE06B6B19
:10216000634C012B00F2B380664E30682FF01CFEEA
:10217000616C2FF06DFEE36B8046A06B00FB03F0FB
:102180002FF00EFE014640462FF016FF04465E4B30
:102190000122002103201C60FFF7D8FD3C683EE0CF
:1021A000584E534C30682FF0FFFDD5F8B830002B57
:1021B00000F08680D4F8C4102FF04AFED4F8C03066
:1021C0008046D4F8BC0000FB03F02FF0E9FD014687
:1021D00040462FF0F1FE4C4B044601220021022024
:1021E0001C60FFF7B3FD3C6819E0464E464C306872
:1021F0002FF0DAFD69692FF02BFE2B698046E86825
:1022000000FB03F02FF0CCFD014640462FF0D4FE3A
:102210000122206000211046FFF798FD3C683B4BEF
:1022200032681B683A493B48DFF8FCE03A4F002629
:10223000524264425B420A600460314630460122E9
:10224000CEF800303E60FFF781FDD5F8D800A0F150
:102250000A031D2B03D8C0B201212AF01FFE04B0CF
:10226000BDE8F08168462D491E4E2DF047FB2946FA
:102270006846FFF74FFD68462DF000FB3168684661
:102280002DF03CFB29466846FFF744FD68462DF0DB
:10229000F5FA684622492DF031FB29466846FFF7DA
:1022A00039FD68462DF0EAFA316868462DF026FBC4
:1022B00068462946FFF72EFD68462DF0DFFAD4E682
:1022C000A16A2FF0C5FD636A8046206A7BE700247F
:1022D0000C4E5CE700240B4E38E70A4E9FE700BF28
:1022E0006C9BFF1FA487FF1F8C6503001C93FF1FBF
:1022F000BC96FF1FA06503000000B443E898FF1FD1
:102300005594FF1F5499FF1FF899FF1FB093FF1FAB
:10231000AC93FF1FA893FF1FDC95FF1F64650300AC
:1023200078650300F099FF1FF09AFF1F70B506460D
:1023300082B00446002520462FF066FF2FF034FDC2
:1023400021462FF019FF1B4930B920462FF080FDA0
:102350000135062D0446EED1174B1B68012B1CD00E
:10236000032B0ED00BB102B070BD30462FF0C6F873
:10237000EDB202460B46009510482DF07DF802B0F4
:1023800070BD30462FF0BAF8EDB202460B4600950C
:102390000B482DF071F802B070BD30462FF0AEF84A
:1023A000EDB202460B46009506482DF065F802B0E6
:1023B00070BD00BF000020418087FF1F6488FF1FA1
:1023C0003C88FF1F2888FF1F064B1B68012B07D086
:1023D000032B03D003B170472CF0E4BC2BF0D6BC28
:1023E0002BF0BCB88087FF1FF8B50D4F0D4E0E4D7A
:1023F0000446014638462CF0BBFF38462CF0DEFF81
:10240000214630462CF0B4FF30462CF0D7FF214651
:1024100028462CF0ADFF2846BDE8F8402CF0CEBF92
:102420006488FF1F2888FF1F3C88FF1F012808D0F1
:10243000032804D008B1002070472CF0C9BB2BF052
:10244000FDBC2BF05DB900BF38B5094C2068FFF723
:10245000EDFFC5B202E02068FFF7E8FF2BF03CF982
:102460000028F8DCFEF716F90028F4DC284638BD11
:102470008087FF1F08B52BF02FF900282EDD1B4B9E
:102480001868FFF7D3FF1A4BC0B25328187001D059
:10249000002008BD002108460122FFF757FC154B1C
:1024A0001B68013B032B1FD8DFE803F002070C1168
:1024B000012200210220FFF749FC01220021022015
:1024C000FFF744FC012200210320FFF73FFC01221B
:1024D00000210420FFF73AFC012008BDFEF7DAF8DE
:1024E0000028CCDA002008BD012008BD8087FF1F2E
:1024F0008595FF1FE898FF1F2DE9F8431A4D2B68BB
:10250000092B2FD0192B2BD0032B22D0174EDFF8FD
:102510006890DFF86080164F002407E0192B15D073
:10252000032B00D1E05501340D2C0DD03068FFF79E
:102530007DFFC0B2FF2807D02B68092BEED104F82D
:10254000090001340D2CF1D1BDE8F88304F808002E
:10255000E9E7074B00221A605A609A601A73D5E7C0
:10256000044BF7E7044BF5E76C87FF1F8087FF1FDD
:10257000009AFF1F2093FF1FA498FF1F2DE9F04F23
:10258000A1B0A049A04C0026054603A82DF0B6F93D
:1025900033460CA89D4A9E49266028F049FE1E9BA2
:1025A000002B00F08B815C202CF0C6FE0646994B78
:1025B0009DF834000E9A9849336000279DF83C300E
:1025C00030730DF14008B16032614146337506F158
:1025D0001800776028F014FD73689049DFF868A24E
:1025E000B76501334FF47A728DF820708DF828703A
:1025F0000B96B16073600992CDF81CA04046DFF8DD
:102600004CB2CDF830B028F029FD0B98002800F02E
:10261000CD800368824A1B6B934240F06281036D58
:10262000002B00F0BF807F4A136802930299136861
:102630000193019B5B1A632BF9D900282AD07A4FAA
:10264000714E6FF000484FF0000903681B69BB42F0
:1026500061D1036D002B37D01A7812073AD5DA69A9
:102660005869101A01D4002834D078230A2207A907
:102670000CA82CF0FDFF0CA903A82DF0A3F90CA8C1
:102680002DF0FCF82368AB4224D00B980133336063
:102690000028DAD10398654B002808BF18462FF0B0
:1026A000BDFF06460F460B9CCDF81CA024B1656803
:1026B000013D6560002D3ED003A82DF0DFF83046C7
:1026C000394621B0BDE8F08F416D19B191F8313034
:1026D0001B0722D40B9C002CDCD02368544EDB6AF1
:1026E000B34240F0E880A06D18B12FF0F7FF00234F
:1026F000A365236D002B00F0FA8004F1180028F088
:10270000ADFC0B9D6C68013C6C60002C00F0A0805F
:1027100000230B93BEE79847A5E7D1E90423D1E94D
:102720000001101A63EB0101894508BF80459AD268
:102730006FF0004097E723683D4ADB6A934240F020
:10274000DB80A06D10B12FF0C9FFA565236D002BB4
:1027500000F0DB8004F1180028F080FC0B9C002CBA
:10276000AAD02368334A5B68934240F0C880A06DCA
:10277000284B236018B12FF0B1FF0023A365236D10
:1027800004F11805002B00F0C880284628F066FCEC
:10279000C4F808B0284628F061FC20465C212CF0E3
:1027A000CFFD89E7436D002B7FF43DAF224B2349DA
:1027B00001220CA81A702DF0A1F800210CA8FFF737
:1027C000A9FA0CA82DF05AF82220FFF7FDFD1C49AC
:1027D0000CA82DF093F800210CA8FFF79BFA0CA889
:1027E0002DF04CF8174B0CA819682DF087F8002134
:1027F0000CA8FFF78FFA0CA82DF040F80026002750
:1028000051E700BFAC940300809AFF1F009AFF1F9E
:10281000749BFF1F0863030070620300B86203002B
:10282000750400007CA0FF1F790B00004C9803008A
:102830006D050000590D00008495FF1FB46503006D
:10284000D0650300A087FF1FDC62030094620300D1
:102850002B68DB6AB34255D1A86D10B12FF03EFF53
:10286000AC652B6D002B5DD005F1180028F0F6FB50
:102870000B9C002C3FF44CAF23682E4A5B689342BC
:1028800048D1A06D2C4B236018B12FF027FF0023F7
:10289000A365236D04F11805002B47D0284628F0C6
:1028A000DDFBC4F808B0284628F0D8FB20465C21A0
:1028B0002CF046FD2CE72046984722E71F9B002B73
:1028C0007FF471AE4FF47A72DFF870A08DF820308B
:1028D0008DF828300B930992CDF81CA00DF140081B
:1028E0008CE6984700283FF461AF0B989BE6636D38
:1028F000002B7FF402AF04E7204698472EE72046DE
:102900009847D9E628469847B2E7636D002B7FF4D5
:1029100021AF23E720469847FAE6636D002B7FF44A
:1029200034AF35E76B6D002B9ED1A1E7636D002BB3
:10293000B4D1B6E7590D000008630300DC62030060
:102940002DE9F04FADF2A45DBA49019002A82CF038
:10295000D5FFB94906A82CF0D1FF40F2145200214E
:1029600023A830F07BFA00230FA8B44AB44928F01A
:102970005FFC219B002B00F028845C202CF0DCFC09
:102980000446B04D9DF84000119A9DF84830AE497C
:10299000256013AE00252073A16022612375656058
:1029A00004F11800314628F02BFB6368A74AA5659F
:1029B0000133A2606360DFF8C892CDF83C903046E6
:1029C00028F04CFBA24D4FF0000A002C00F0F380E1
:1029D0002368A04ADB6B934240F0AD8200231A4685
:1029E0004FF47A7B994F8DF8403004F1180130464E
:1029F0008DF8483021932293CDF844B00F9728F0FA
:102A000081FB219A002A00F0EE825C202CF094FCDD
:102A100083464FF000089DF840001199894B8A4A7F
:102A20009DF848E08BF80C00CBF81010CBF8003084
:102A300031460BF11800CBF808208BF814E0CBF8E6
:102A4000048028F0DDFADBF80410CBF808700131BF
:102A50004FF47A70CBF858808DF82C808DF8348044
:102A6000CDF838B00A95CBF804100C903046CDF86C
:102A70003C9028F0F3FA0E9F002F00F00B843B6887
:102A8000754A5B6B934240F09F81B96D002900F05D
:102A9000D1820FA82CF032FF0E98002800F09C8005
:102AA00002686E49136B8B4240F05981036D002B15
:102AB00000F07481926B6A498A4240F089811B78E8
:102AC00013F0700F14BF01200020002800F04F8188
:102AD000DDF838B0BBF1000F23D0DBF80020614FE8
:102AE000D26ABA4240F06D81DBF8580020B12FF075
:102AF000F5FD0022CBF85820DBF85020002A00F02A
:102B00006C820BF1180028F0A9FADDF838B0DBF878
:102B10000430013BCBF80430002B00F0E3800023AD
:102B20000E930FA82CF0AAFE0E9F0A95002F3FF4DB
:102B30004CAF7B68013B7B60002B7FF446AF3A686B
:102B40004849D26A00938A4240F08D82B86D18B12C
:102B50002FF0C4FD009BBB653B6D002B00F01A837A
:102B600007F1180028F07AFA0E9F002F3FF42DAFDE
:102B70003B683D4A5B68934240F00383B86D314B3C
:102B80003B6018B12FF0AAFD0023BB653B6D07F138
:102B9000180B002B00F00883584628F05FFAC7F89E
:102BA0000890584628F05AFA38465C212CF0C8FBA9
:102BB000002C7FF40DAF4FF47A732C498DF82C4024
:102BC0000FA88DF834400A950E940C932CF096FEC5
:102BD0000E9800287FF464AF0FA82CF04FFE0E9ED5
:102BE0000A952EB17568013D7560002D00F0728266
:102BF0001F49204D204E0FA82CF080FE00210FA869
:102C0000FFF788F80FA82CF039FE50462FF0CCF8CB
:102C100000210746FFF78AFB29680FA82CF06EFEFB
:102C200000210FA8FFF776F80FA82CF027FE134914
:102C30000FA827E0E4650300EC650300F4650300DA
:102C4000749BFF1F0863030070620300B8620300F7
:102C5000DC620300950500002907000075040000F0
:102C6000410900006D050000590D0000AC940300FF
:102C7000F8650300A487FF1FA087FF1F18660300E5
:102C8000946203002CF03AFE00210FA8FFF742F8EF
:102C90000FA82CF0F3FD38460021FFF747FB296809
:102CA0000FA82CF02BFE00210FA8FFF733F80FA878
:102CB0002CF0E4FD019A02EB4207134602EB870772
:102CC00023AA174403F1FF380125AB1E08EB050AC0
:102CD000052B7FD8DFE813F0F700F500F300F100D3
:102CE000BA003501DBF800100093C96AB94240F020
:102CF000B781DBF8580020B12FF0F0FC009BCBF837
:102D00005830DBF85030002B00F03E820BF11800F9
:102D100028F0A4F90E9F002F3FF401AF3B68B84A9A
:102D20005B68934240F02A82B86DB64B3B6018B1A5
:102D30002FF0D4FC0023BB653B6D07F1180B002B73
:102D400000F02D82584628F089F9C7F808905846B7
:102D500028F084F938465C212CF0F2FADFE6984737
:102D600000283FF439AF0E98002840F0888202A96D
:102D70000FA82CF0D5FE0028BFF6AAAE06A90FA812
:102D80002CF0CEFE0028BFF6A3AEBAF1620F40F3DE
:102D9000DB81DDF838B00AF1010A9BE6436D002BB8
:102DA0003FF41AAF926B984B9A4211D1436D002BAE
:102DB000DDD093F8313013F0500F14BF0120002004
:102DC00083E658469047A0E638469847014660E6B5
:102DD00090477AE68D490FA82CF090FD00210FA8AE
:102DE000FEF798FF0FA82CF049FD89490FA82CF099
:102DF00085FD00210FA8FEF78DFF0FA82CF03EFDEA
:102E000039460FA82CF07AFD00210FA8FEF782FFAB
:102E10000FA82CF033FD384630F012FD014638463D
:102E20002BF03CFF7B482CF0C9FA31680FA82CF03E
:102E300065FD00210FA8FEF76DFF0FA82CF01EFD09
:102E4000072D00F0BA8001350D373EE772490FA813
:102E50002CF054FD00210FA8FEF75CFF0FA82CF00A
:102E60000DFD6B490FA82CF049FD00210FA8FEF7BE
:102E700051FF0FA82CF002FD39460FA82CF03EFDA3
:102E800000210FA8FEF746FF0FA82CF0F7FC3846EC
:102E900030F0D6FC014638462BF000FF5D482CF0A0
:102EA0008DFA31680FA82CF029FD0FA80021FEF73C
:102EB00031FF0FA82CF0E2FCC5E75849C7E7584995
:102EC000C5E75849C3E758490FA82CF017FD002162
:102ED0000FA8FEF71FFF0FA82CF0D0FC4C490FA83D
:102EE0002CF00CFD00210FA8FEF714FF0FA82CF00A
:102EF000C5FC39460FA82CF001FD00210FA8FEF7F4
:102F000009FF0FA82CF0BAFC384630F099FC0146B6
:102F100038462BF0C3FE3F482CF050FA31680FA81A
:102F20002CF0ECFC00210FA8FEF7F4FE0FA82CF00B
:102F3000A5FC3E498BE7002221460AA898470E9F30
:102F40009AE53B490FA82CF0D9FC00210FA8FEF709
:102F5000E1FE0FA82CF092FC2D490FA82CF0CEFC1E
:102F600000210FA8FEF7D6FE0FA82CF087FC0AEB75
:102F70004A030AEB830A23AB9A4451460FA82CF06C
:102F8000BDFC00210FA8FEF7C5FE0FA82CF076FCB3
:102F9000504630F055FC014650462BF07FFE1D4850
:102FA0002CF00CFA31680FA82CF0A8FC0FA8002117
:102FB000FEF7B0FE0FA82CF061FC24B16568013D5E
:102FC0006560002D52D006A82CF058FC02A82CF009
:102FD00055FC0DF2A45DBDE8F08FDBF85420002A0B
:102FE0007FF48FAD91E5229A002A7FF40EAD8DF823
:102FF0002C20CDF830B08DF834200A950E9235E5AE
:10300000590D000008630300410900003066030009
:10301000486603006488FF1FC4660300AC660300B3
:10302000946603007C6603004C660300646603003C
:10303000DC6603004FF4807000912FF047FBB86509
:1030400000287ED0009901703B6D002B00F0B3800A
:1030500001464FF48072184627F00AFEB96D18E554
:103060005846884756E6384690477DE523688B4AA0
:10307000DB6A934240F0B680A06D10B12FF02EFBBA
:10308000A565236D002B00F0D68004F1180027F011
:10309000E5FF2368824A5B68934240F0B180A06DEF
:1030A000804B236018B12FF019FB0023A365236D1B
:1030B00004F11805002B00F0C380284627F0CEFF4E
:1030C000C4F80890284627F0C9FF20465C212CF060
:1030D00037F978E73368714ADB6A934240F08580BC
:1030E000B06D10B12FF0FAFAB565336D002B00F01A
:1030F000828006F1180027F0B1FF0E9D002D3FF4ED
:1031000077AD2B68664A5B68934271D1A86D654BB9
:103110002B6018B12FF0E2FA0023AB652B6D05F19F
:103120001806002B00F09180304627F097FFC5F875
:103130000890304627F092FF28465C212CF000F9D9
:1031400056E55949B965A4E40AEB4A07DDF838B0F9
:103150000AEB870723AB1F44BBF1000F29D0DBF834
:1031600000205249526B8A4236D1DBF858100029B0
:1031700049D038460D2230F021FC0CE638469847FD
:10318000CDE43846984720E4DBF85430002B7FF438
:10319000BDADBFE57B6D002B7FF4E2ACE4E47B6D5D
:1031A000002B7FF4CFADD0E57B6D002B7FF4F4AC2A
:1031B000F5E43F49DDE77B6D2BB101464FF48072AA
:1031C000184625F099FBB96D63E4229C002C7FF42E
:1031D000D4AB13AEFFF7EFBB58469047DDF838B0DD
:1031E0000146C6E72046984753E73046984784E7AC
:1031F00028469847FCE4736D002B7FF47AAF7CE798
:1032000020469847DFE64FF4807000912FF05EFA79
:10321000CBF85800F0B100990170DBF85020EAB10A
:10322000014610464FF4807227F022FDDBF858105B
:10323000DDF838B09DE7636D002B7FF426AF28E7FB
:10324000636D002B7FF439AF3AE76B6D002B7FF491
:103250006BAF6CE71449CBF858108AE7DBF85420C1
:1032600052B1014610464FF4807225F045FBDBF861
:103270005810DDF838B07CE7DBF8581079E70268C1
:103280000C4B926B9A427FF4A3AD036D002B7FF43D
:1032900016AC8BE50649FFF7FCBB00BF6D050000CF
:1032A000590D000008630300E492FF1F2907000086
:1032B000AC940300410900002DE9F04FA5B0AC49E2
:1032C000019007A82CF01AFB88202CF037F808236F
:1032D000102280E80C00C118074603910C4600F14B
:1032E00088052046002110342CF008FBA542F8D1B7
:1032F000002310A89F4AA04927F09AFF229B002B89
:1033000000F03A845C202CF017F805469DF8441034
:103310009DF84C3001732B75984B129A2B6000244A
:10332000974B2A6100F1180B14A96C60AB605846EA
:1033300027F066FE6B68AC6501336B60914BAB6048
:1033400014A8914B109327F089FE6C68002C00F0B4
:103350009B832B68DFF860921A6B4A4540F0CB8361
:103360002A6D002A00F0E7839B6A884A934240F066
:10337000E783019B002B00F0C380019B13F106083B
:1033800000F1AF800024DFF834A2029405972B6887
:10339000DB6B534540F0118300231A464FF47A76D5
:1033A000594614A8774F8DF844308DF84C3022934D
:1033B00023931097129627F0A5FE229B002B00F076
:1033C00006835C202BF0B8FF6C490160064600279D
:1033D0009DF84430129A9DF84CE06949B16033730E
:1033E000326114A9183086F814E0776027F008FEDF
:1033F00072686749634BB36001324FF47A70B76506
:103400008DF830708DF838700F9672600D900B91BA
:103410005D4B109314A827F021FE21465D482CF047
:1034200021F802215C482BF039FC0F9E002E00F0A1
:1034300005823368594A5B6B934240F07382B76DE3
:10344000002F00F0D882384630F0FAF901463846AD
:103450002BF024FC4F482BF0B1FF0F9F002F00F002
:10346000EB8139684E488A6B824240F03B813A6D6D
:10347000002A00F09682127812F0700F14BF012219
:103480000022002A00F03881013C002F00F0698101
:103490003A68126B4A4540F02E823A6D002A00F0DD
:1034A0003C823A683F4ED26AB24240F03382B86DF5
:1034B00018B12FF013F90022BA653A6D002A00F016
:1034C000818207F1180027F0C9FD0F9F7B68013B3F
:1034D0007B60002B00F0D681013444457FF757AF65
:1034E000059F314EDDF80C800124A31E052B0DD85D
:1034F000DFE813F0DF00C600AD00940066001F0295
:103500002A4B64221A604FF006083BE7284910A8AE
:103510002CF0F4F9002110A8FEF7FCFB10A82CF009
:10352000ADF9244910A82CF0E9F9002110A8FEF704
:10353000F1FB10A82CF0A2F9414610A82CF0F2F9EA
:10354000002110A8FEF7E6FB10A82CF097F93168CF
:1035500010A82CF0D3F9002110A8FEF7DBFB10A86F
:103560002CF08CF9072C00F011820134BDE700BF6C
:10357000E4650300F4650300749BFF1F0863030008
:1035800070620300B862030094620300F508000053
:10359000DC6203006488FF1FB0720300290700008B
:1035A000410900006D050000A087FF1F2C87FF1F49
:1035B00030660300486603007504000095050000AE
:1035C000A04910A82CF09AF9002110A8FEF7A2FB40
:1035D00010A82CF053F99C4910A82CF08FF9002169
:1035E00010A8FEF797FB10A82CF048F907F1580136
:1035F00010A82CF097F9002110A8FEF78BFB10A85B
:103600002CF03CF9316810A82CF078F910A80021B2
:10361000FEF780FB10A82CF031F9A6E78B4910A823
:103620002CF06CF9002110A8FEF774FB10A82CF008
:1036300025F9854910A82CF061F9002110A8FEF7A2
:1036400069FB10A82CF01AF907F14801D0E780496E
:1036500010A82CF053F9002110A8FEF75BFB10A86E
:103660002CF00CF9784910A82CF048F9002110A88A
:10367000FEF750FB10A82CF001F907F13801B7E76D
:10368000744910A82CF03AF9002110A8FEF742FB6B
:1036900010A82CF0F3F86C4910A82CF02FF9002199
:1036A00010A8FEF737FB10A82CF0E8F807F1280166
:1036B0009EE7694910A82CF021F9002110A8FEF717
:1036C00029FB10A82CF0DAF85F4910A82CF016F9A5
:1036D000002110A8FEF71EFB10A82CF0CFF807F170
:1036E000180185E7384690470F9F00287FF4CCAE3D
:1036F000002F00F0A18039684A6B58498A4240F097
:103700007381BE6D002E00F00082314610A82CF0AF
:10371000F5F807A910A82CF003FA00281ADB019B82
:10372000A34217DC039B029A0F9E03EB0217002EA5
:1037300000F0A88132684949526B8A4240F03082D9
:10374000B16D002900F03E8238462CF043F9029B0F
:103750000133029310A82CF091F80F9F002F7FF4F3
:1037600097AE3F4B3F49059F3F4E04F1080210A81A
:103770001A602CF0C3F8002110A8FEF7CBFA10A8AD
:103780002CF07CF82220FEF71FFE601E2EF00CFBB2
:103790000021FEF7CBFD316810A82CF0AFF8002116
:1037A00010A8FEF7B7FA10A82CF068F80F9C2F4B62
:1037B0000B93002C3FF496AE6368013B6360002BD3
:1037C0007FF490AE22682A49D26A01938A4240F07F
:1037D0004A82A06D18B12EF081FF019BA365236D75
:1037E000002B00F0118204F1180027F037FC0F9C29
:1037F000002C3FF477AE23681E4A5B68934240F08A
:103800000082A06D1C4B236018B12EF067FF0023CF
:10381000A365236D04F11808002B00F027824046B1
:1038200027F01CFC154BA360404627F017FC2046F0
:103830005C212BF085FD55E6114967E7104F3146B5
:1038400005E600BFC466030048660300AC660300DB
:10385000946603007C6603004C66030029070000A1
:103860002C87FF1FF4660300A087FF1FDC620300A4
:103870006D050000590D0000086303009462030009
:10388000AC94030039680493C96AB14240F0B08037
:10389000B86D18B12EF022FF049BBB653B6D002B69
:1038A00000F0518107F1180027F0D8FB0F9E002E81
:1038B0003FF412AE3368A64A5B68934240F022811F
:1038C000B06DA44B336018B12EF008FF0023B36530
:1038D000336D06F11807002B00F05D81384627F0A4
:1038E000BDFB9D4BB360384627F0B8FB30465C21EA
:1038F0002BF026FDF0E53846904700283FF431AF25
:103900000F9F002F3FF4E8AD3A68944ED26AB2425E
:103910003FF4CDAD38469047D7E57A6D002A7FF465
:10392000C0AD1EE73046984707462FF089FF014695
:103930008DE58B4910A82BF0E1FF002110A8FEF7C0
:10394000E9F910A82BF09AFF864910A82BF0D6FFB2
:10395000002110A8FEF7DEF910A82BF08FFF07F169
:10396000680110A82BF0DEFF002110A8FEF7D2F9A5
:1039700010A82BF083FF316810A82BF0BFFF10A810
:103980000021FEF7C7F910A82BF078FF07A82BF04D
:1039900075FF6C68013C6C60002C40D025B0BDE820
:1039A000F08F7A6D002A3FF4A7AE92F8312012F022
:1039B000500F14BF0122002263E5002229460BA804
:1039C00098472AE57A6D002A7FF47BAD7DE5239B3D
:1039D000002B7FF4F6AC644A8DF830300D968DF8EC
:1039E00038300F930B9213E53846904701468DE629
:1039F000384688475AE74FF480702EF067FE01463C
:103A0000B065002800F094800770306D002800F049
:103A1000CB804FF4807227F02BF9B76D13E52B683C
:103A20004E4ADB6A934240F0CA80A86D10B12EF076
:103A300055FEAC652B6D002B00F0FC80584627F03E
:103A40000DFB2B68424A5B68934240F0E280A86D10
:103A5000404B2B6018B12EF041FE0023AB652B6D5F
:103A6000002B00F0EC80584627F0F8FA3A4BAB6098
:103A7000584627F0F3FA28465C212BF061FC25B06C
:103A8000BDE8F08F39495FE62B68344ADB6A934220
:103A900040F0AC80A86D10B12EF020FEAC652B6D0F
:103AA000002B00F0A680584627F0D8FA2B68284A49
:103AB0005B68934240F0B080A86D264B2B6018B134
:103AC0002EF00CFE0023AB652B6D002B00F0BC80AC
:103AD000584627F0C3FA204BAB60584627F0BEFA91
:103AE0005C2128462BF02CFC2B68DFF888901A6BA1
:103AF0004A453FF435AC2846904700283FF446AF8E
:103B00002B6831E430469847E6E44FF480702EF09D
:103B1000DDFDB86500284FD006703A6D002A7FD0D1
:103B2000014610464FF4807227F0A2F8BE6DECE516
:103B30000F4FB76587E46A6D002A7FF415AC25E75F
:103B40002846984715E47B6D002B7FF4ABAEADE6BD
:103B5000590D000008630300946203006D05000026
:103B6000DC66030048660300DC620300AC940300DB
:103B7000E492FF1F75040000239B002B7FF4C2AB6F
:103B80003D4B109314A827F069FA07A82BF076FE96
:103B900025B0BDE8F08F736D002B7FF49FAEA0E6DB
:103BA000304690470146CFE5706D18B14FF48072F2
:103BB00024F0A2FEB76D46E4304EBE65A5E528466A
:103BC00098473EE74FF4807004912EF07FFDB0657A
:103BD000A0B104990170326D002A3AD00146104616
:103BE0004FF4807227F044F8B16DADE52846984750
:103BF0005CE76B6D002B7FF456AF57E71F49B1654B
:103C0000A2E5204698476DE4636D002B7FF4EBAD91
:103C1000EDE528469847C1E628469847FFF799BB47
:103C20007A6D2AB1014610464FF4807224F064FE8A
:103C3000BE6D6AE56B6D002B7FF400AF01E76B6D25
:103C4000002B7FF410AF11E76B6D002B7FF440AFBA
:103C500041E7726D2AB1014610464FF4807224F09C
:103C60004BFEB16D70E520469047C0E5636D002BBB
:103C70007FF4D5ADD6E500BF94620300E492FF1F48
:103C80002DE9F04F914C9249C7B0002605460DA88A
:103C900026602BF033FE314611A82BF02FFE314663
:103CA00015A82BF02BFE334632A88A4A8A4927F002
:103CB000BFFA449B002B00F070825C202BF03CFB91
:103CC0000646864B9DF8CC00349A85493360002720
:103CD0009DF8D43030730DF1D808B160326141469F
:103CE000337506F11800776027F08AF973687D490B
:103CF000DFF810A2B76501334FF47A728DF8B8700F
:103D00008DF8C0703196B16073602F92CDF8B4A079
:103D10004046DFF8F4B1CDF8C8B027F09FF9319BE9
:103D2000002B00F0B8801A686F49126B8A4240F08D
:103D3000AC801A6D002A00F0E0816C490A68049298
:103D400004980A680392039A121A132AF9D9002BCD
:103D50002FD0674F5D4E6FF000484FF000091A6892
:103D60001269BA4240F0B0811A6D002A00F0AF81AA
:103D70001378190740F18781D3695069181A02D462
:103D8000002800F080810A2278232DA932A82BF088
:103D90006FFC32A90DA82BF015FE32A82BF06EFD9A
:103DA0002268AA4200F06F81319B01323260002B01
:103DB000D5D100210DA82BF08BFE4E4C037823604B
:103DC00001220DA932A82BF0E1FE32A911A82BF097
:103DD000F9FD32A82BF052FD0DA947482BF0EAFD62
:103DE00023680D3B4D2B00F28582DFE813F0410183
:103DF000830283028302830283028302830283029B
:103E0000830283028302830283028302830283028A
:103E1000830283028302830283028302830283027A
:103E2000830283028302830283028302830283026A
:103E3000830283028302830283028302830283025A
:103E4000830283028302830283025A028302830273
:103E50008302830283024101410141014101410189
:103E600053020A02310241012A028B018B018302B3
:103E70004C0241014101110283024101C800830249
:103E80002302620241018302410118469047319B9F
:103E900000287FF452AF194A194D012111700024F6
:103EA000CDF8B4A01BB15E68013E5E6076B315A884
:103EB0002BF0E4FC11A82BF0E1FC0DA82BF0DEFCAC
:103EC0002046294647B0BDE8F08F00BF809AFF1F0B
:103ED000AC940300A498FF1F749BFF1F08630300AA
:103EE00070620300B8620300750400007CA0FF1F2D
:103EF000790B0000109BFF1F5C95FF1F8495FF1F2F
:103F00000000F0BFDC620300946203001A68AF494E
:103F1000D26A8A4240F05781986D20B101932EF009
:103F2000DDFB019B9E651A6D002A00F0ED8103F117
:103F3000180027F093F8319E002EB8D03368A44AB9
:103F40005B68934240F05A81B06DA24B336018B168
:103F50002EF0C4FB0023B365336D06F11807002B68
:103F600000F0DA81384627F079F8C6F808B038460C
:103F700027F074F830465C212BF0E2F997E7012135
:103F80000DA82BF0A5FD017819A82BF0E9FC022261
:103F90000DA932A82BF0FAFD32A911A82BF012FDC1
:103FA00032A82BF06BFC1422002332A911A82BF0AD
:103FB0009DFD894B93E803000590ADF8181032A8D9
:103FC00005A92FF009FC00220346044611A91DA8EB
:103FD0002BF0B8FD224621A811A92BF0D7FD29AD61
:103FE00021A925A8012300222BF0ACFD21A92846F8
:103FF00001222BF0CBFD19A878492BF053FD0028A6
:1040000000F0AD81764B00221A60744925A82BF090
:1040100049FD002800F09A81724B00221A600023AB
:104020000A2207A91DA82BF061FD07A82EF0F6FAB9
:104030002DF0B0FD6C4B6D4C18600A2200230AA9CC
:1040400028462BF053FD0AA82EF0E8FA2DF0A2FD29
:10405000206028462BF012FC25A82BF00FFC21A88D
:104060002BF00CFC1DA82BF009FC19A82BF006FC6A
:104070005F4B1198002808BF18462EF0CFFA319BED
:1040800004460D460CE7319C002C3FF492AE2368A9
:104090004E4EDB6AB34240F09380A06D18B12EF013
:1040A0001DFB0023A365236D002B00F0288104F184
:1040B000180026F0D3FF319D6C68013C6C60002C29
:1040C00035D00023319374E61846904758E6596D71
:1040D0000029D8D091F831301B07D4D5D1E9042379
:1040E000D1E90001101A63EB0101894508BF804541
:1040F000BFF446AE6FF0004042E65A6D002A7FF4EE
:104100001CAEC8E601210DA82BF0E2FC017839486D
:104110002BF06AFC02220DA932A82BF037FD32A940
:1041200011A82BF04FFC32A82BF0A8FBA0E72B68BE
:10413000DB6AB34240F0ED80A86D10B12EF0CEFAEC
:10414000AC652B6D002B00F0EF8005F1180026F018
:1041500085FF319C002CB4D023681D4A5B689342D4
:1041600040F0DF80A06D1B4B236018B12EF0B6FA33
:104170000023A365236D04F11805002B00F0D980FE
:10418000284626F06BFFC4F808B0284626F066FFE4
:1041900020465C212BF0D4F893E7459B002B7FF45D
:1041A0008CAD4FF47A72DFF850A08DF8B8308DF8EE
:1041B000C03031932F92CDF8B4A00DF1D808A7E507
:1041C0002046984777E718469047B4E66D0500000B
:1041D000590D000008630300786703003867030087
:1041E000289BFF1F0C9BFF1FB887FF1FAC87FF1F7B
:1041F0004C980300B497FF1FDC62030030469847D9
:1042000055E601210DA82BF063FC01787E487FE77D
:104210007E4C7F480123292123702AF03FFD21781D
:104220007C482BF01FF97B482BF0C8F800240025B0
:10423000319B35E601210DA82BF04AFC0178764828
:1042400066E701210DA82BF043FC017873485FE776
:104250000023142232A911A82BF048FC7049714D9B
:10426000714C32A830F0C4FD2EF0D8F92DF092FC3C
:104270006E492860002030F0BBFD2EF0CFF92DF004
:1042800089FC2060F4E601210DA82BF021FC0178C7
:1042900067483DE701210DA82BF01AFC017865481D
:1042A00036E711A964482BF085FB00240025319BDB
:1042B000F6E501210DA82BF00BFC29AD017828466D
:1042C0002BF04EFB28465D492BF0ECFB002835D047
:1042D0000123236002220DA932A82BF057FC32A93A
:1042E00011A82BF06FFB32A82BF0C8FA28462BF050
:1042F000C5FABDE6454C524801232E218CE7636D7B
:10430000002B7FF4D4AED6E65A6D002A7FF40FAEB0
:1043100011E6284698471CE7736D002B7FF422AE08
:1043200023E620469847CCE66B6D002B7FF40DAF5B
:104330000FE7636D002B7FF423AF24E74149284644
:104340002BF0B0FBA0B102232360C3E73E4925A8B0
:104350002BF0A8FBA0B13D4B01221A605FE63A4961
:1043600019A82BF09FFBA0B1394B01221A604CE633
:10437000384928462BF096FBA0B103232360A9E718
:10438000354925A82BF08EFBA8B1304B02221A60CC
:1043900045E6314919A82BF085FBA8B12C4B022228
:1043A0001A6032E62D4928462BF07CFB002891D07C
:1043B000042323608EE7274925A82BF073FB60B107
:1043C000224B03221A602AE6224919A82BF06AFB25
:1043D00070B11F4B03221A6017E6204925A82BF065
:1043E00061FB00283FF41BAE184B04221A6016E64E
:1043F0001A4919A82BF056FB00283FF406AE144BBF
:1044000004221A6001E600BF4C95FF1FAC94FF1F09
:104410000C6703006488FF1FA09AFF1FA497FF1F6B
:1044200008670300189BFF1F8095FF1FBC940300C3
:10443000FC92FF1F4493FF1F3493FF1F3867030054
:1044400048670300446703007C6703000C9BFF1F61
:10445000289BFF1F3C670300A49C030040670300E8
:1044600008B5084B1B68014618462DF0F1FC0649BB
:104470002BF0F4FD2BF05AFD044B19682DF0E8FCED
:1044800008BD00BF5896FF1FDB0FC940EC99FF1F06
:10449000F8B5324A324B556818682DF085FC014654
:1044A00030482DF089FD044628462DF07DFC01465C
:1044B00020462DF0CDFC2C4B5B6C013B0546032BBD
:1044C00049D8DFE803F0363C3002284B58682DF01D
:1044D0006BFC07462846FFF7C3FF254C254A0023FF
:1044E000166884F8903072B639462DF0A7FB224941
:1044F0002DF062FD054630462DF056FC014628465B
:104500002DF05AFDD4F880102DF0A2FCE16FA067C9
:104510002DF05AFEC8B9D4F8883003F10043C4F82E
:104520008C3062B6F8BD154B58682DF03DFC07463F
:10453000D0E7134B58682DF037FC0746CAE7114BFC
:1045400058682DF031FC0746C4E7D4F88830C4F829
:104550008C3062B6F8BD0027BCE700BF2C9BFF1F64
:10456000249BFF1FDB0FC940109AFF1F6893FF1F9A
:104570005899FF1F5493FF1FCDCCCC3C8895FF1F4B
:104580006498FF1F2098FF1F2DE9F043C14BC1B075
:104590001D6807AC2D1B40AE281928F003FB04F85A
:1045A000010BA642F8D1BC49BC4CBD4EBD4DBE4F1F
:1045B00003A82BF0A3F9002103A8FDF7ABFB03A888
:1045C0002BF05CF92220FDF7FFFE07982DF0E8FBA9
:1045D0000021FDF7ABFE216803A82BF08FF9002125
:1045E00003A8FDF797FB03A82BF048F9AF4903A8F0
:1045F0002BF084F9002103A8FDF78CFB03A82BF016
:104600003DF92220FDF7E0FE08982DF0C9FB0021BE
:10461000FDF78CFE216803A82BF070F9002103A898
:10462000FDF778FB03A82BF029F9A14903A82BF08B
:1046300065F9002103A8FDF76DFB03A82BF01EF917
:104640002220FDF7C1FE04210998FDF76FFE2168C5
:1046500003A82BF053F9002103A8FDF75BFB03A887
:104660002BF00CF9934903A82BF048F9002103A87B
:10467000FDF750FB03A82BF001F92220FDF7A4FE63
:104680009DF8B81003A8002914BF314629462BF025
:1046900035F9002103A8FDF73DFB03A82BF0EEF848
:1046A000216803A82BF02AF9002103A8FDF732FBAB
:1046B00003A82BF0E3F8804903A82BF01FF9002191
:1046C00003A8FDF727FB03A82BF0D8F82220FDF75D
:1046D0007BFE0A982DF064FB0021FDF727FE216880
:1046E00003A82BF00BF9002103A8FDF713FB03A887
:1046F0002BF0C4F8714903A82BF000F9002103A89E
:10470000FDF708FB03A82BF0B9F82220FDF75CFEAB
:104710000B982DF045FB0021FDF708FE216803A84A
:104720002BF0ECF8002103A8FDF7F4FA03A82BF016
:10473000A5F8634903A82BF0E1F8002103A8FDF7D1
:10474000E9FA03A82BF09AF82220FDF73DFEDDF8E8
:10475000309006214846FDF7E9FD216803A82BF0BB
:10476000CDF8002103A8FDF7D5FA03A82BF086F8B1
:10477000232154482AF092FA78692CF0BFFE4FF0BA
:10478000080802460B46CDF800804F482AF074FE18
:104790004D482AF013FE27214C482AF07FFA48465C
:1047A0002CF0ACFECDF8008002460B4646482AF0BD
:1047B00063FE45482AF002FE454903A82BF09EF807
:1047C000002103A8FDF7A6FA03A82BF057F8222032
:1047D000FDF7FAFD9DF8B91003A8002914BF314672
:1047E00029462BF08BF8002103A8FDF793FA03A8C4
:1047F0002BF044F8216803A82BF080F8002103A8CF
:10480000FDF788FA03A82BF039F8324903A82BF0FA
:1048100075F8002103A8FDF77DFA03A82BF02EF808
:104820002220FDF7D1FD0F982DF0BAFA0021FDF7F7
:104830007DFD216803A82BF061F8002103A8FDF796
:1048400069FA03A82BF01AF8234903A82BF056F8AD
:10485000002103A8FDF75EFA03A82BF00FF8222031
:10486000FDF7B2FD10982DF09BFA0021FDF75EFDDB
:10487000216803A82BF042F8002103A8FDF74AFAAB
:1048800003A82AF0FBFF154903A82BF037F80021F5
:1048900003A825E0D895FF1F8C670300A087FF1FA2
:1048A0008067030084670300BC96FF1FA4670300B2
:1048B000BC670300D4670300EC670300FC670300D8
:1048C0000C6803001C6803006488FF1F4068030035
:1048D000686803007868030088680300986803002C
:1048E000FDF718FA03A82AF0C9FF2220FDF76CFD96
:1048F00005211198FDF71AFD216803A82AF0FEFF93
:10490000002103A8FDF706FA03A82AF0B7FFBF4964
:1049100003A82AF0F3FF002103A8FDF7FBF903A881
:104920002AF0ACFF2220FDF74FFD9DF8BA1003A836
:10493000002914BF314629462AF0E0FF002103A8D0
:10494000FDF7E8F903A82AF099FF216803A82AF0E7
:10495000D5FF002103A8FDF7DDF903A82AF08EFF9B
:10496000AB4903A82AF0CAFF002103A8FDF7D2F93A
:1049700003A82AF083FF2220FDF726FD36982DF0AC
:104980000FFA0021FDF7D2FC216803A82AF0B6FF38
:10499000002103A8FDF7BEF903A82AF06FFF9D4987
:1049A00003A82AF0ABFF002103A8FDF7B3F903A881
:1049B0002AF064FF2220FDF707FD37982DF0F0F96B
:1049C0000021FDF7B3FC216803A82AF097FF00211E
:1049D00003A8FDF79FF903A82AF050FF8E4903A80A
:1049E0002AF08CFF002103A8FDF794F903A82AF010
:1049F00045FF2220FDF7E8FC05213898FDF796FCDD
:104A0000216803A82AF07AFF002103A8FDF782F9A4
:104A100003A82AF033FF814903A82AF06FFF002181
:104A200003A8FDF777F903A82AF028FF2220FDF755
:104A3000CBFC9DF8E41003A8002914BF3146294699
:104A40002AF05CFF002103A8FDF764F903A82AF00F
:104A500015FF216803A82AF051FF03A80021FDF7E4
:104A600059F903A82AF00AFF359B012B00F048836F
:104A70006B496C4D03A82AF041FF002103A8FDF704
:104A800049F903A82AF0FAFE296803A82AF036FF9C
:104A9000002103A8FDF73EF903A82AF0EFFE6249C2
:104AA00003A82AF02BFF002103A8FDF733F903A880
:104AB0002AF0E4FE296803A82AF020FF002103A8B9
:104AC000FDF728F903A82AF0D9FE584903A82AF0CF
:104AD00015FF002103A8FDF71DF903A82AF0CEFE5B
:104AE000296803A82AF00AFF002103A8FDF712F99C
:104AF00003A82AF0C3FE4E4903A82AF0FFFE0021B6
:104B000003A8FDF707F903A82AF0B8FE296803A84F
:104B10002AF0F4FE002103A8FDF7FCF803A82AF010
:104B2000ADFE444903A82AF0E9FE002103A8FDF7E1
:104B3000F1F803A82AF0A2FE2220FDF745FC159803
:104B40002DF02EF90021FDF7F1FB216803A82AF0D2
:104B5000D5FE002103A8FDF7DDF803A82AF08EFE9C
:104B6000354903A82AF0CAFE002103A8FDF7D2F8B0
:104B700003A82AF083FE2220FDF726FC16982DF0CC
:104B80000FF90021FDF7D2FB216803A82AF0B6FE39
:104B9000002103A8FDF7BEF803A82AF06FFE2749FD
:104BA00003A82AF0ABFE002103A8FDF7B3F803A881
:104BB0002AF064FE2220FDF707FC04211798FDF778
:104BC000B5FB216803A82AF099FE002103A8FDF790
:104BD000A1F803A82AF052FE194903A82AF08EFE74
:104BE000002103A8FDF796F803A82AF047FE22202B
:104BF000FDF7EAFB134A144B9DF8BB1003A80029EC
:104C000014BF114619462AF079FE1FE0A868030078
:104C1000B8680300D0680300E86803000069030077
:104C200068690300A487FF1F78690300886903008F
:104C3000A0690300B8690300D0690300E8690300B4
:104C4000006A03008067030084670300002103A853
:104C5000FDF760F803A82AF011FE216803A82AF0E6
:104C60004DFE002103A8FDF755F803A82AF006FE23
:104C7000149E002E00F0D381BF4903A82AF03EFE07
:104C8000002103A8FDF746F803A82AF0F7FD2968DC
:104C900003A82AF033FE002103A8FDF73BF803A880
:104CA0002AF0ECFDB54903A82AF028FE002103A84C
:104CB000FDF730F803A82AF0E1FD296803A82AF0DF
:104CC0001DFE03A80021FDF725F803A82AF0D6FD54
:104CD000AB4903A82AF012FE002103A8FDF71AF839
:104CE00003A82AF0CBFD2220FDF76EFB04211898C3
:104CF000FDF71CFB216803A82AF000FE002103A891
:104D0000FDF708F803A82AF0B9FD9E4903A82AF088
:104D1000F5FD002103A8FCF7FDFF03A82AF0AEFD76
:104D20002220FDF751FB1D982DF03AF80021FDF7E8
:104D3000FDFA216803A82AF0E1FD002103A8FCF791
:104D4000E9FF03A82AF09AFD8F4903A82AF0D6FDAF
:104D5000002103A8FCF7DEFF03A82AF08FFD222024
:104D6000FDF732FBF86D2DF01BF80021FDF7DEFAA0
:104D7000216803A82AF0C2FD002103A8FCF7CAFF9E
:104D800003A82AF07BFD1121804829F087FF1E9E91
:104D90007F48314600230A222AF024FB7C482AF06F
:104DA0000DFB1121794829F079FF00230A223146B1
:104DB00077482AF017FB76482AF000FB754903A8CC
:104DC0002AF09CFD002103A8FCF7A4FF03A82AF009
:104DD00055FD2220FDF7F8FA05211F98FDF7A6FAE8
:104DE000216803A82AF08AFD002103A8FCF792FF9E
:104DF00003A82AF043FD684903A82AF07FFD00219B
:104E000003A8FCF787FF03A82AF038FD2220FDF74E
:104E1000DBFA624A624B9DF8BC1003A8002914BF5C
:104E2000114619462AF06AFD002103A8FCF772FF1B
:104E300003A82AF023FD216803A82AF05FFD0021C2
:104E400003A8FCF767FF03A82AF018FD1C9E002E9C
:104E500000F01281534903A82AF050FD002103A855
:104E6000FCF758FF03A82AF009FD296803A82AF0D7
:104E700045FD002103A8FCF74DFF03A82AF0FEFC26
:104E8000494903A82AF03AFD002103A8FCF742FF94
:104E900003A82AF0F3FC296803A82AF02FFD03A831
:104EA0000021FCF737FF03A82AF0E8FC3F4903A8DC
:104EB0002AF024FD002103A8FCF72CFF03A82AF008
:104EC000DDFC2220FDF780FA04212098FDF72EFA60
:104ED000216803A82AF012FD002103A8FCF71AFF9D
:104EE00003A82AF0CBFC324903A82AF007FD0021D1
:104EF00003A8FCF70FFF03A82AF0C0FC2220FDF74F
:104F000063FA3D9E30462CF04BFF0021FDF70EFA70
:104F10002021284829F0C2FE1D482AF04FFA00231C
:104F20000A2231461A482AF05DFA19482AF046FA50
:104F3000216803A82AF0E2FC002103A8FCF7EAFE9E
:104F400003A82AF09BFC3A9C002C00F0C2801A496E
:104F500003A82AF0D3FC002103A8FCF7DBFE03A87A
:104F60002AF08CFC296803A82AF0C8FC03A80021B9
:104F7000FCF7D0FE03A821E0186A0300306A0300A2
:104F8000786A0300906A0300A86A0300C06A0300FD
:104F90006488FF1FD46A0300EC6A03008067030083
:104FA00084670300046B03001C6B0300646B030045
:104FB0007C6B0300906B0300C86B03002AF05EFC5F
:104FC000724903A82AF09AFC002103A8FCF7A2FE6C
:104FD00003A82AF053FC296803A82AF08FFC0021BB
:104FE00003A8FCF797FE03A82AF048FC684903A829
:104FF0002AF084FC002103A8FCF78CFE03A82AF009
:105000003DFC296803A82AF079FC002103A8FCF7DD
:1050100081FE03A82AF032FC41B0BDE8F0835D496F
:1050200003A82AF06BFC314603A8FCF773FE03A823
:105030002AF024FC296803A82AF060FC314603A862
:10504000FCF768FE03A82AF019FC534903A82AF0CC
:1050500055FC314603A8FCF75DFE03A82AF00EFCC0
:10506000296803A82AF04AFC03A83146FCF752FE3F
:1050700003A82AF003FC2BE6484903A82AF03EFCCB
:10508000314603A8FCF746FE03A82AF0F7FB29687F
:1050900003A82AF033FC314603A8FCF73BFE03A823
:1050A0002AF0ECFB3E4903A82AF028FC314603A86D
:1050B000FCF730FE03A82AF0E1FB296803A82AF0D8
:1050C0001DFC03A83146FCF725FE03A82AF0D6FBF9
:1050D000ECE6344903A82AF011FC214603A8FCF7AA
:1050E00019FE03A82AF0CAFB296803A82AF006FCC7
:1050F00003A82146FCF70EFE03A82AF0BFFB5FE7DA
:1051000029492A4D03A82AF0F9FB002103A8FCF73E
:1051100001FE03A82AF0B2FB296803A82AF0EEFBDF
:10512000002103A8FCF7F6FD03A82AF0A7FB2049FD
:1051300003A82AF0E3FB002103A8FCF7EBFD03A87A
:105140002AF09CFB296803A82AF0D8FB002103A8B9
:10515000FCF7E0FD03A82AF091FB164903A82AF00A
:10516000CDFB002103A8FCF7D5FD03A82AF086FBA0
:10517000296803A82AF0C2FB002103A8FCF7CAFD96
:1051800003A82AF07BFB0C49B6E400BFDC6B0300EC
:10519000F46B0300486A0300606A0300346B030089
:1051A0004C6B0300B46B030018690300A487FF1F56
:1051B00028690300386903005069030070B5C14BCA
:1051C000C0B01D6807AC2D1B40AE281927F0EAFCC3
:1051D00004F8010BA642F8D1BB4A13680293029966
:1051E00013680193019B5B1AC72BF9D9B749B84CD7
:1051F000B84D03A82AF082FB002103A8FCF78AFD22
:1052000003A82AF03BFB2220FDF7DEF8A0692CF072
:10521000C7FD0021FDF78AF8296803A82AF06EFB74
:10522000002103A8FCF776FD03A82AF027FBAA4972
:1052300003A82AF063FB002103A8FCF76BFD03A879
:105240002AF01CFB2220FDF7BFF8E0692CF0A8FD36
:105250000021FDF76BF8296803A82AF04FFB002115
:1052600003A8FCF757FD03A82AF008FB9B4903A8F5
:105270002AF044FB002103A8FCF74CFD03A82AF008
:10528000FDFA2220FDF7A0F8E06A2CF089FD00214C
:10529000FDF74CF8296803A82AF030FB002103A889
:1052A000FCF738FD03A82AF0E9FA8D4903A82AF093
:1052B00025FB002103A8FCF72DFD03A82AF0DEFA48
:1052C0002220FDF781F8206B2CF06AFD0021FDF70C
:1052D0002DF8296803A82AF011FB002103A8FCF788
:1052E00019FD03A82AF0CAFA7E4903A82AF006FB92
:1052F000002103A8FCF70EFD03A82AF0BFFA222024
:10530000FDF762F8E06C2CF04BFD0021FDF70EF884
:10531000296803A82AF0F2FA002103A8FCF7FAFC96
:1053200003A82AF0ABFA704903A82AF0E7FA002193
:1053300003A8FCF7EFFC03A82AF0A0FA2220FDF74F
:1053400043F8206D2CF02CFD0021FCF7EFFF2968BD
:1053500003A82AF0D3FA002103A8FCF7DBFC03A87A
:105360002AF08CFA614903A82AF0C8FA002103A8A0
:10537000FCF7D0FC03A82AF081FA2220FDF724F8DC
:10538000E06E2CF00DFD0021FCF7D0FF296803A88A
:105390002AF0B4FA002103A8FCF7BCFC03A82AF009
:1053A0006DFA0921524829F079FC00230A22E16EA6
:1053B00050482AF017F84F482AF000F84E4903A841
:1053C0002AF09CFA002103A8FCF7A4FC03A82AF009
:1053D00055FA2220FCF7F8FF206F2CF0E1FC0021A9
:1053E000FCF7A4FF296803A82AF088FA002103A883
:1053F000FCF790FC03A82AF041FA09213F4829F064
:105400004DFC00230A22216F3A4829F0EBFF39486E
:1054100029F0D4FF3A4903A82AF070FA002103A822
:10542000FCF778FC03A82AF029FA2220FCF7CCFF2D
:10543000D4F8D0002CF0B4FC0021FCF777FF2968E9
:1054400003A82AF05BFA002103A8FCF763FC03A879
:105450002AF014FA0D212B4829F020FCD4F8B410BE
:10546000244800230A2229F0BDFF224829F0A6FF84
:10547000D4F8B450002D00F09F80234903A82AF0EF
:105480003DFA03A80021FCF745FC03A82AF0F6F931
:105490001E4D03A829682AF031FA002103A8FCF761
:1054A00039FC03A82AF0EAF9D4F8D440002C00F023
:1054B0008F80174903A82AF021FA002103A8FCF7DE
:1054C00029FC27E0D895FF1F7CA0FF1F086C030074
:1054D000BC96FF1FA087FF1F1C6C0300306C0300ED
:1054E000446C0300586C03006C6C0300806C030078
:1054F000946C03006488FF1FA06C0300B46C03006D
:10550000C06C0300D46C0300E46C0300A487FF1F8D
:10551000346D030003A82AF0B1F9296803A82AF022
:10552000EDF9002103A8FCF7F5FB03A82AF0A6F982
:105530003E4903A82AF0E2F9002103A8FCF7EAFBA0
:1055400003A82AF09BF9296803A82AF0D7F903A831
:105550000021FCF7DFFB03A82AF090F9344903A8E7
:105560002AF0CCF9002103A8FCF7D4FB03A82AF009
:1055700085F9296803A82AF0C1F9002103A8FCF7DE
:10558000C9FB03A82AF07AF92A4903A82AF0B6F938
:10559000002103A8FCF7BEFB03A82AF06FF92968D5
:1055A00003A82AF0ABF9002103A8FCF7B3FB03A87A
:1055B0002AF064F940B070BD1F4903A82AF09EF993
:1055C00003A82946FCF7A6FB03A82AF057F95FE7D2
:1055D0001A4903A82AF092F9214603A8FCF79AFB7E
:1055E00003A82AF04BF9296803A82AF087F9214675
:1055F00003A8FCF78FFB03A82AF040F9104903A881
:105600002AF07CF9214603A8FCF784FB03A82AF0C2
:1056100035F9296803A82AF071F903A82146FCF797
:1056200079FB03A82AF02AF998E700BF486D030028
:105630005C6D0300786D0300F86C03000C6D0300D3
:10564000206D030070B5B94BBEB01D6805AC2D1BB5
:105650003EAE281927F0A6FA04F8010BB442F8D19F
:1056600001A8B349B34CB44D2AF048F9002101A870
:10567000FCF750FB01A82AF001F92220FCF7A4FE58
:1056800022982CF08DFB0021FCF750FE216801A828
:105690002AF034F901A80021FCF73CFB01A82AF00C
:1056A000EDF801A8A5492AF029F9002101A8FCF785
:1056B00031FB01A82AF0E2F82220FCF785FE2398AE
:1056C0002CF06EFB0021FCF731FE216801A82AF0C6
:1056D00015F901A80021FCF71DFB01A82AF0CEF85E
:1056E00001A897492AF00AF9002101A8FCF712FB4A
:1056F00001A82AF0C3F82220FCF766FE24982CF0BB
:105700004FFB0021FCF712FE216801A82AF0F6F8F1
:1057100001A80021FCF7FEFA01A82AF0AFF801A8C1
:1057200088492AF0EBF8002101A8FCF7F3FA01A858
:105730002AF0A4F82220FCF747FE25982CF030FB35
:105740000021FCF7F3FD216801A82AF0D7F801A891
:105750000021FCF7DFFA01A82AF090F801A87A49A5
:105760002AF0CCF8002101A8FCF7D4FA01A82AF00D
:1057700085F82220FCF728FE26982CF011FB00214A
:10578000FCF7D4FD216801A82AF0B8F801A800218F
:10579000FCF7C0FA01A82AF071F801A86B492AF0B9
:1057A000ADF8002101A8FCF7B5FA01A82AF066F8C7
:1057B0002220FCF709FE27982CF0F2FA0021FCF7D2
:1057C000B5FD216801A82AF099F801A80021FCF78D
:1057D000A1FA01A82AF052F801A85D492AF08EF832
:1057E000002101A8FCF796FA01A82AF047F8222028
:1057F000FCF7EAFD28982CF0D3FA0021FCF796FD7F
:10580000216801A82AF07AF801A80021FCF782FAA1
:1058100001A82AF033F801A84E492AF06FF80021B8
:1058200001A8FCF777FA01A82AF028F82220FCF753
:10583000CBFD29982CF0B4FA0021FCF777FD216804
:1058400001A82AF05BF801A80021FCF763FA01A87F
:105850002AF014F801A840492AF050F8002101A8C4
:10586000FCF758FA01A82AF009F82220FCF7ACFD51
:105870002A982CF095FA0021FCF758FD216801A820
:105880002AF03CF801A80021FCF744FA01A829F00D
:10589000F5FF01A831492AF031F8002101A8FCF7F1
:1058A00039FA01A829F0EAFF2220FCF78DFD2B9898
:1058B0002CF076FA0021FCF739FD216801A82AF0C6
:1058C0001DF801A80021FCF725FA01A829F0D6FF50
:1058D00001A823492AF012F801A80021FCF71AFABE
:1058E00001A829F0CBFF296801A82AF007F801A830
:1058F0000021FCF70FFA01A829F0C0FF01A81949FF
:1059000029F0FCFF01A80021FCF704FA01A829F006
:10591000B5FF296801A829F0F1FF01A80021FCF7D3
:10592000F9F901A829F0AAFF3EB070BDD895FF1F74
:10593000906D0300A087FF1FA487FF1FA46D0300C5
:10594000B86D0300CC6D0300E06D0300F46D03003F
:10595000086E03001C6E0300346E03004C6E0300DF
:10596000646E0300806E03002DE9F047094B1B684D
:10597000013BA0B00A2B00F26985DFE813F0910526
:105980001A06260659066705A10661078F089309BE
:10599000E70A0D006C87FF1FE24EE349736DE34D8C
:1059A00005AC204603F0100729F0A8FF002120468F
:1059B000FCF7B0F9204629F061FF2220FCF704FD36
:1059C000DB49204629F09AFF00212046FCF7A2F986
:1059D000204629F053FF2968204629F08FFF002137
:1059E0002046FCF797F9204629F048FFD149204688
:1059F00029F084FF00212046FCF78CF9204629F08D
:105A00003DFF2220FCF7E0FC336C012B0CBFCA49A0
:105A1000CA49204629F072FF00212046FCF77AF996
:105A2000204629F02BFF2968204629F067FF002136
:105A30002046FCF76FF9204629F020FFC049204698
:105A400029F05CFF00212046FCF764F9204629F08C
:105A500015FF2220FCF7B8FC0021F06DFCF766FC76
:105A60002968204629F04AFF00212046FCF752F918
:105A7000204629F003FFB349204629F03FFF0021CB
:105A80002046FCF747F9204629F0F8FE2220FCF7D3
:105A90009BFC002F44F08582AB49204629F02EFF65
:105AA00000212046FCF736F9204629F0E7FE296858
:105AB000204629F023FF00212046FCF72BF9204641
:105AC00029F0DCFEA149204629F018FF00212046DC
:105AD000FCF720F9204629F0D1FE2220FCF774FCC7
:105AE000B06A2CF061F90021FCF720FC29682046FF
:105AF00029F004FF00212046FCF70CF9204629F08C
:105B0000BDFE9349204629F0F9FE00212046FCF70E
:105B100001F9204629F0B2FE2220FCF755FC30683E
:105B20002CF042F90021FCF701FC2968204629F0FD
:105B3000E5FE00212046FCF7EDF8204629F09EFE08
:105B40008449204629F0DAFE00212046FCF7E2F8DD
:105B5000204629F093FE2220FCF736FC70692CF0D9
:105B600023F90021FCF7E2FB2968204629F0C6FE54
:105B700000212046FCF7CEF8204629F07FFE1521B3
:105B8000754829F08BF8F16B744829F06BFC734869
:105B900029F014FC6449204629F0B0FE002120467B
:105BA000FCF7B8F8204629F069FE2220FCF70CFC2F
:105BB0006B49204629F0A2FE00212046FCF7AAF8F6
:105BC000204629F05BFE2968204629F097FE002137
:105BD0002046FCF79FF8204629F050FE61492046F8
:105BE00029F08CFE00212046FCF794F8204629F08D
:105BF00045FE2220FCF7E8FBB0692CF0D5F8002127
:105C0000FCF794FB2968204629F078FE0021204605
:105C1000FCF780F8204629F031FE5349204629F050
:105C20006DFE00212046FCF775F8204629F026FE7F
:105C30002220FCF7C9FB70682CF0B6F80021FCF7B5
:105C400075FB2968204629F059FE00212046FCF703
:105C500061F8204629F012FE4449204629F04EFE04
:105C600000212046FCF756F8204629F007FE2220A6
:105C7000FCF7AAFBF06A2CF097F80021FCF756FB22
:105C80002968204629F03AFE00212046FCF742F818
:105C9000204629F0F3FD3649204629F02FFE002149
:105CA0002046FCF737F8204629F0E8FD2220FCF7D3
:105CB0008BFB736DDB074CBF2E492349204629F02F
:105CC0001DFE00212046FCF725F8204629F0D6FDD0
:105CD0002968204629F012FE00212046FCF71AF818
:105CE000204629F0CBFD2449204629F007FE00215B
:105CF0002046FCF70FF8204629F0C0FD2220FCF7D3
:105D000063FB0021306EFCF711FB2968204629F067
:105D1000F5FD00212046FBF7FDFF204629F0AEFDF2
:105D20002CE000BFBC94FF1F346F0300A087FF1F4F
:105D3000307C03001C6F0300B46F0300B86F0300D6
:105D4000046F0300EC6E0300646F0300B06E030089
:105D5000986E0300C86E0300BC6F03006488FF1FC9
:105D60007C6703004C6F03006C6F0300D46F03006B
:105D7000EC6F0300686F0300846F0300E449204662
:105D800029F0BCFD00212046FBF7C4FF204629F086
:105D900075FD2220FCF718FB736C012B0CBFDD494D
:105DA000DD49204629F0AAFD00212046FBF7B2FF7D
:105DB000204629F063FD2968204629F09FFD002137
:105DC0002046FBF7A7FF204629F058FDD34920467F
:105DD00029F094FD00212046FBF79CFF204629F086
:105DE0004DFD2220FCF7F0FACD49204629F086FD32
:105DF00000212046FBF78EFF204629F03FFD296851
:105E0000204629F07BFD00212046FBF783FF20463A
:105E100029F034FDC349204629F070FD00212046B9
:105E2000FBF778FF204629F029FD2220FCF7CCFA69
:105E3000F0692BF0B9FF0021FCF778FA29682046B9
:105E400029F05CFD00212046FBF764FF204629F085
:105E500015FDB549204629F051FD00212046FBF7EC
:105E600059FF204629F00AFD2220FCF7ADFAB06860
:105E70002BF09AFF0021FCF759FA2968204629F0F7
:105E80003DFD00212046FBF745FF204629F0F6FCAA
:105E9000A649204629F032FD00212046FBF73AFFB3
:105EA000204629F0EBFC2220FCF78EFA306B2BF019
:105EB0007BFF0021FCF73AFA2968204629F01EFDF5
:105EC00000212046FBF726FF204629F0D7FC984901
:105ED000204629F013FD00212046FBF71BFF20463A
:105EE00029F0CCFC2220FCF76FFA736D03F002035B
:105EF000002B44F05C808F49204629F0FFFC0021F4
:105F00002046FBF707FF204629F0B8FC2968204609
:105F100029F0F4FC00212046FBF7FCFE204629F086
:105F2000ADFC8549204629F0E9FC00212046FBF71D
:105F3000F1FE204629F0A2FC2220FCF745FA0021C0
:105F4000706EFCF7F3F92968204629F0D7FC002190
:105F50002046FBF7DFFE204629F090FC77492046DB
:105F600029F0CCFC00212046FBF7D4FE204629F086
:105F700085FC2220FCF728FAB36C012B0CBF654985
:105F80006549204629F0BAFC00212046FBF7C2FEF5
:105F9000204629F073FC2968204629F0AFFC002137
:105FA0002046FBF7B7FE204629F068FC64492046EE
:105FB00029F0A4FC00212046FBF7ACFE204629F086
:105FC0005DFC2220FCF700FA5E49204629F096FC91
:105FD00000212046FBF79EFE204629F04FFC296851
:105FE000204629F08BFC00212046FBF793FE20463B
:105FF00029F044FC5449204629F080FC0021204629
:10600000FBF788FE204629F039FC2220FCF7DCF95A
:10601000306A2BF0C9FE0021FCF788F92968204678
:1060200029F06CFC00212046FBF774FE204629F085
:1060300025FC4649204629F061FC00212046FBF75B
:1060400069FE204629F01AFC2220FCF7BDF9F06811
:106050002BF0AAFE0021FCF769F92968204629F0F7
:106060004DFC00212046FBF755FE204629F006FC9A
:106070003749204629F042FC00212046FBF74AFE22
:10608000204629F0FBFB2220FCF79EF9706B2BF0D9
:106090008BFE0021FCF74AF92968204629F02EFCE6
:1060A00000212046FBF736FE204629F0E7FB294970
:1060B000204629F023FC00212046FBF72BFE20463A
:1060C00029F0DCFB2220FCF77FF9736D03F0040359
:1060D000002B43F0698717491F4FDFF884A0204643
:1060E00029F00CFC00212046FBF714FE204629F085
:1060F000C5FB2968204629F001FC00212046FBF75A
:1061000009FE204629F0BAFB144920462AE000BFC8
:106110009C6F0300047003000C70030014700300F4
:10612000A49C03002C700300447003005C70030007
:1061300074700300646F03008C700300A47003008C
:10614000BC700300147D0300D4700300EC700300E6
:10615000047103001C710300BC96FF1F347103001F
:10616000BC94FF1F29F0CAFB00212046FBF7D2FD9B
:10617000204629F083FB2220FCF726F90021B06E8F
:10618000FCF7D4F82968204629F0B8FB0021204606
:10619000FBF7C0FD204629F071FBAE49204629F0EF
:1061A000ADFB00212046FBF7B5FD204629F066FB3C
:1061B0002220FCF709F9F36BD7F8349003F00408B8
:1061C000DAF84C30B9F1000F40F0B587012B0CBF65
:1061D000A149A249204629F091FB20464946FBF7F8
:1061E00099FD204629F04AFB2968204629F086FBC4
:1061F00000212046FBF78EFD204629F03FFB1221AF
:10620000974828F04BFD00230A22796B954829F026
:10621000E9F8944829F0D2F81221934828F03EFD7D
:106220004146904829F01EF98E4829F0C7F88F4959
:10623000204629F063FB00212046FBF76BFD20463A
:1062400029F01CFB2220FCF7BFF88949204629F0E1
:1062500055FB00212046FBF75DFD204629F00EFB93
:106260002968204629F04AFB00212046FBF752FD11
:10627000204629F003FB7F49204629F03FFB0021FF
:106280002046FBF747FD204629F0F8FA2220FCF7CC
:106290009BF8706A2BF088FD0021FCF747F829680D
:1062A000204629F02BFB00212046FBF733FD20463A
:1062B00029F0E4FA7049204629F020FB002120460D
:1062C000FBF728FD204629F0D9FA2220FCF77CF8BC
:1062D00030692BF069FD0021FCF728F82968204679
:1062E00029F00CFB00212046FBF714FD204629F085
:1062F000C5FA6249204629F001FB00212046FBF740
:1063000009FD204629F0BAFA2220FCF75DF8B06BAF
:106310002BF04AFD0021FCF709F82968204629F0F6
:10632000EDFA00212046FBF7F5FC204629F0A6FAFD
:106330005349204629F0E2FA00212046FBF7EAFC07
:10634000204629F09BFA2220FCF73EF8736D03F0FB
:106350000803002B43F02E864A49DFF8409120467F
:1063600029F0CCFA00212046FBF7D4FC204629F086
:1063700085FA2968204629F0C1FA00212046FBF75A
:10638000C9FC204629F07AFA12213F4828F086FC01
:1063900000230A22796D334829F024F8314829F086
:1063A0000DF81221304828F079FC41462D4829F09B
:1063B00059F82C4829F002F83449204629F09EFA71
:1063C00000212046FBF7A6FC204629F057FA2220A0
:1063D000FBF7FAFFF06E0021FBF7A8FF29682046C3
:1063E00029F08CFA00212046FBF794FC204629F086
:1063F00045FA2749204629F081FA00212046FBF77B
:1064000089FC204629F03AFA2220FBF7DDFF7E6D59
:10641000D9F85030002E03F09D84012B0CBF1D498C
:106420001D49204629F06AFA20460021FBF772FC3C
:10643000204629F023FA2968204629F05FFA2046F1
:106440000021FBF767FC204629F018FA20B0BDE8D0
:10645000F08700BF4C710300B46F0300B86F0300F6
:10646000647103006488FF1F787103008C7103005E
:10647000647D0300A4710300BC710300D4710300A8
:10648000EC710300646F03000472030018720300D0
:1064900030720300047003000C700300BC94FF1FF3
:1064A000764E774FB36D774AD7F8E0007569137071
:1064B0001B02D7F8DC10744CDFF800E203F47F43D2
:1064C000EAB243EA006313430A0402F47F0213436F
:1064D0006E4A23606E4B8EF8000005AC11702046AA
:1064E0006C491D7029F00AFA00212046FBF712FCC6
:1064F000204629F0C3F92220FBF766FF664D30687D
:106500002BF052FC0021FBF711FF2968204629F0EF
:10651000F5F900212046FBF7FDFB204629F0AEF9F6
:106520005E49204629F0EAF900212046FBF7F2FBFC
:10653000204629F0A3F92220FBF746FFB06A2BF092
:1065400033FC0021FBF7F2FE2968204629F0D6F93A
:1065500000212046FBF7DEFB204629F08FF9504949
:10656000204629F0CBF900212046FBF7D3FB20463B
:1065700029F084F92220FBF727FF70692BF014FC27
:106580000021FBF7D3FE2968204629F0B7F9204601
:106590000021FBF7BFFB204629F070F9B36D013BEA
:1065A000032B03F27D86DFE813F0450DA2113011B5
:1065B000BE103C4EB36D042B3FF648AFDFE813F03E
:1065C000CE13BD154A15C6145314374E374815213E
:1065D00028F064FB00230A223168354828F002FFC6
:1065E000334828F0EBFE2721324828F057FB716929
:1065F0002F4800230A2228F0F5FE2D4828F0DEFE61
:106600003768032F05AC03F0D785042F00F05A87B5
:10661000002F03F01585204D7368013B042B02F217
:106620006182DFE813F09812E7115613F71267132F
:10663000214C2368013B0D2B3FF608AF01A252F815
:1066400023F000BF55930000F39B0000C59A0000A3
:10665000779900004D6400004D6400004D64000017
:106660004D6400004D6400004D6400004998000036
:10667000FB960000CD95000081940000E095FF1F7F
:10668000BC96FF1FC49AFF1FB09AFF1F5494FF1FB0
:106690001C98FF1F986E0300A087FF1FB06E0300B9
:1066A000C86E0300BC94FF1FB498FF1F487203001C
:1066B0006488FF1F607203005894FF1FC497FF1F78
:1066C00005AC5849584E594D204629F017F900217C
:1066D0002046FBF71FFB204629F0D0F82220FBF7CD
:1066E00073FEF06A2BF05CFB0021FBF71FFE2968AC
:1066F000204629F003F900212046FBF70BFB20463A
:1067000029F0BCF84A49204629F0F8F80021204633
:10671000FBF700FB204629F0B1F82220FBF754FEDE
:1067200070682BF03DFB0021FBF700FE2968204636
:1067300029F0E4F800212046FBF7ECFA204629F086
:106740009DF83C49204629F0D9F800212046FBF766
:10675000E1FA204629F092F82220FBF735FEB068D6
:106760002BF01EFB0021FBF7E1FD2968204629F0F4
:10677000C5F820460021FBF7CDFA204629F07EF827
:10678000336C012B03F0B883C2F04A85302B02F042
:106790004785312B03F0B0832749204629F0AEF816
:1067A00000212046FBF7B6FA204629F067F82220A0
:1067B000FBF70AFE0021B06CFBF7B8FD2968204604
:1067C00029F09CF800212046FBF7A4FA204629F086
:1067D00055F81A49204629F091F800212046FBF788
:1067E00099FA204629F04AF82220FBF7EDFD002116
:1067F000706CFBF79BFD2968204629F07FF800218B
:106800002046FBF787FA204629F038F83368013B29
:10681000032B3FF61BAEDFE813F0110F8D0E180EA1
:10682000A30D00BFC86E0300CC97FF1FA087FF1FFA
:10683000986E0300B06E03006C6F0300D46F03000A
:1068400005AC8B49DFF850828A4D204629F056F876
:1068500000212046FBF75EFA204629F00FF822209F
:10686000FBF7B2FDD8F800002BF09AFA0021FBF7F5
:106870005DFD2968204629F041F800212046FBF7FC
:1068800049FA204628F0FAFF7B49204629F036F8DD
:1068900000212046FBF73EFA204628F0EFFF222099
:1068A000FBF792FDD8F828002BF07AFA0021FBF7CD
:1068B0003DFD2968204629F021F800212046FBF7FC
:1068C00029FA204628F0DAFF6C49204629F016F80C
:1068D00000212046FBF71EFA204628F0CFFF222099
:1068E000FBF772FDD8F814002BF05AFA0021FBF7E1
:1068F0001DFD2968204629F001F800212046FBF7FC
:1069000009FA204628F0BAFF5D49204628F0F6FF34
:1069100000212046FBF7FEF9204628F0AFFF222099
:10692000FBF752FDD8F85C002BF03AFA0021FBF798
:10693000FDFC2968204628F0E1FF20460021FBF7F6
:10694000E9F9204628F09AFFD8F85860002E03F0A5
:106950005182012E7FD14B49204628F0CFFF0021E4
:106960002046FBF7D7F9204628F088FF2220FBF7C6
:106970002BFD4549204628F0C1FF00212046FBF7AA
:10698000C9F9204628F07AFF2968204628F0B6FF8A
:1069900000212046FBF7BEF9204628F06FFF3B4957
:1069A000204628F0ABFF00212046FBF7B3F9204634
:1069B00028F064FF2220FBF707FDD8F83C002BF0FD
:1069C000EFF90021FBF7B2FC2968204628F096FF7A
:1069D00000212046FBF79EF9204628F04FFF2C4966
:1069E000204628F08BFF00212046FBF793F9204634
:1069F00028F044FF2220FBF7E7FC0021D8F84800EC
:106A0000FBF794FC2968204628F078FF00212046F7
:106A1000FBF780F9204628F031FF1E49204628F078
:106A20006DFF00212046FBF775F9204628F026FF70
:106A30002220FBF7C9FC0021D8F84400FBF776FCC4
:106A40002968204628F05AFF20460021FBF762F90A
:106A5000204628F013FFD8F85430013B032B3FF6B3
:106A6000F5ACDFE813F07707B7064006C90500BFAD
:106A7000986E0300A087FF1FB06E0300C86E03006E
:106A8000846F03004C6F0300A07703006C6F03005A
:106A9000D46F0300EC6F03005C96FF1F05AC7749D1
:106AA000774E784D204628F029FF00212046FBF73D
:106AB00031F9204628F0E2FE2220FBF785FC706CBD
:106AC0002BF06EF90021FBF731FC2968204628F0F5
:106AD00015FF00212046FBF71DF9204628F0CEFEC9
:106AE0006949204628F00AFF00212046FBF712F9E9
:106AF000204628F0C3FE2220FBF766FC306B2BF00B
:106B00004FF90021FBF712FC2968204628F0F6FE19
:106B100000212046FBF7FEF8204628F0AFFE5B4937
:106B2000204628F0EBFE00212046FBF7F3F8204634
:106B300028F0A4FE2220FBF747FCB06D2BF030F9C3
:106B40000021FBF7F3FB2968204628F0D7FE00213F
:106B50002046FBF7DFF8204628F090FE4C492046FF
:106B600028F0CCFE00212046FBF7D4F8204628F080
:106B700085FE2220FBF728FC30692BF011F900215B
:106B8000FBF7D4FB2968204628F0B8FE00212046F8
:106B9000FBF7C0F8204628F071FE3E49204628F059
:106BA000ADFE00212046FBF7B5F8204628F066FE32
:106BB0002220FBF709FCF0680021FBF7B7FB2968EE
:106BC000204628F09BFE00212046FBF7A3F8204634
:106BD00028F054FE3049204628F090FE002120463F
:106BE000FBF798F8204628F049FE2220FBF7ECFB43
:106BF000B0690021FBF79AFB2968204628F07EFE49
:106C000020460021FBF786F8204628F037FE7769FA
:106C1000002F03F0AF80012F23D12049204628F018
:106C20006DFE00212046FBF775F8204628F026FE71
:106C30002220FBF7C9FB1A49204628F05FFE0021FD
:106C40002046FBF767F8204628F018FE2968204602
:106C500028F054FE20460021FBF75CF8204628F07F
:106C60000DFEB368023B052B00F25A82DFE813F0F9
:106C7000FE1234024213311320130F13C86E0300A7
:106C8000E898FF1FA087FF1F986E0300B06E0300F7
:106C90004C6F03006C6F0300D46F0300EC6F0300B4
:106CA000A077030005AC9C499C4E9D4D204628F0E2
:106CB00025FE00212046FBF72DF8204628F0DEFDBA
:106CC0002220FBF781FB306B2BF06AF80021FBF7E9
:106CD0002DFB2968204628F011FE00212046FBF7F5
:106CE00019F8204628F0CAFD8E49204628F006FEF5
:106CF00000212046FBF70EF8204628F0BFFD222099
:106D0000FBF762FBB06D2BF04BF80021FBF70EFB9D
:106D10002968204628F0F2FD00212046FAF7FAFF04
:106D2000204628F0ABFD8049204628F0E7FD0021F1
:106D30002046FAF7EFFF204628F0A0FD2220FBF7BF
:106D400043FB706C2BF02CF80021FBF7EFFA29685D
:106D5000204628F0D3FD00212046FAF7DBFF20462D
:106D600028F08CFD7149204628F0C8FD00212046FE
:106D7000FAF7D0FF204628F081FD2220FBF724FB04
:106D8000F0692BF00DF80021FBF7D0FA29682046B6
:106D900028F0B4FD00212046FAF7BCFF204628F079
:106DA0006DFD6349204628F0A9FD00212046FAF731
:106DB000B1FF204628F062FD2220FBF705FB306A78
:106DC0000021FBF7B3FA2968204628F097FD00213F
:106DD0002046FAF79FFF204628F050FD55492046EF
:106DE00028F08CFD00212046FAF794FF204628F079
:106DF00045FD2220FBF7E8FAF06A0021FBF796FA3E
:106E00002968204628F07AFD00212046FAF782FF03
:106E1000204628F033FD4849204628F06FFD002128
:106E20002046FAF777FF204628F028FD2220FBF7BE
:106E3000CBFA4249204628F061FD00212046FAF7AE
:106E400069FF204628F01AFD2968204628F056FDE3
:106E50002046FBF7C9FA204628F010FD7769002F7D
:106E600003F06880012F00F082813549204628F028
:106E700045FD00212046FAF74DFF204628F0FEFC94
:106E80002220FBF7A1FAB76A002F03F04680012FFA
:106E900000F061812968224F204628F02FFD002153
:106EA0002046FAF737FF204628F0E8FC736A022BE9
:106EB00003F06680032B23D12249204628F01EFDD3
:106EC00000212046FAF726FF204628F0D7FC222092
:106ED000FBF77AFA1C49204628F010FD00212046D5
:106EE000FAF718FF204628F0C9FC3968204628F038
:106EF00005FD20460021FAF70DFF204628F0BEFCD4
:106F00003368013B032B3FF6A1AADFE813F06702C9
:106F10009A09F301550100BF986E0300E898FF1F1E
:106F2000A087FF1FB06E0300C86E03004C6F030004
:106F30006C6F0300D46F03009C6F0300A498FF1FC5
:106F4000EC6F0300846F03009073030005ACD64917
:106F5000D64ED74D204628F0D1FC00212046FAF726
:106F6000D9FE204628F08AFC2220FBF72DFAB06AD1
:106F70002AF016FF0021FBF7D9F92968204628F0EE
:106F8000BDFC00212046FAF7C5FE204628F076FC1D
:106F9000C849204628F0B2FC00212046FAF7BAFE84
:106FA000204628F06BFC2220FBF70EFA30682AF00E
:106FB000F7FE0021FBF7BAF92968204628F09EFC6D
:106FC00000212046FAF7A6FE204628F057FCBA49D1
:106FD000204628F093FC00212046FAF79BFE20462D
:106FE00028F04CFC2220FBF7EFF970692AF0D8FE5C
:106FF0000021FBF79BF92968204628F07FFC00213F
:107000002046FAF787FE204628F038FCAB49204698
:1070100028F074FC00212046FAF77CFE204628F078
:107020002DFC2220FBF7D0F9F06B2AF0B9FE0021ED
:10703000FBF77CF92968204628F060FC00212046F7
:10704000FAF768FE204628F019FC9D49204628F0F2
:1070500055FC00212046FAF75DFE204628F00EFC84
:107060002220FBF7B1F9306C2AF09AFE0021FBF7E1
:107070005DF92968204628F041FC00212046FAF7F6
:1070800049FE204628F0FAFB8E49204628F036FCBF
:1070900000212046FAF73EFE204628F0EFFB222092
:1070A000FBF792F9F06E0021FBF740F929682046C2
:1070B00028F024FC20460021FAF72CFE204628F078
:1070C000DDFB736C013B032B3FF6C0A9DFE813F037
:1070D0008006EE054B05B9047B49204628F00EFCDE
:1070E00000212046FAF716FE204628F0C7FB222092
:1070F000FBF76AF97549204628F000FC002120467C
:10710000FAF708FE204628F0B9FB2968204628F047
:10711000F5FB20460021FAF7FDFD204628F0AEFBE6
:107120003368013B032B3FF691A9DFE813F05701C9
:10713000E306E3004500012B0CBF65496549204685
:1071400028F0DCFB20460021FAF7E4FD204628F079
:1071500095FBFFF749B86049204628F0CFFB204651
:107160000021FAF7D7FD204628F088FB92E65B491C
:10717000204628F0C3FB00212046FAF7CBFD20462D
:1071800028F07CFB2220FBF71FF95349204628F00A
:10719000B5FB00212046FAF7BDFD204628F06EFB26
:1071A0002968204628F0AAFB20460021FAF7B2FD04
:1071B000204628F063FB58E64949204628F09EFB0C
:1071C00000212046FAF7A6FD204628F057FB222092
:1071D000FBF7FAF84349204628F090FB00212046AF
:1071E000FAF798FD204628F049FB2968204628F048
:1071F00085FB00212046FAF78DFD204628F03EFB56
:107200003949204628F07AFB00212046FAF782FD12
:10721000204628F033FB2220FBF7D6F8306C2AF00A
:10722000BFFD0021FBF782F82968204628F066FBA5
:1072300000212046FAF76EFD204628F01FFB2B495F
:10724000204628F05BFB00212046FAF763FD20462C
:1072500028F014FB2220FBF7B7F8B06E2AF0A0FD4F
:107260000021FBF763F82968204628F047FB00213E
:107270002046FAF74FFD204628F000FB1C49204627
:1072800028F03CFB00212046FAF744FD204628F078
:10729000F5FA2220FBF798F8706D2AF081FD0021A5
:1072A000FBF744F8FFF7C7B8C86E0300109AFF1F3A
:1072B000A087FF1F986E0300B06E03004C6F0300A1
:1072C0006C6F0300D46F0300846F030050730300DE
:1072D000047003000C700300A07703009C6F030090
:1072E000EC6E0300647D03001C6F0300346F030029
:1072F000046F0300B549204628F000FB002120461A
:10730000FAF708FD204628F0B9FA2220FBF75CF8CE
:10731000AF49204628F0F2FA00212046FAF7FAFC9D
:10732000204628F0ABFA2968204628F0E7FA002129
:107330002046FAF7EFFC204628F0A0FAA54920469F
:1073400028F0DCFA00212046FAF7E4FC204628F079
:1073500095FA2220FBF738F8F06B2AF021FD002186
:10736000FAF7E4FF2968204628F0C8FA00212046F1
:10737000FAF7D0FC204628F081FA9749204628F0F9
:10738000BDFA00212046FAF7C5FC204628F076FA1F
:107390002220FBF719F8706E2AF002FD0021FAF79F
:1073A000C5FF2968204628F0A9FA00212046FAF7EF
:1073B000B1FC204628F062FA8849204628F09EFA5F
:1073C00000212046FAF7A6FC204628F057FA222092
:1073D000FAF7FAFF306D2AF0E3FC60E77B492046BC
:1073E00028F08CFA00212046FAF794FC204628F079
:1073F00045FA2220FAF7E8FF7949204628F07EFA7C
:1074000000212046FAF786FC204628F037FA296842
:10741000204628F073FA00212046FAF77BFC20462C
:1074200028F02CFA6B49204628F068FA0021204603
:10743000FAF770FC204628F021FA2220FAF7C4FF60
:10744000706B2AF0ADFC0021FAF770FF2968204626
:1074500028F054FA00212046FAF75CFC204628F078
:107460000DFA5D49204628F049FA00212046FAF736
:1074700051FC204628F002FA2220FAF7A5FFF06D11
:107480002AF08EFC0021FAF751FF2968204628F0E7
:1074900035FA00212046FAF73DFC204628F0EEF9A7
:1074A0004E49204628F02AFA00212046FAF732FCFD
:1074B000204628F0E3F92220FAF786FFB06C2AF084
:1074C0006FFCECE64749484D204628F017FA0021AA
:1074D0002046FAF71FFC204628F0D0F92220FAF7C0
:1074E00073FF4249204628F009FA00212046FAF7A6
:1074F00011FC204628F0C2F92968204628F0FEF940
:1075000000212046FAF706FC204628F0B7F9384952
:10751000204628F0F3F900212046FAF7FBFB20462D
:1075200028F0ACF92220FAF74FFFF0692AF038FC76
:107530000021FAF7FBFE2968204628F0DFF9002138
:107540002046FAF7E7FB204628F098F9294920461B
:1075500028F0D4F900212046FAF7DCFB204628F079
:107560008DF92220FAF730FF30692AF019FC00214A
:10757000FAF7DCFE2968204628F0C0F900212046F1
:10758000FAF7C8FB204628F079F91049204628F080
:10759000B5F900212046FAF7BDFB204628F06EF928
:1075A0002220FAF711FFB06A2AF0FAFB0021FAF75D
:1075B000BDFE2968204628F0A1F920460021FAF7EF
:1075C000A9FB204628F05AF9FFF726B8EC6E030015
:1075D000147D03001C6F0300346F0300046F03006D
:1075E0007C670300C86E0300A087FF1F647D030053
:1075F000986E0300B06E0300CB49204628F07EF958
:1076000000212046FAF786FB204628F037F9222091
:10761000FAF7DAFEC549204628F070F90021204625
:10762000FAF778FB204628F029F92968204628F047
:1076300065F900212046FAF76DFB204628F01EF977
:10764000BB49204628F05AF900212046FAF762FB90
:10765000204628F013F92220FAF7B6FED8F81000D9
:107660002AF09EFB0021FAF761FE2968204628F0E7
:1076700045F900212046FAF74DFB204628F0FEF898
:10768000AC49204628F03AF900212046FAF742FB9F
:10769000204628F0F3F82220FAF796FED8F83800B2
:1076A0002AF07EFB0021FAF741FE2968204628F0E7
:1076B00025F900212046FAF72DFB204628F0DEF8B8
:1076C0009D49204628F01AF900212046FAF722FBAE
:1076D000204628F0D3F82220FAF776FED8F82400C6
:1076E0002AF05EFBDBE59049204628F007F90021EF
:1076F0002046FAF70FFB204628F0C0F82220FAF7C0
:1077000063FE8E49204628F0F9F800212046FAF75A
:1077100001FB204628F0B2F82968204628F0EEF850
:1077200000212046FAF7F6FA204628F0A7F880490B
:10773000204628F0E3F800212046FAF7EBFA20462D
:1077400028F09CF82220FAF73FFED8F80C002AF027
:1077500027FB0021FAF7EAFD2968204628F0CEF839
:1077600000212046FAF7D6FA204628F087F871491A
:10777000204628F0C3F800212046FAF7CBFA20462D
:1077800028F07CF82220FAF71FFED8F834002AF0FF
:1077900007FB0021FAF7CAFD2968204628F0AEF859
:1077A00000212046FAF7B6FA204628F067F8624929
:1077B000204628F0A3F800212046FAF7ABFA20462D
:1077C00028F05CF82220FAF7FFFDD8F820002AF014
:1077D000E7FA64E55A4B1E681DAF361B301925F0D9
:1077E000E1F904F8010BA742F8D11D21554827F013
:1077F00055FA00230A220799534827F0F3FD52480F
:1078000027F0DCFD484901A828F078F8002101A8FC
:10781000FAF780FA01A828F031F82220FAF7D4FD0F
:107820004A4901A828F06AF8002101A8FAF772FA7B
:1078300001A828F023F8296801A828F05FF80021A2
:1078400001A8FAF767FA01A828F018F819214048AA
:1078500027F024FA00230A22D8F808103A4827F023
:10786000C1FD334901A828F049F8002101A8FAF721
:1078700051FA01A828F002F82220FAF7A5FDD8F85D
:1078800008002AF08DFA0021FAF750FD296801A8B6
:1078900028F034F8002101A8FAF73CFA01A827F0F3
:1078A000EDFF244901A828F029F8002101A8FAF7E2
:1078B00031FA01A827F0E2FF2220FAF785FDD8F877
:1078C00030002AF06DFA0021FAF730FD296801A88E
:1078D00028F014F8002101A8FAF71CFA01A827F0F3
:1078E000CDFF154901A828F009F8002101A8FAF7F1
:1078F00011FA01A827F0C2FF2220FAF765FDD8F897
:107900001C002AF04DFA0021FAF710FD296801A8A1
:1079100027F0F4FF01A80021FAF7FCF901A827F0ED
:10792000ADFFFEF793BD00BFEC6E0300647D030066
:107930001C6F0300346F0300046F0300147D030009
:107940009887FF1F107303006488FF1FA49C030027
:1079500030730300CD49204627F0D0FF0021204698
:10796000FAF7D8F9204627F089FF2220FAF72CFDF4
:10797000C749204627F0C2FF00212046FAF7CAF97E
:10798000204627F07BFF2968204627F0B7FF00211B
:107990002046FAF7BFF9204627F070FFBD49204680
:1079A00027F0ACFF00212046FAF7B4F9204627F073
:1079B00065FF2220FAF708FDD8F804002AF0F0F954
:1079C0000021FAF7B3FC2968204627F097FF002131
:1079D0002046FAF79FF9204627F050FFAE4920468F
:1079E00027F08CFF00212046FAF794F9204627F073
:1079F00045FF2220FAF7E8FCD8F82C002AF0D0F94D
:107A00000021FAF793FC2968204627F077FF002130
:107A10002046FAF77FF9204627F030FF9F4920469D
:107A200027F06CFF00212046FAF774F9204627F072
:107A300025FF2220FAF7C8FCD8F818002AF0B0F980
:107A40002DE49249204627F059FF00212046FAF7FD
:107A500061F9204627F012FF2220FAF7B5FC904981
:107A6000204627F04BFF00212046FAF753F9204625
:107A700027F004FF2968204627F040FF0021204618
:107A8000FAF748F9204627F0F9FE8249204627F008
:107A900035FF00212046FAF73DF9204627F0EEFE9B
:107AA0002220FAF791FC30692AF07AF90021FAF7DE
:107AB0003DFC2968204627F021FF00212046FAF7E7
:107AC00029F9204627F0DAFE7349204627F016FFF1
:107AD00000212046FAF71EF9204627F0CFFE22208B
:107AE000FAF772FC706A2AF05BF90021FAF71EFCC3
:107AF0002968204627F002FF00212046FAF70AF9FC
:107B0000204627F0BBFE6549204627F0F7FE0021FE
:107B10002046FAF7FFF8204627F0B0FE2220FAF7B9
:107B200053FCB06B2AF03CF90021FAF7FFFB2968FF
:107B3000204627F0E3FE00212046FAF7EBF8204626
:107B400027F09CFE5749204627F0D8FE002120460A
:107B5000FAF7E0F8204627F091FE2220FAF734FCED
:107B6000B06EFFF79CBB4949204627F0C7FE0021B5
:107B70002046FAF7CFF8204627F080FE2220FAF7B9
:107B800023FC4949204627F0B9FE00212046FAF798
:107B9000C1F8204627F072FE2968204627F0AEFE85
:107BA00000212046FAF7B6F8204627F067FE39494B
:107BB000204627F0A3FE00212046FAF7ABF8204626
:107BC00027F05CFE2220FAF7FFFBF0682AF0E8F8C5
:107BD0000021FAF7ABFB2968204627F08FFE002131
:107BE0002046FAF797F8204627F048FE2A49204613
:107BF00027F084FE00212046FAF78CF8204627F073
:107C00003DFE2220FAF7E0FB306A2AF0C9F8002195
:107C1000FAF78CFB2968204627F070FE00212046E9
:107C2000FAF778F8204627F029FE1C49204627F06D
:107C300065FE00212046FAF76DF8204627F01EFE6B
:107C40002220FAF7C1FB706B2AF0AAF80021FAF79C
:107C50006DFB2968204627F051FE00212046FAF7E7
:107C600059F8204627F00AFE0E49204627F046FE26
:107C700000212046FAF74EF8204627F0FFFD22208B
:107C8000FAF7A2FB706EFFF70ABB00BFEC6E0300B1
:107C90007C6703001C6F0300346F0300046F030054
:107CA000647D0300EC6F0300147D0300D749204678
:107CB00027F024FE00212046FAF72CF8204627F072
:107CC000DDFD2220FAF780FBD149204627F016FE81
:107CD00000212046FAF71EF8204627F0CFFD29683C
:107CE000204627F00BFE00212046FAF713F8204625
:107CF00027F0C4FDC749204627F000FE002120469A
:107D0000FAF708F8204627F0B9FD2220FAF75CFBC5
:107D1000B0682AF045F80021FAF708FB29682046E8
:107D200027F0ECFD00212046F9F7F4FF204627F06C
:107D3000A5FDB949204627F0E1FD00212046F9F7CD
:107D4000E9FF204627F09AFD2220FAF73DFBF06973
:107D50002AF026F80021FAF7E9FA2968204627F0E8
:107D6000CDFD00212046F9F7D5FF204627F086FDFE
:107D7000AA49204627F0C2FD00212046F9F7CAFF94
:107D8000204627F07BFD2220FAF71EFB306B2AF0FD
:107D900007F80021FAF7CAFA2968204627F0AEFD55
:107DA00000212046F9F7B6FF204627F067FD9C49E1
:107DB000204627F0A3FD00212046F9F7ABFF20461F
:107DC00027F05CFD2220FAF7FFFA306EFFF767BA62
:107DD0008E49204627F092FD00212046F9F79AFFB0
:107DE000204627F04BFD2220FAF7EEFA8D49204677
:107DF00027F084FD00212046F9F78CFF204627F06C
:107E00003DFD2968204627F079FD00212046F9F73D
:107E100081FF204627F032FD8049204627F06EFD85
:107E200000212046F9F776FF204627F027FD222083
:107E3000FAF7CAFAF06A29F0B3FF0021FAF776FAE6
:107E40002968204627F05AFD00212046F9F762FFF5
:107E5000204627F013FD6F49204627F04FFD0021F3
:107E60002046F9F757FF204627F008FD2220FAF7B1
:107E7000ABFA706829F094FF0021FAF757FA2968E5
:107E8000204627F03BFD00212046F9F743FF20461E
:107E900027F0F4FC6049204627F030FD0021204601
:107EA000F9F738FF204627F0E9FC2220FAF78CFA90
:107EB000B06929F075FF0021FAF738FA29682046E1
:107EC00027F01CFD00212046F9F724FF204627F06B
:107ED000D5FC5349204627F011FD00212046F9F733
:107EE00019FF204627F0CAFC2220FAF76DFAF06D40
:107EF000FFF7D5B94C4B1F680DF180083F1B3819AF
:107F000024F050FE04F8010BA045F8D11D2147488C
:107F100026F0C4FE00230A221399454827F062FA8E
:107F2000434827F04BFA394901A827F0E7FC002124
:107F300001A8F9F7EFFE01A827F0A0FC2220FAF72C
:107F400043FA334901A827F0D9FC002101A8F9F729
:107F5000E1FE01A827F092FC296801A827F0CEFCD9
:107F6000002101A8F9F7D6FE01A827F087FC2949CE
:107F700001A827F0C3FC002101A8F9F7CBFE01A856
:107F800027F07CFC2220FAF71FFAB06B29F008FFDB
:107F90000021FAF7CBF9296801A827F0AFFC0021EE
:107FA00001A8F9F7B7FE01A827F068FC1A4901A853
:107FB00027F0A4FC002101A8F9F7ACFE01A827F0E6
:107FC0005DFC2220FAF700FA306E29F0E9FE00216C
:107FD000FAF7ACF9296801A827F090FC002101A864
:107FE000F9F798FE01A827F049FC0C4901A827F0F1
:107FF00085FC002101A8F9F78DFE01A827F03EFCC1
:108000002220FAF7E1F9F06C7BE400BFEC6E03008C
:10801000A49C03001C6F0300346F0300046F030073
:10802000EC6F03007C6703008487FF1F6473030009
:108030006488FF1F0B21BD4826F030FEB16DBC489F
:1080400027F010FABA4827F0B9F9BA49204627F0C4
:1080500055FC00212046F9F75DFE204627F00EFC76
:108060002220FAF7B1F9B449204627F047FC002155
:108070002046F9F74FFE204627F000FC29682046ED
:1080800027F03CFC00212046F9F744FE204627F06B
:10809000F5FBAA49204627F031FC00212046F9F7DC
:1080A00039FE204627F0EAFB2220FAF78DF9B06965
:1080B00029F07AFE0021FAF739F92968204627F0DD
:1080C0001DFC00212046F9F725FE204627F0D6FBAF
:1080D0009B49204627F012FC00212046F9F71AFEA2
:1080E000204627F0CBFB2220FAF76EF9706829F0C2
:1080F0005BFE0021FAF71AF92968204627F0FEFBFB
:1081000000212046F9F706FE204627F0B7FB8D49EF
:10811000204627F0F3FB00212046F9F7FBFD20461F
:1081200027F0ACFB2220FAF74FF9F06A29F03CFE69
:108130000021FAF7FBF82968204627F0DFFB002131
:108140002046F9F7E7FD204627F098FB7E492046B8
:1081500027F0D4FB00212046F9F7DCFD204627F06C
:108160008DFB2220FAF730F9D6F87480B8F1000FB1
:1081700041F0E3857549204627F0C0FB2046414683
:10818000F9F7C8FD204627F079FB2968204627F03B
:10819000B5FB00212046F9F7BDFD204627F06EFB18
:1081A0006B49204627F0AAFB00212046F9F7B2FDD3
:1081B000204627F063FB2220FAF706F9306F0021F2
:1081C000FAF7B4F82968204627F098FB00212046EA
:1081D000F9F7A0FD204627F051FB5E49204627F025
:1081E0008DFB00212046F9F795FD204627F046FB40
:1081F0002220FAF7E9F8D7F8E00029F0D1FD0021B4
:10820000FAF794F82968204627F078FB00212046E9
:10821000F9F780FD204627F031FB4F49204627F033
:108220006DFB00212046F9F775FD204627F026FB5F
:108230002220FAF7C9F8D7F8DC0029F0B1FDFFF7E2
:108240002EB83C49204627F059FB00212046F9F77B
:1082500061FD204627F012FB2220FAF7B5F83F49CE
:10826000204627F04BFB00212046F9F753FD20461E
:1082700027F004FB2968204627F040FB0021204618
:10828000F9F748FD204627F0F9FA2D49204627F056
:1082900035FB00212046F9F73DFD204627F0EEFA98
:1082A0002220FAF791F8B06B29F07AFD0021FAF755
:1082B0003DF82968204627F021FB00212046F9F7E8
:1082C00029FD204627F0DAFA1E49204627F016FB42
:1082D00000212046F9F71EFD204627F0CFFA222084
:1082E000FAF772F8306E29F05BFD0021FAF71EF8FC
:1082F0002968204627F002FB00212046F9F70AFDF5
:10830000204627F0BBFA0D49204627F0F7FA002156
:108310002046F9F7FFFC204627F0B0FA2220FAF7B2
:1083200053F8F06C29F03CFDFEF7B9BFE06E030096
:108330006488FF1FEC6E03007C670300046F03007A
:108340001C6F0300346F03004C6F0300646F030065
:108350006C6F0300846F03009C6F0300A49C0300F8
:10836000AF49204627F0CAFA00212046F9F7D2FC8F
:10837000204627F083FA2220FAF726F8A94920465A
:1083800027F0BCFA00212046F9F7C4FC204627F06C
:1083900075FA2968204627F0B1FA00212046F9F73E
:1083A000B9FC204627F06AFA9F49204627F0A6FA32
:1083B00000212046F9F7AEFC204627F05FFA222084
:1083C000FAF702F8706A29F0EBFC0021F9F7AEFF2A
:1083D0002968204627F092FA00212046F9F79AFCF6
:1083E000204627F04BFA9149204627F087FA0021D2
:1083F0002046F9F78FFC204627F040FA2220F9F7B3
:10840000E3FFB06A29F0CCFC0021F9F78FFF29685F
:10841000204627F073FA00212046F9F77BFC20461E
:1084200027F02CFA8249204627F068FA00212046DE
:10843000F9F770FC204627F021FA2220F9F7C4FF53
:10844000F06B29F0ADFCFEF72ABF7549204627F0F6
:1084500055FA00212046F9F75DFC204627F00EFA78
:108460002220F9F7B1FF7349204627F047FA00218F
:108470002046F9F74FFC204627F000FA29682046ED
:1084800027F03CFA00212046F9F744FC204627F06B
:10849000F5F96549204627F031FA00212046F9F721
:1084A00039FC204627F0EAF92220F9F78DFFF06920
:1084B00029F076FC0021F9F739FF2968204627F0DA
:1084C0001DFA00212046F9F725FC204627F0D6F9B1
:1084D0005649204627F012FA00212046F9F71AFCE7
:1084E000204627F0CBF92220F9F76EFF306A29F0F9
:1084F00057FC0021F9F71AFF2968204627F0FEF9FA
:1085000000212046F9F706FC204627F0B7F9484934
:10851000204627F0F3F900212046F9F7FBFB20461F
:1085200027F0ACF92220F9F74FFFB06B29F038FCA7
:10853000FEF7B5BE3A49204627F0E0F90021204673
:10854000F9F7E8FB204627F099F92220F9F73CFFDC
:108550003949204627F0D2F900212046F9F7DAFB05
:10856000204627F08BF92968204627F0C7F900211B
:108570002046F9F7CFFB204627F080F92A4920460C
:1085800027F0BCF900212046F9F7C4FB204627F06C
:1085900075F92220F9F718FF706929F001FC002114
:1085A000F9F7C4FE2968204627F0A8F900212046E3
:1085B000F9F7B0FB204627F061F91C49204627F067
:1085C0009DF900212046F9F7A5FB204627F056F932
:1085D0002220F9F7F9FEB06929F0E2FB0021F9F752
:1085E000A5FE2968204627F089F900212046F9F7E1
:1085F00091FB204627F042F90D49204627F07EF9ED
:1086000000212046F9F786FB204627F037F9222083
:10861000F9F7DAFE706B29F0C3FBFEF740BE00BF2E
:10862000EC6E0300647D03001C6F0300346F0300D5
:10863000046F0300147D0300A49C0300E549204659
:1086400027F05CF900212046F9F764FB204627F06B
:1086500015F92220F9F7B8FEDF49204627F04EF938
:1086600000212046F9F756FB204627F007F9296834
:10867000204627F043F900212046F9F74BFB20461E
:1086800027F0FCF8D549204627F038F9002120468C
:10869000F9F740FB204627F0F1F82220F9F794FE85
:1086A000F06829F07DFB0021F9F740FE296820469B
:1086B00027F024F900212046F9F72CFB204627F06B
:1086C000DDF8C749204627F019F900212046F9F7BF
:1086D00021FB204627F0D2F82220F9F775FE3069F9
:1086E00029F05EFB0021F9F721FE2968204627F0DA
:1086F00005F900212046F9F70DFB204627F0BEF8CA
:10870000B849204627F0FAF800212046F9F702FB85
:10871000204627F0B3F82220F9F756FE306B29F0F7
:108720003FFBFEF7BCBDAB49204627F0E7F8002130
:108730002046F9F7EFFA204627F0A0F82220F9F7B3
:1087400043FEA949204627F0D9F800212046F9F731
:10875000E1FA204627F092F82968204627F0CEF863
:1087600000212046F9F7D6FA204627F087F89D49E0
:10877000204627F0C3F800212046F9F7CBFA20461F
:1087800027F07CF82220F9F71FFE706A29F00CFB15
:108790000021F9F7CBFD2968204627F0AFF800212A
:1087A0002046F9F7B7FA204627F068F88B492046AB
:1087B00027F0A4F800212046F9F7ACFA204627F06C
:1087C0005DF82220F9F700FE306929F0EDFA00216A
:1087D000F9F7ACFD2968204627F090F800212046E3
:1087E000F9F798FA204627F049F87D49204627F006
:1087F00085F800212046F9F78DFA204627F03EF84B
:108800002220F9F7E1FDB06B90E47249204627F091
:1088100075F800212046F9F77DFA204627F02EF85A
:108820002220F9F7D1FD7149204627F067F8002191
:108830002046F9F76FFA204627F020F829682046ED
:1088400027F05CF800212046F9F764FA204627F06B
:1088500015F86449204627F051F800212046F9F721
:1088600059FA204627F00AF82220F9F7ADFD306AC0
:1088700029F09AFA0021F9F759FD2968204627F0D6
:108880003DF800212046F9F745FA204626F0F6FF8C
:108890005249204627F032F800212046F9F73AFAEB
:1088A000204626F0EBFF2220F9F78EFDF06829F034
:1088B0007BFA0021F9F73AFD2968204627F01EF8D7
:1088C00000212046F9F726FA204626F0D7FF444932
:1088D000204627F013F800212046F9F71BFA20461E
:1088E00026F0CCFF2220F9F76FFD706B1EE43949AA
:1088F000204627F003F800212046F9F70BFA20461E
:1089000026F0BCFF2220F9F75FFD3949204626F00A
:10891000F5FF00212046F9F7FDF9204626F0AEFFCD
:108920002968204626F0EAFF00212046F9F7F2F9EF
:10893000204626F0A3FF2B49204626F0DFFF00212A
:108940002046F9F7E7F9204626F098FF2220F9F7AC
:108950003BFDF06929F028FA0021F9F7E7FC2968C6
:10896000204626F0CBFF00212046F9F7D3F9204618
:1089700026F084FF1949204626F0C0FF002120463A
:10898000F9F7C8F9204626F079FF2220F9F71CFDF7
:10899000B06829F009FA0021F9F7C8FC29682046D7
:1089A00026F0ACFF00212046F9F7B4F9204626F066
:1089B00065FF0B49204626F0A1FF00212046F9F76C
:1089C000A9F9204626F05AFF2220F9F7FDFC306B6A
:1089D000FFF7ACBBEC6E03007C6703001C6F030069
:1089E000346F0300046F0300647D0300147D0300F3
:1089F000A49C0300C849C94F204626F07FFF0021F0
:108A00002046F9F787F9204626F038FF2220F9F7AB
:108A1000DBFCC349204626F071FF00212046F9F710
:108A200079F9204626F02AFF2968204626F066FFBD
:108A300000212046F9F76EF9204626F01FFFB949BC
:108A4000204626F05BFF00212046F9F763F9204617
:108A500026F014FF2220F9F7B7FCD7F80080B8F110
:108A6000000F41F0E082B049204626F047FF204643
:108A70004146F9F74FF9204626F000FF29682046C5
:108A800026F03CFF00212046F9F744F9204626F065
:108A9000F5FEA649204626F031FF00212046F9F7D1
:108AA00039F9204626F0EAFE2220F9F78DFC002154
:108AB000F868F9F73BFC2968204626F01FFF0021E3
:108AC0002046F9F727F9204626F0D8FE7B68012BCF
:108AD00001F09982C1F07182302B01F06E82312B4E
:108AE00001F091829249204626F008FF002120469D
:108AF000F9F710F9204626F0C1FE2220F9F764FCB0
:108B0000376B002F41F00C818A49204626F0F6FE93
:108B100020463946F9F7FEF8204626F0AFFE2968D0
:108B2000204626F0EBFE00212046F9F7F3F8204618
:108B300026F0A4FE8049204626F0E0FE00212046D3
:108B4000F9F7E8F8204626F099FE2220F9F73CFCD8
:108B5000F06AFEF7A4BB7049784F204626F0CEFE9F
:108B600000212046F9F7D6F8204626F087FE22207D
:108B7000F9F72AFC7249204626F0C0FE0021204663
:108B8000F9F7C8F8204626F079FE2968204626F035
:108B9000B5FE00212046F9F7BDF8204626F06EFE0E
:108BA0006049204626F0AAFE00212046F9F7B2F8D7
:108BB000204626F063FE2220F9F706FCD7F8008055
:108BC000B8F1000F41F07D835749204626F096FE0C
:108BD00020464146F9F79EF8204626F04FFE2968C8
:108BE000204626F08BFE00212046F9F793F8204618
:108BF00026F044FE4D49204626F080FE0021204606
:108C0000F9F788F8204626F039FE2220F9F7DCFB38
:108C100005214DE740494B4F204626F06FFE0021CD
:108C20002046F9F777F8204626F028FE2220F9F7AB
:108C3000CBFB4549204626F061FE00212046F9F78E
:108C400069F8204626F01AFE2968204626F056FECE
:108C500000212046F9F75EF8204626F00FFE314944
:108C6000204626F04BFE00212046F9F753F8204617
:108C700026F004FE2220F9F7A7FBD7F80080B8F110
:108C8000000F41F02B832849204626F037FE20466E
:108C90004146F9F73FF8204626F0F0FD29682046C6
:108CA00026F02CFE00212046F9F734F8204626F065
:108CB000E5FD1E49204626F021FE00212046F9F759
:108CC00029F8204626F0DAFD2220F9F77DFB042161
:108CD000EEE611491D4F204626F010FE00212046E9
:108CE000F9F718F8204626F0C9FD2220F9F76CFBA9
:108CF00017498FE60849174F204626F0FFFD00214F
:108D00002046F9F707F8204626F0B8FD2220F9F7AB
:108D10005BFB11497EE600BF046F0300EC92FF1F6E
:108D2000508D03001C6F0300B4720300346F030006
:108D3000D46F0300646F0300EC6F0300B49AFF1F4D
:108D4000448D0300C89AFF1F688D03000C93FF1F1A
:108D50005C8D0300D89AFF1FD07E0300B549B64C46
:108D600005A826F0CBFD002105A8F8F7D3FF05A83C
:108D700026F084FD2220F9F727FBB04905A826F04C
:108D8000BDFD002105A8F8F7C5FF05A826F076FD72
:108D9000216805A826F0B2FD002105A8F8F7BAFF62
:108DA00005A826F06BFDA64905A826F0A7FD002121
:108DB00005A8F8F7AFFF05A826F060FD2220F9F717
:108DC00003FBB06A28F0F0FF0021F9F7AFFA216841
:108DD00005A826F093FD002105A8F8F79BFF05A83C
:108DE00026F04CFD974905A826F088FD002105A82E
:108DF000F8F790FF05A826F041FD2220F9F7E4FAE4
:108E0000306828F0D1FF0021F9F790FA216805A811
:108E100026F074FD002105A8F8F77CFF05A826F0D0
:108E20002DFD894905A826F069FD002105A8F8F760
:108E300071FF05A826F022FD2220F9F7C5FA706916
:108E400028F0B2FF0021F9F771FA216805A826F091
:108E500055FD05A80021F8F75DFF05A826F00EFDD9
:108E600020B0BDE8F0877349734C05A826F046FD95
:108E7000002105A8F8F74EFF05A826F0FFFC2220E8
:108E8000F9F7A2FA714905A826F038FD002105A8D6
:108E9000F8F740FF05A826F0F1FC216805A826F0A8
:108EA0002DFD002105A8F8F735FF05A826F0E6FC02
:108EB000654905A826F022FD002105A8F8F72AFF3C
:108EC00005A826F0DBFC2220F9F77EFA706A28F06C
:108ED0006BFF0021F9F72AFA216805A826F00EFD9C
:108EE000002105A8F8F716FF05A826F0C7FC55498C
:108EF00005A826F003FD002105A8F8F70BFF05A83B
:108F000026F0BCFC2220F9F75FFA306928F04CFF0C
:108F10000021F9F70BFA216805A826F0EFFC0021E3
:108F200005A8F8F7F7FE05A826F0A8FC444905A80F
:108F300026F0E4FC002105A8F8F7ECFE05A826F0D1
:108F40009DFC2220F9F740FAB06B79E739493A4C99
:108F500005A826F0D3FC002105A8F8F7DBFE05A83C
:108F600026F08CFC2220F9F72FFA394905A826F0C3
:108F7000C5FC002105A8F8F7CDFE05A826F07EFC6B
:108F8000216805A826F0BAFC002105A8F8F7C2FE62
:108F900005A826F073FC2C4905A826F0AFFC00219B
:108FA00005A8F8F7B7FE05A826F068FC2220F9F717
:108FB0000BFA306A28F0F8FE0021F9F7B7F92168BA
:108FC00005A826F09BFC002105A8F8F7A3FE05A83C
:108FD00026F054FC1B4905A826F090FC002105A8AA
:108FE000F8F798FE05A826F049FC2220F9F7ECF9DD
:108FF000F06828F0D9FE0021F9F798F9216805A852
:1090000026F07CFC002105A8F8F784FE05A826F0D0
:1090100035FC0B4905A826F071FC002105A8F8F7DE
:1090200079FE05A826F02AFC2220F9F7CDF9706B0D
:1090300006E700BFC86E0300A087FF1F307C030057
:10904000EC6E0300986E0300B06E0300647D0300B5
:10905000147D0300B049B14C05A826F04FFC002157
:1090600005A8F8F757FE05A826F008FC2220F9F716
:10907000ABF9AB4905A826F041FC002105A8F8F79B
:1090800049FE05A826F0FAFB216805A826F036FC63
:10909000002105A8F8F73EFE05A826F0EFFBA14940
:1090A00005A826F02BFC002105A8F8F733FE05A83B
:1090B00026F0E4FB2220F9F787F9F06928F074FE26
:1090C0000021F9F733F9216805A826F017FC0021E3
:1090D00005A8F8F71FFE05A826F0D0FB924905A8C1
:1090E00026F00CFC002105A8F8F714FE05A826F0D0
:1090F000C5FB2220F9F768F9B06828F055FE002179
:10910000F9F714F9216805A826F0F8FB002105A855
:10911000F8F700FE05A826F0B1FB844905A826F063
:10912000EDFB002105A8F8F7F5FD05A826F0A6FB44
:109130002220F9F749F9306B82E67749774C05A888
:1091400026F0DCFB002105A8F8F7E4FD05A826F0D1
:1091500095FB2220F9F738F9754905A826F0CEFBD2
:10916000002105A8F8F7D6FD05A826F087FB2168A1
:1091700005A826F0C3FB002105A8F8F7CBFD05A83C
:1091800026F07CFB674905A826F0B8FB002105A85E
:10919000F8F7C0FD05A826F071FB2220F9F714F9B5
:1091A000B06928F001FE0021F9F7C0F8216805A890
:1091B00026F0A4FB002105A8F8F7ACFD05A826F0D1
:1091C0005DFB594905A826F099FB002105A8F8F791
:1091D000A1FD05A826F052FB2220F9F7F5F87068EA
:1091E00028F0E2FD0021F9F7A1F8216805A826F092
:1091F00085FB002105A8F8F78DFD05A826F03EFBAC
:109200004A4905A826F07AFB002105A8F8F782FD57
:1092100005A826F033FB2220F9F7D6F8F06A0FE60E
:109220004449204626F06AFB00212046F8F772FDEB
:10923000204626F023FB2220F9F7C6F83E492046B7
:1092400026F05CFB00212046F8F764FD204626F05E
:1092500015FB2968204626F051FB20460021F8F72F
:1092600059FD204626F00AFBFDF796BA3349204601
:1092700026F044FB00212046F8F74CFD204626F05E
:10928000FDFA2220F9F7A0F82D49FDF734BF2B494C
:10929000204626F033FB00212046F8F73BFD204610
:1092A00026F0ECFA2220F9F78FF82649FDF723BFC4
:1092B0002249204626F022FB00212046F8F72AFD0D
:1092C000204626F0DBFA2220F9F77EF81E49FDF74A
:1092D00012BF1A49204626F011FB00212046F8F75C
:1092E00019FD204626F0CAFA2220F9F76DF8174931
:1092F000FDF701BF1149204626F000FB0021204662
:10930000F8F708FD204626F0B9FA2220F9F75CF8B4
:109310000F49FDF7F0BE00BFC86E0300A087FF1F16
:10932000A49C0300B06E0300986E0300EC6E030073
:109330007C6703004C6F03000C700300846F030014
:109340004C730300607303005C73030058730300E5
:10935000547303009549964D05A826F0CFFA0021D5
:1093600005A8F8F7D7FC05A826F088FA2220F9F717
:109370002BF8904905A826F0C1FA002105A8F8F7B6
:10938000C9FC05A826F07AFA296805A826F0B6FADD
:10939000002105A8F8F7BEFC05A826F06FFA86495B
:1093A00005A826F0ABFA002105A8F8F7B3FC05A83C
:1093B00026F064FA2220F9F707F8606828F0F0FC3C
:1093C0000021F8F7B3FF296805A826F097FA0021D5
:1093D00005A8F8F79FFC05A826F050FA774905A8DC
:1093E00026F08CFA002105A8F8F794FC05A826F0D1
:1093F00045FA2220F8F7E8FFA06828F0D1FC002108
:10940000F8F794FF296805A826F078FA002105A846
:10941000F8F780FC05A826F031FA694905A826F07E
:109420006DFA002105A8F8F775FC05A826F026FAC4
:109430002220F8F7C9FFE06828F0B2FC0021F8F715
:1094400075FF296805A826F059FA002105A8F8F744
:1094500061FC05A826F012FA5A4905A826F04EFA32
:10946000002105A8F8F756FC05A826F007FA2220E7
:10947000F8F7AAFF0021606BF8F758FF2968E5E4C8
:109480004A494B4D05A826F039FA002105A8F8F7FE
:1094900041FC05A826F0F2F92220F8F795FF4A4989
:1094A00005A826F02BFA002105A8F8F733FC05A83B
:1094B00026F0E4F9296805A826F020FA002105A87D
:1094C000F8F728FC05A826F0D9F93B4905A826F0AD
:1094D00015FA002105A8F8F71DFC05A826F0CEF91D
:1094E0002220F8F771FFA06A28F05AFC0021F8F753
:1094F0001DFF296805A826F001FA002105A8F8F744
:1095000009FC05A826F0BAF92C4905A826F0F6F9B9
:10951000002105A8F8F7FEFB05A826F0AFF92220E8
:10952000F8F752FFE06A28F03BFC0021F8F7FEFE56
:10953000296805A826F0E2F9002105A8F8F7EAFB5A
:1095400005A826F09BF91E4905A826F0D7F90021A9
:1095500005A8F8F7DFFB05A826F090F92220F8F718
:1095600033FF206B28F01CFC0021F8F7DFFE296890
:1095700005A826F0C3F9002105A8F8F7CBFB05A83C
:1095800026F07CF90F4905A826F0B8F9002105A8B6
:10959000F8F7C0FB05A826F071F92220F8F714FFB0
:1095A0000021206DF8F7C2FE29684FE4C86E030061
:1095B000A087FF1FD8720300B06E0300EC6E03009B
:1095C000986E0300046F0300007303009649974DE3
:1095D00005A826F093F9002105A8F8F79BFB05A83C
:1095E00026F04CF92220F8F7EFFE914905A826F065
:1095F00085F9002105A8F8F78DFB05A826F03EF9AE
:10960000296805A826F07AF9002105A8F8F782FB59
:1096100005A826F033F9874905A826F06FF900213F
:1096200005A8F8F777FB05A826F028F92220F8F717
:10963000CBFEE06928F0B4FB0021F8F777FE29683B
:1096400005A826F05BF9002105A8F8F763FB05A83B
:1096500026F014F9784905A826F050F9002105A84C
:10966000F8F758FB05A826F009F92220F8F7ACFE18
:10967000206A28F095FB0021F8F758FE296805A814
:1096800026F03CF9002105A8F8F744FB05A826F0D0
:10969000F5F86A4905A826F031F9002105A8F8F780
:1096A00039FB05A826F0EAF82220F8F78DFE606A5B
:1096B00028F076FB0021F8F739FE296805A826F086
:1096C0001DF9002105A8F8F725FB05A826F0D6F816
:1096D0005B4905A826F012F9002105A8F8F71AFB46
:1096E00005A826F0CBF82220F8F76EFE0021E06CEA
:1096F000F8F71CFE2968FFF7A9BB4B494B4D05A89D
:1097000026F0FCF8002105A8F8F704FB05A826F0D0
:10971000B5F82220F8F758FE4A4905A826F0EEF8D9
:10972000002105A8F8F7F6FA05A826F0A7F8296899
:1097300005A826F0E3F8002105A8F8F7EBFA05A83C
:1097400026F09CF83B4905A826F0D8F8002105A88A
:10975000F8F7E0FA05A826F091F82220F8F734FE91
:10976000206928F01DFB0021F8F7E0FD296805A815
:1097700026F0C4F8002105A8F8F7CCFA05A826F0D1
:109780007DF82D4905A826F0B9F8002105A8F8F7BD
:10979000C1FA05A826F072F82220F8F715FE6069D4
:1097A00028F0FEFA0021F8F7C1FD296805A826F087
:1097B000A5F8002105A8F8F7ADFA05A826F05EF88F
:1097C0001E4905A826F09AF8002105A8F8F7A2FA84
:1097D00005A826F053F82220F8F7F6FDA06928F036
:1097E000DFFA0021F8F7A2FD296805A826F086F81F
:1097F000002105A8F8F78EFA05A826F03FF81049D1
:1098000005A826F07BF8002105A8F8F783FA05A83B
:1098100026F034F82220F8F7D7FD0021A06CF8F7E5
:1098200085FD2968FFF712BBC86E0300A087FF1FE4
:10983000F0720300B06E0300EC6E0300986E03003C
:10984000046F0300E47203009649974D05A826F0C3
:1098500055F8002105A8F8F75DFA05A826F00EF8DE
:109860002220F8F7B1FD914905A826F047F800211C
:1098700005A8F8F74FFA05A826F000F8296805A80A
:1098800026F03CF8002105A8F8F744FA05A825F0D1
:10989000F5FF874905A826F031F8002105A8F8F75B
:1098A00039FA05A825F0EAFF2220F8F78DFD606857
:1098B00028F076FA0021F8F739FD296805A826F086
:1098C0001DF8002105A8F8F725FA05A825F0D6FF10
:1098D000784905A826F012F8002105A8F8F71AFA29
:1098E00005A825F0CBFF2220F8F76EFDA06828F030
:1098F00057FA0021F8F71AFD296805A825F0FEFFA0
:10990000002105A8F8F706FA05A825F0B7FF6A496F
:1099100005A825F0F3FF002105A8F8F7FBF905A835
:1099200025F0ACFF2220F8F74FFDE06828F038FA68
:109930000021F8F7FBFC296805A825F0DFFF0021CE
:1099400005A8F8F7E7F905A825F098FF5B4905A8F1
:1099500025F0D4FF002105A8F8F7DCF905A825F0CB
:109960008DFF2220F8F730FD0021606CF8F7DEFC57
:109970002968FFF76BBA4B494B4D05A825F0BEFF90
:10998000002105A8F8F7C6F905A825F077FF2220E1
:10999000F8F71AFD4A4905A825F0B0FF002105A8EF
:1099A000F8F7B8F905A825F069FF296805A825F09A
:1099B000A5FF002105A8F8F7ADF905A825F05EFF81
:1099C0003B4905A825F09AFF002105A8F8F7A2F960
:1099D00005A825F053FF2220F8F7F6FCA06A28F02E
:1099E000DFF90021F8F7A2FC296805A825F086FF19
:1099F000002105A8F8F78EF905A825F03FFF2D49AD
:109A000005A825F07BFF002105A8F8F783F905A834
:109A100025F034FF2220F8F7D7FCE06A28F0C0F9DF
:109A20000021F8F783FC296805A825F067FF0021CD
:109A300005A8F8F76FF905A825F020FF1E4905A82D
:109A400025F05CFF002105A8F8F764F905A825F0CA
:109A500015FF2220F8F7B8FC206B28F0A1F90021AF
:109A6000F8F764FC296805A825F048FF002105A83F
:109A7000F8F750F905A825F001FF104905A825F0D1
:109A80003DFF002105A8F8F745F905A825F0F6FEE9
:109A90002220F8F799FC0021206CF8F747FC296890
:109AA000FFF7D4B9C86E0300A087FF1FDC72030064
:109AB000B06E0300EC6E0300986E0300046F0300A9
:109AC000F8720300BE49BF4D05A825F017FF00211D
:109AD00005A8F8F71FF905A825F0D0FE2220F8F711
:109AE00073FCB94905A825F009FF002105A8F8F77E
:109AF00011F905A825F0C2FE296805A825F0FEFE8B
:109B0000002105A8F8F706F905A825F0B7FEAF492A
:109B100005A825F0F3FE002105A8F8F7FBF805A835
:109B200025F0ACFE2220F8F74FFCE06928F038F968
:109B30000021F8F7FBFB296805A825F0DFFE0021CE
:109B400005A8F8F7E7F805A825F098FEA04905A8AC
:109B500025F0D4FE002105A8F8F7DCF805A825F0CB
:109B60008DFE2220F8F730FC206A28F019F9002138
:109B7000F8F7DCFB296805A825F0C0FE002105A840
:109B8000F8F7C8F805A825F079FE924905A825F050
:109B9000B5FE002105A8F8F7BDF805A825F06EFE72
:109BA0002220F8F711FC606A28F0FAF80021F8F793
:109BB000BDFB296805A825F0A1FE002105A8F8F73E
:109BC000A9F805A825F05AFE834905A825F096FEB8
:109BD000002105A8F8F79EF805A825F04FFE2220E1
:109BE000F8F7F2FB0021E06BF8F7A0FB2968FFF71C
:109BF0002DB97349734D05A825F080FE002105A8F5
:109C0000F8F788F805A825F039FE2220F8F7DCFBE4
:109C1000724905A825F072FE002105A8F8F77AF828
:109C200005A825F02BFE296805A825F067FE002170
:109C300005A8F8F76FF805A825F020FE634905A8E8
:109C400025F05CFE002105A8F8F764F805A825F0CA
:109C500015FE2220F8F7B8FB206928F0A1F80021B2
:109C6000F8F764FB296805A825F048FE002105A83F
:109C7000F8F750F805A825F001FE554905A825F08C
:109C80003DFE002105A8F8F745F805A825F0F6FDEA
:109C90002220F8F799FB606928F082F80021F8F794
:109CA00045FB296805A825F029FE002105A8F8F73D
:109CB00031F805A825F0E2FD464905A825F01EFE6D
:109CC000002105A8F8F726F805A825F0D7FD2220E1
:109CD000F8F77AFBA06928F063F80021F8F726FB73
:109CE000296805A825F00AFE002105A8F8F712F852
:109CF00005A825F0C3FD384905A825F0FFFD002182
:109D000005A8F8F707F805A825F0B8FD2220F8F710
:109D10005BFB0021A06BF8F709FB2968FFF796B8F9
:109D20002F49204625F0EAFD20460021F7F7F2FFF3
:109D3000204625F0A3FDFEF7F2BE2949204625F076
:109D4000DDFD20460021F7F7E5FF204625F096FDD2
:109D5000FEF71BBA012B0CBF22492349204625F0F0
:109D6000CDFD20463146F7F7D5FF204625F086FD8C
:109D7000FCF761BB1D49204625F0C0FD3946204651
:109D8000F7F7C8FF204625F079FD2220F8F71CFBE5
:109D90001749204625F0B2FD39462046F7F7BAFFAD
:109DA000204625F06BFD2968204625F0A7FD2046BA
:109DB0003946F7F7AFFF204625F060FDFCF751BFAD
:109DC000C86E0300A087FF1FE8720300B06E030097
:109DD000EC6E0300986E0300046F0300E072030052
:109DE000686F0300B46F0300B86F0300EC6F0300EB
:109DF00008730300DB49204625F080FD31462046EC
:109E0000F7F788FF204625F039FD2220F8F7DCFA25
:109E1000D549204625F072FD31462046F7F77AFFF6
:109E2000204625F02BFD2968204625F067FD3146A8
:109E30002046F7F76FFF204625F020FDCB4920464E
:109E400025F05CFD31462046F7F764FF204625F0FB
:109E500015FD2220F8F7B8FAD8F8400027F0A0FF47
:109E60003146F8F763FA2968204625F047FD314668
:109E70002046F7F74FFF204625F000FDBC4920465D
:109E800025F03CFD31462046F7F744FF204625F0FB
:109E9000F5FC2220F8F798FA3146D8F85000F8F788
:109EA00045FA2968204625F029FD31462046F7F776
:109EB00031FF204625F0E2FCAE49204625F01EFD8C
:109EC00031462046F7F726FF204625F0D7FC222012
:109ED000F8F77AFA3146D8F84C00F8F727FA2968EB
:109EE000204625F00BFD20463146F7F713FF2046AC
:109EF00025F0C4FCFCF7AFBD9A49204625F0FEFCD6
:109F000000212046F7F706FF204625F0B7FC222067
:109F1000F8F75AFA9849FFF792B99349204625F085
:109F2000EDFC20463946F7F7F5FE204625F0A6FC65
:109F3000FCF7B0BF9149204625F0E0FC39462046A9
:109F4000F7F7E8FE204625F099FC2220F8F73CFAC6
:109F50008549204625F0D2FC39462046F7F7DAFE3F
:109F6000204625F08BFC2968204625F0C7FC2046BA
:109F70003946F7F7CFFE204625F080FCFCF775BF89
:109F80007F49204625F0BAFC00212046F7F7C2FEA3
:109F9000204625F073FC2220F8F716FA7949FCF7E1
:109FA0009ABF7949FBF779BD7749FCF795B87649AF
:109FB000FBF7A2BF7449FCF7D0B96A49204625F0E7
:109FC0009DFC00212046F7F7A5FE204625F056FC13
:109FD0002220F8F7F9F96D49204625F08FFC002181
:109FE0002046F7F797FE204625F048FC29682046D2
:109FF00025F084FC20460021F7F78CFE204625F052
:10A000003DFCFEF76FBD5749204625F077FC002147
:10A010002046F7F77FFE204625F030FC2220F8F797
:10A02000D3F95B49D8E75B49204625F067FC204619
:10A030000021F7F76FFE204625F020FCFEF71EBD3D
:10A0400020465549554D25F059FC39462046F7F72D
:10A0500061FE204625F012FC2220F8F7B5F92046D3
:10A060004F4925F04BFC39462046F7F753FE204672
:10A0700025F004FC2968204625F040FC394620469E
:10A08000F7F748FE204625F0F9FB2A21454824F041
:10A0900005FE3B460A227169434825F0A3F9424870
:10A0A00025F08CF92046414925F028FC3946204608
:10A0B000F7F730FE204625F0E1FB2220F8F784F97F
:10A0C000706927F06DFE3946F8F730F929682046A7
:10A0D00025F014FC39462046F7F71CFE204625F0F3
:10A0E000CDFB2046324925F009FC39462046F7F7DA
:10A0F00011FE204625F0C2FB2220F8F765F9B06872
:10A1000027F04EFE3946F8F711F92968204625F068
:10A11000F5FB39462046F7F7FDFD204625F0AEFB5E
:10A120002046244925F0EAFB39462046F7F7F2FDA0
:10A13000204625F0A3FB2220F8F746F9306A27F0E5
:10A140002FFE3946F8F7F2F82968204625F0D6FBAD
:10A1500020463946F7F7DEFD204625F08FFBFCF759
:10A160005BBA00BF4C6F0300087303006C6F030001
:10A17000D46F0300EC6F0300047003009C6F0300B6
:10A18000846F030084730300686F0300C8720300C8
:10A19000D0720300C0720300C86E0300A087FF1FC7
:10A1A000307C0300887203006488FF1F986E0300F0
:10A1B000B06E0300EC6E03004F49504D204625F071
:10A1C0009DFB00212046F7F7A5FD204625F056FB14
:10A1D0002220F8F7F9F84A49204625F08FFB0021A4
:10A1E0002046F7F797FD204625F048FB29682046D2
:10A1F00025F084FB00212046F7F78CFD204625F052
:10A200003DFB4049204625F079FB00212046F7F729
:10A2100081FD204625F032FB2220F8F7D5F8B06901
:10A2200027F0BEFD0021F8F781F82968204625F0C7
:10A2300065FB00212046F7F76DFD204625F01EFB4B
:10A240003149204625F05AFB00212046F7F762FDF0
:10A25000204625F013FB2220F8F7B6F8F06827F027
:10A260009FFD0021F8F762F82968204625F046FB9B
:10A2700000212046F7F74EFD204625F0FFFA23493E
:10A28000204625F03BFB00212046F7F743FD204602
:10A2900025F0F4FA2220F8F797F8706AFDF784B9F0
:10A2A0001A49204625F02AFB00212046F7F732FD07
:10A2B000204625F0E3FA2220F8F786F8B06DFDF786
:10A2C00035BF1349204625F019FB20460021F7F73A
:10A2D00021FD204625F0D2FAFEF781BC0C4920462C
:10A2E00025F00CFB20460021F7F714FD204625F051
:10A2F000C5FAFEF7D3BC00BFC86E0300A087FF1FDE
:10A30000147D0300986E0300B06E0300EC6E030032
:10A31000C072030030B585B005465449544C6846B8
:10A3200025F0ECFA00216846F7F7F4FC684625F0C2
:10A33000A5FA284627F034FD0021F7F7F7FF21683A
:10A34000684625F0DBFA68460021F7F7E3FC68462B
:10A3500025F094FA6846474925F0D0FA002168466E
:10A36000F7F7D8FC684625F089FA434B187827F0B0
:10A3700017FD0021F7F7DAFF2168684625F0BEFADD
:10A3800068460021F7F7C6FC684625F077FA68466C
:10A390003A4925F0B3FA00216846F7F7BBFC684656
:10A3A00025F06CFA364B187827F0FAFC0021F7F705
:10A3B000BDFF2168684625F0A1FA68460021F7F73D
:10A3C000A9FC684625F05AFA68462E4925F096FA07
:10A3D00000216846F7F79EFC684625F04FFA2A4BA5
:10A3E000187827F0DDFC0021F7F7A0FF2168684608
:10A3F00025F084FA68460021F7F78CFC684625F0C2
:10A400003DFA6846214925F079FA00216846F7F7B8
:10A4100081FC684625F032FA1D4B187827F0C0FC05
:10A420000021F7F783FF2168684625F067FA684640
:10A430000021F7F76FFC684625F020FA68461549B9
:10A4400025F05CFA68460021F7F764FC684625F0C1
:10A4500015FA2168684625F051FA68460021F7F799
:10A4600059FC684625F00AFA05B030BD9873030020
:10A47000A487FF1FB07303001C98FF1FC473030061
:10A48000C49AFF1FD87303005494FF1FEC7303009A
:10A49000C497FF1F007403002DE9F04F0646ABB0D0
:10A4A0000F46AF480E219146984624F0F7FBAD4881
:10A4B00029F0C6F90146AB4824F0F0FBAA4824F085
:10A4C0007DFF0E21A64824F0E9FBA64829F0B8F943
:10A4D0000146A44824F0E2FBA34824F06FFF0023C8
:10A4E00009A81A469F4921F053FF149C002C36D02E
:10A4F00023689E4A1B6B93422BD1236D002B00F0E7
:10A500009C8123689A4DDB6AAB4240F09282A06D39
:10A5100018B128F0E3F80023A365236D002B00F0A9
:10A52000C78204F1180020F099FDDDF850A0DAF898
:10A530000440013CCAF80440002C00F03A828D4DE2
:10A54000002314939DF83E30012B0DD144F20223D9
:10A550000FE02046984710B1149C002CD1D19DF8F3
:10A560003E30844D012BF1D0022B40F2022318BF64
:10A57000002316A809AA804920F05AFE289B002B28
:10A5800057D05C2024F0D8FE04467C4A9DF85C003D
:10A59000189B7B4922604FF0000A9DF864202073CD
:10A5A000A16023611AA9227504F11800C4F804A05F
:10A5B00020F026FD6368734AA26001336360C4F82B
:10A5C00058A01AA8169520F049FD6368149A013323
:10A5D0006360002A00F0E1815368013B5360002B67
:10A5E0007AD01494002C2FD06368013B6360002B59
:10A5F00000F0D480149838B303685C4A1B6B934214
:10A6000040F0CD81036D002B00F0CE81002450225C
:10A6100016A909A88DF83F4022F01AF8002840F04A
:10A62000F280002509A821F0DFFE28462BB0BDE806
:10A63000F08F299C002CA4D11AA8169520F00EFDAD
:10A64000149A002AC8D1149201234F498DF83F3043
:10A6500016A825F053F94D4C002116A8F7F75AFB20
:10A6600016A825F00BF9216816A825F047F9002156
:10A6700016A8F7F74FFB16A825F000F9444916A8CD
:10A6800025F03CF9002116A8F7F744FB16A825F0A1
:10A69000F5F8216816A825F031F9002116A8F7F77A
:10A6A00039FB16A825F0EAF83A4916A825F026F94C
:10A6B000002116A8F7F72EFB16A825F0DFF8216871
:10A6C00016A825F01BF916A80021F7F723FB16A8FA
:10A6D000002525F0D3F8A5E711682548C96A02933B
:10A6E000814240F09D81906D28B1039227F0F6FFE2
:10A6F000039A029B9365136D002B00F0CE8102F14B
:10A70000180020F0ABFCDDF850A0BAF1000F3FF4C8
:10A7100068AFDAF80030204A5B68934240F08681E7
:10A72000DAF85800154BCAF8003020B127F0D6FFF0
:10A730000023CAF85830DAF850300AF1180B002B11
:10A7400000F0B081584620F089FCCAF808505846FD
:10A7500020F084FC50465C2124F0F2FD41E700BF6C
:10A760000C7403002093FF1F6488FF1F7504000012
:10A770006D05000094620300749BFF1F08630300D3
:10A7800070620300B86203001C740300A487FF1FFB
:10A79000CC89030044850300590D00002268B149AB
:10A7A000D26A02938A4240F03E81A06D18B127F030
:10A7B00095FF029BA365236D002B00F0498104F1F6
:10A7C000180020F04BFC2368A74A5B68934240F0D6
:10A7D0006181A06DA54B236018B127F07FFF002396
:10A7E000A365236D04F1180A002B00F06681504622
:10A7F00020F034FCA560504620F030FC20465C215F
:10A8000024F09EFDF6E6502300933A4616AB3146FF
:10A8100009A822F08DF8A8B9954A136805930599FF
:10A8200013680493049B5B1A632BF9D916A827F0CD
:10A83000F5FE27F0AFF90546F4E6636D002B7FF4D3
:10A8400060AE8CE68B4905A825F058F805A821468E
:10A85000F7F760FA05A825F011F8B8F1000F00F03D
:10A86000EB802220F7F7B0FD16A905A825F046F8E1
:10A87000214605A8F7F74EFA05A824F0FFFF22208D
:10A88000F7F7A2FD7C497D4C05A825F037F800219B
:10A8900005A8F7F73FFA05A824F0F0FF484627F08F
:10A8A00083FA0021F7F742FD754B05A8196825F0DA
:10A8B00025F8002105A8F7F72DFA05A824F0DEFFFA
:10A8C000704905A825F01AF8002105A8F7F722FA23
:10A8D00005A824F0D3FF2220F7F776FD314605A81E
:10A8E00025F00CF8002105A8F7F714FA05A824F0C4
:10A8F000C5FF216805A825F001F8002105A8F7F794
:10A9000009FA05A824F0BAFF5F4905A824F0F6FF6C
:10A91000002105A8F7F7FEF905A824F0AFFF2220D3
:10A92000F7F752FD394605A824F0E8FF002105A8F5
:10A93000F7F7F0F905A824F0A1FF216805A824F095
:10A94000DDFF002105A8F7F7E5F905A824F096FF3B
:10A950004E4905A824F0D2FF002105A8F7F7DAF93F
:10A9600005A824F08BFF2220F7F72EFD16A905A8D5
:10A9700024F0C4FF002105A8F7F7CCF905A824F0BE
:10A980007DFF216805A824F0B9FF05A80021F7F78D
:10A99000C1F905A824F072FF3EE7149425E6984714
:10A9A00000283FF451AE31E6436D002B7FF42EAE0C
:10A9B0004AE6DAF80030DB6AAB4240F08380DAF82E
:10A9C000580018B127F08AFECAF85840DAF850301B
:10A9D000002B7DD00AF1180020F040FB149C002CC5
:10A9E0003FF4ADAD2368204A5B6893426DD1A06D02
:10A9F0001E4B236018B127F071FE0023A365236D61
:10AA000004F1180A4BB3504620F028FB204DA560F6
:10AA1000504620F023FB20465C2124F091FC8FE57A
:10AA2000104688476FE620469047CCE65046984748
:10AA3000D7E52046984778E516A905A824F05EFFDB
:10AA400005A84146F7F766F905A824F017FF19E7AE
:10AA5000636D002B7FF4B3AEB5E6636D002BD2D1EE
:10AA6000D4E700BF6D050000590D00000863030026
:10AA70007CA0FF1F2874030030740300A087FF1F11
:10AA8000A487FF1F34740300487403005C74030040
:10AA90009462030020469847ACE5536D002B7FF489
:10AAA0002EAE30E6DAF85430002B7FF44BAE4CE695
:10AAB000636D002B7FF435AD37E5636D002B7FF4BC
:10AAC00096AE97E65046984788E72046984736E581
:10AAD000DAF85430002B7FF47DAF7FE738B5124DA4
:10AAE0001249134C284600234FF4BA72FFF7D4FCE6
:10AAF0000023E0604FF4F8720E492846FFF7CCFCC3
:10AB000027F082FB012320614FF41B7228460A497B
:10AB1000FFF7C2FC094BA061196820466C22BDE812
:10AB2000384022F059B800BF8074030070740300ED
:10AB3000E898FF1F8C7403009C7403008487FF1F38
:10AB400038B50D4D0D490E4C284601234FF41972AE
:10AB5000FFF7A2FC0123A0644FF41D7228460949A7
:10AB6000FFF79AFC084B6064196820464C22BDE848
:10AB7000384022F031B800BF24820300AC740300D7
:10AB8000CC97FF1FB87403007087FF1F38B51E4DA8
:10AB90001E491F4C00234FF40B722846FFF77CFC24
:10ABA00027F032FB012320644FF49A72284619499A
:10ABB000FFF772FC01232065E82228461649FFF7BB
:10ABC0006BFC0023E0644FF4397214492846FFF708
:10ABD00063FC27F019FB0123E0634FF43A72284627
:10ABE0000F49FFF759FC0123A0644FF4A2722846D5
:10ABF0000C49FFF751FC0C4B606419682046602239
:10AC0000BDE8384021F0E8BFD4740300C4740300E9
:10AC10005C96FF1FDC740300F47403000C750300E2
:10AC200018750300307503009887FF1F38B5394D3C
:10AC300039493A4C00234FF43E722846FFF72CFC6A
:10AC400027F0E2FA002360674FF43F723449284648
:10AC5000FFF722FC27F0D8FA0023A0674FF44072D8
:10AC600030492846FFF718FC27F0CEFA0023E067AA
:10AC70004FF441722C492846FFF70EFC27F0C4FA26
:10AC80000023C4F880004FF4447228492846FFF797
:10AC900003FC27F0B9FA0023C4F884004FF445728E
:10ACA00023492846FFF7F8FB27F0AEFA0023C4F843
:10ACB00088004FF442721F492846FFF7EDFB27F04A
:10ACC000A3FA0023C4F88C004FF443721A492846B3
:10ACD000FFF7E2FB27F098FA0023C4F8900038222F
:10ACE00016492846FFF7D8FB27F08EFA0023C4F850
:10ACF0009400542212492846FFF7CEFB27F084FA2D
:10AD0000104BC4F8980019682046E422BDE838408A
:10AD100021F062BF5875030044750300BC96FF1F05
:10AD20006075030070750300807503009075030063
:10AD3000A0750300B0750300C4750300D47503004B
:10AD4000E8750300D895FF1F2DE9F0430746ABB027
:10AD500088469F480E2123F0A1FF9E4828F070FDF1
:10AD600001469C4823F09AFF9B4824F027FB0023D0
:10AD700009A81A46974921F00BFB149C002C33D0EC
:10AD80002368964A1B6B934228D1236D002B00F059
:10AD90008A812368924EDB6AB34240F03E82A06D06
:10ADA00018B127F09BFC0023A365236D002B00F056
:10ADB0004D8204F1180020F051F9149D6C68013C9B
:10ADC0006C60002C00F0EE81864E002314939DF8F9
:10ADD0003E30012B0DD144F202230FE0204698476C
:10ADE00010B1149C002CD4D19DF83E307D4E012B27
:10ADF000F1D0022B40F2022318BF002316A809AAA3
:10AE0000794920F015FA289B002B54D05C2024F0BF
:10AE100093FA0446754B9DF85C00189A74492360B8
:10AE200000259DF864302073A16022611AA9237562
:10AE3000656004F1180020F0E3F863686D4AA565C9
:10AE4000013363601AA8A260169620F007F96368C0
:10AE5000149D01336360002D00F098816B68013B05
:10AE60006B60002B7AD01494002C2FD063685D1E89
:10AE70006560002D00F0CA80149838B30368574A03
:10AE80001B6B934240F08481036D002B00F08581A1
:10AE90000024502216A909A88DF83F4021F0D8FBC4
:10AEA000002840F0E680002509A821F09DFA2846F8
:10AEB0002BB0BDE8F083299C002CA7D11AA81696C8
:10AEC00020F0CCF8149D002DC8D1149501234A49D7
:10AED0008DF83F3016A824F011FD484C002116A82B
:10AEE000F6F718FF16A824F0C9FC216816A824F06C
:10AEF00005FD002116A8F6F70DFF16A824F0BEFCEC
:10AF00003F4916A824F0FAFC002116A8F6F702FF24
:10AF100016A824F0B3FC216816A824F0EFFC002149
:10AF200016A8F6F7F7FE16A824F0A8FC354916A8CF
:10AF300024F0E4FC002116A8F6F7ECFE16A824F095
:10AF40009DFC216816A824F0D9FC16A80021F6F76C
:10AF5000E1FE16A8002524F091FCA5E72A68204907
:10AF6000D26A03938A4240F04F81A86D18B127F04E
:10AF7000B5FB039BAB652B6D002B00F05D8105F1EC
:10AF8000180020F06BF8149D002D3FF46CAF2B6877
:10AF90001D4A5B68934240F03D81A86D134B2B60C6
:10AFA00018B127F09BFB0023AB652B6D05F1180949
:10AFB000002B00F04681484620F050F8AE6048462D
:10AFC00020F04CF828465C2124F0BAF94BE700BF8A
:10AFD0000C7403002093FF1F6488FF1F750400009A
:10AFE0006D05000094620300749BFF1F086303005B
:10AFF00070620300B86203001C740300A487FF1F83
:10B00000CC89030044850300590D00002368994A48
:10B01000DB6A934240F0FB80A06D10B127F05EFB2D
:10B02000A565236D002B00F0FB8004F1180020F0D3
:10B0300015F82368904A5B68934240F0FA80A06D4F
:10B040008E4B236018B127F049FB0023A365236DC5
:10B0500004F11805002B00F0FE8028461FF0FEFFCB
:10B06000A66028461FF0FAFF20465C2124F068F90C
:10B0700002E750230093424616AB394609A821F057
:10B0800057FCA8B97E4A1368059305991368049381
:10B09000049B5B1A632BF9D916A827F0BFFA26F098
:10B0A00079FD054600E7636D002B7FF472AE9BE6E9
:10B0B00005A87449744D24F021FC214605A8F6F733
:10B0C00029FE05A824F0DAFB2220F7F77DF939469E
:10B0D00005A824F013FC214605A8F6F71BFE05A8D9
:10B0E00024F0CCFB296805A824F008FC214605A81B
:10B0F000F6F710FE05A824F0C1FB05A8634924F06B
:10B10000FDFB214605A8F6F705FE05A824F0B6FBD1
:10B110002220F7F759F9414605A824F0EFFB214614
:10B1200005A8F6F7F7FD05A824F0A8FB296805A8EF
:10B1300024F0E4FB214605A8F6F7ECFD05A824F071
:10B140009DFB05A8524924F0D9FB214605A8F6F736
:10B15000E1FD05A824F092FB2220F7F735F916A9A6
:10B1600005A824F0CBFB214605A8F6F7D3FD05A8DA
:10B1700024F084FB296805A824F0C0FB05A821461B
:10B18000F6F7C8FD05A824F079FB7BE714946EE67A
:10B19000984700283FF49AAE7AE6436D002B7FF47F
:10B1A00077AE93E62B68DB6AB34259D1A86D10B134
:10B1B00027F094FAAC652B6D002B57D005F11800E1
:10B1C0001FF04CFF149C002C3FF4FEAD23682A4A6C
:10B1D0005B68934247D1A06D284B236018B127F0DC
:10B1E0007DFA0023A365236D04F11805EBB1284611
:10B1F0001FF034FF274EA66028461FF02FFF204681
:10B200005C2124F09DF8E0E528469047BBE6204607
:10B2100098470EE72846984725E620469847CCE50C
:10B22000636D002B7FF401AF03E7636D002BDED16C
:10B23000E0E7204698471FE66B6D002B7FF49FAE3A
:10B24000A1E66B6D002B7FF4B6AEB7E6636D002B05
:10B250007FF4AFADB1E5636D002B7FF4FEAEFFE68A
:10B2600028469847AEE720469847ADE56B6D002B22
:10B27000A4D1A7E76D050000590D00000863030085
:10B280007CA0FF1F34740300A087FF1F48740300D5
:10B290005C74030094620300F8B598499848994C8F
:10B2A000994F9A4E9A4DFFF74FFD26F0ADFF994901
:10B2B0000346934863613B70FFF746FD26F0A4FF09
:10B2C000954903468E48A3653370FFF73DFD26F090
:10B2D0009BFF636DA06258202B70FFF71BF88F490E
:10B2E0008748FFF731FD26F08FFF8D4903468448DC
:10B2F0003B70A361FFF728FD26F086FF89490346CE
:10B300007F483370E361FFF71FFD26F07DFF86491C
:10B3100003467B482B702362FFF716FD26F074FF6F
:10B32000824A606203464C201370FEF7F3FF00234D
:10B330004FF4F0727E497248FFF7AEF826F064FFD2
:10B34000002394227B4920606D48FFF7A5F826F082
:10B350005BFF0023A422784960606948FFF79CF8EE
:10B3600026F052FF00236C227449A0606448FFF766
:10B3700093F826F049FF00234FF4BC727049E06057
:10B380005F48FFF789F826F03FFF00234FF4227251
:10B390006C4920615A48FFF77FF826F035FF0023FB
:10B3A0004FF4D8726849A0625548FFF775F826F047
:10B3B0002BFF00234FF4E4726449E0625048FFF72A
:10B3C0006BF826F021FF00234FF4EE7260492063F2
:10B3D0004B48FFF761F826F017FF00234FF4217266
:10B3E0005C4960634648FFF757F826F00DFF0123DC
:10B3F000A0634FF4C27258494148FFF74DF801234A
:10B40000E0654FF4237255493D48FFF745F80123A5
:10B4100020668C2252493A48FFF73EF801236066C5
:10B42000F42250493648FFF737F80123A0664FF45D
:10B4300080724D493248FFF72FF84C49E0660023EF
:10B440004FF432722E48FFF727F8494926F094FE50
:10B45000002842D04FF0FF33236446492848002398
:10B460004FF43372FFF718F8414926F085FE0028A3
:10B470003CD04FF0FF3363643F49214800234FF431
:10B480003472FFF709F83A4926F076FE58B34FF0C8
:10B49000FF33A36439491A4800234FF43572FEF78D
:10B4A000FBFF334926F068FED0B14FF0FF33E36471
:10B4B0003349134800234FF43672FEF7EDFF2C4951
:10B4C00026F05AFEA8B9012323652E4B0D481968B2
:10B4D0007822BDE8F84021F07FBB01232364BCE75C
:10B4E0000123E364E4E70123A364D3E70123636456
:10B4F000C2E74FF0FF332365E7E700BFF8750300AD
:10B5000010760300BC94FF1F1C98FF1FC49AFF1FF6
:10B510005494FF1F1C760300247603003476030046
:10B52000487603005C76030070760300C497FF1F23
:10B530004475030084760300907603009C76030034
:10B54000A876030060750300B4760300BC760300A0
:10B55000C4760300D0760300DC760300F4760300A3
:10B56000087703001C77030030770300447703005B
:10B5700000004040587703006477030070770300B1
:10B58000807703005C87FF1F2DE9F84FA84CA94E78
:10B59000A94FDFF814B3DFF814A3DFF81483DFF842
:10B5A0001493E06A2268236CB56DA4498BF80000FF
:10B5B00038468AF8002088F8003089F80050FFF7F4
:10B5C000C3FB26F021FE9E4D9E49E06203463846AD
:10B5D00073618BF800306B64FFF7B6FB26F014FE46
:10B5E00099492060034638462B6073658AF800301D
:10B5F000FFF7AAFB26F02EFE944903469448B36554
:10B600006B61AB6289F80030FFF79EFB26F0FCFD12
:10B6100003461420236488F80030FEF77BFE0023E5
:10B620004FF460728B493846FEF736FF26F0ECFD8A
:10B63000014600234FF46A72616029633160384625
:10B640008549FEF729FF26F0DFFD616BA060A86544
:10B65000B06294F83000A26BE36B8BF800008AF8BC
:10B66000001038467D4989F8002088F80030FFF73F
:10B670006BFB26F0C9FD7A498BF80000034638467B
:10B680002363AB64B361FFF75FFB26F0BDFD754933
:10B690008AF80000034638466363EB64F361FFF702
:10B6A00053FB26F0B1FD704989F800000346384687
:10B6B000A3632B653362FFF747FB814626F0A4FDA9
:10B6C00003466B654846E363736226F0C3FD88F862
:10B6D00000003020FEF71EFE00234FF4797263490C
:10B6E0003846FEF7D9FE26F08FFD002386464FF43C
:10B6F0007C725F49C4F80CE03846C5F834E0C6F8FF
:10B7000004E0FEF7C9FE26F07FFD002386464FF4D5
:10B7100070725849C4F810E03846C5F85CE0C6F8C5
:10B720002CE0FEF7B9FE26F06FFD002386464FF4AD
:10B7300075725149C4F814E03846C5F838E0C6F8C7
:10B7400008E0FEF7A9FE26F05FFD002386464FF4D1
:10B7500047724A49C4F818E03846C5F860E0C6F8B0
:10B7600030E0FEF799FE26F04FFD002386464FF4A9
:10B7700048724349C4F81CE03846C5F83CE0C6F8B6
:10B780000CE0FEF789FE26F03FFD002386464FF4CD
:10B7900071723C49C4F820E03846C5F864E0C6F848
:10B7A00034E0FEF779FE26F02FFD002386464FF4A5
:10B7B00074723549C4F824E03846C5F840E0C6F84C
:10B7C00010E0FEF769FE26F01FFD002386460422E6
:10B7D0002E49C4F828E03846C5F868E0C6F838E0D5
:10B7E000FEF75AFE26F010FD294A2A495067012328
:10B7F00018223846FEF750FE274B254A1968106775
:10B800001046782221F0E8F9244B204619684C2292
:10B8100021F0E2F9224B30461968602221F0DCF970
:10B82000204B284619686C22BDE8F84F21F0D4B9A6
:10B83000CC97FF1F5C96FF1F90770300F8750300FD
:10B84000E898FF1F1C76030098770300A877030091
:10B8500024820300447503006075030034760300FE
:10B86000487603005C76030070760300847603005C
:10B87000B476030090760300BC7603009C76030048
:10B88000C4760300A8760300D0760300B4770300E3
:10B89000E095FF1FCC7703008C87FF1F7087FF1F89
:10B8A0009887FF1F8487FF1F1C98FF1FC49AFF1FE4
:10B8B000C497FF1F5494FF1F2DE9F843944C954DF6
:10B8C000DFF8D092944FDFF8D082944EA06AE36BF9
:10B8D000626C934989F800003B70284694F8403028
:10B8E00088F800203370FFF72FFA26F08DFC8D4981
:10B8F000A0620346284689F80030FFF725FA26F0B3
:10B9000083FC894960640346284688F80030FFF7C5
:10B910001BFA26F079FC8549E063034628463B7014
:10B92000FFF712FA26F070FC03466420236433709C
:10B93000FEF7F0FC0023F0227D492846FEF7ACFD1F
:10B9400026F062FC0123A0644FF42E722846794948
:10B95000FEF7A2FD0023E0664FF44F7276492846B9
:10B96000FEF79AFD26F050FC002320604FF4507241
:10B9700072492846FEF790FD26F046FC236B88F8B6
:10B98000003094F83430E26A60616D493B702846BB
:10B9900094F8383089F800203370FFF7D5F926F095
:10B9A00033FC684989F8000003462846E362FFF744
:10B9B000CBF926F029FC644988F8000003462846A4
:10B9C0002363FFF7C1F926F01FFC60493870034676
:10B9D00028466363FFF7B8F926F016FC03463420C7
:10B9E0003370A363FEF796FC00234FF45C72584952
:10B9F0002846FEF751FD26F007FC002360604FF457
:10BA00006D7254492846FEF747FD26F0FDFB0123E1
:10BA1000A0614FF48A7228464F49FEF73DFD01238D
:10BA2000E0654FF4927228464C49FEF735FD00233D
:10BA3000E0644FF45B724A492846FEF72DFD26F07C
:10BA4000E3FB0023A0604FF4597246492846FEF7F5
:10BA500023FD26F0D9FB0123E0614FF48E722846C6
:10BA60004149FEF719FD01232066E02228463F499F
:10BA7000FEF712FD002320654FF44E723C49284624
:10BA8000FEF70AFD26F0C0FB0023E0604FF44D7284
:10BA900038492846FEF700FD26F0B6FB0123206258
:10BAA0004FF4027228463449FEF7F6FC0123606623
:10BAB0004FF4047228463149FEF7EEFC002360651E
:10BAC0004FF4E2722E492846FEF7E6FC26F09CFB76
:10BAD00000232061D0222B492846FEF7DDFC26F00A
:10BAE00093FB01236062442228462749FEF7D4FCD9
:10BAF0000123A0663C2228462449FEF7CDFC244BB6
:10BB0000A065196820467022BDE8F84321F064B8AA
:10BB1000109AFF1F4C8203005494FF1FC497FF1F0D
:10BB2000F87503001C760300E0770300E877030054
:10BB300098770300F07703004475030060750300F5
:10BB400034760300487603005C76030070760300C9
:10BB500084760300B47603000478030018780300A9
:10BB600090760300BC7603002C7803004078030035
:10BB70009C760300C47603005478030068780300C1
:10BB8000A8760300D07603007C7803009078030049
:10BB90009087FF1F1C98FF1FC49AFF1F2DE9F047D5
:10BBA0006E4C6F4DDFF81492DFF81482E368A169E0
:10BBB0006C4F6D4E626A89F8003088F80010236B74
:10BBC0006A493A7028463370FFF7BEF826F042FB08
:10BBD0006749DFF8F0A1C3B2284689F80030E36076
:10BBE000FFF7B2F826F036FB6249C3B2284688F860
:10BBF0000030A361FFF7A8F826F02CFB5E49C3B222
:10BC000028463B706362FFF79FF826F023FBC3B220
:10BC10004FF4AE7033702363FEF77CFB00234FF4C8
:10BC2000727256492846FEF737FC26F013FB0023B4
:10BC300060604FF4777252492846FEF72DFC26F0DB
:10BC400009FB0123A060A82228464E49FEF724FCE8
:10BC5000012360634FF4C67228464B49FEF71CFC73
:10BC6000002360644FF47A7248492846FEF714FCBA
:10BC700026F0CAFA002320614FF47D724449284619
:10BC8000FEF70AFC26F0C0FA012360614FF4AA72A5
:10BC900028464049FEF700FC0123A0634FF49E7242
:10BCA00028463D49FEF7F8FB0023A0644FF45E727E
:10BCB0003A492846FEF7F0FB26F0A6FA0023E06199
:10BCC0004FF45F7236492846FEF7E6FB26F09CFAF1
:10BCD000012320624FF4A67228463249FEF7DCFBAE
:10BCE000DAF80010E0635422204620F075FF284661
:10BCF00001234FF4FA722C49FEF7CEFB0023E064D7
:10BD0000D4222A492846FEF7C7FB26F07DFA0023F5
:10BD1000A0624FF4D27226492846FEF7BDFB26F0FA
:10BD200073FA0123E0620C2228462249FEF7B4FB95
:10BD3000DAF8001020645422204620F04DFF2846F7
:10BD400024221D490123FEF7A7FBDAF80010206525
:10BD500054222046BDE8F04720F03EBF5894FF1F14
:10BD6000188203005494FF1FC497FF1F347603000A
:10BD7000487603005C760300707603008476030047
:10BD8000B4760300A4780300B07803009076030033
:10BD9000BC760300BC780300C87803009C760300DF
:10BDA000C4760300D4780300E4780300A876030087
:10BDB000D0760300F4780300047903001C98FF1F79
:10BDC000C49AFF1F2487FF1FF8B52F4D2F49304C11
:10BDD000304E314F2846FEF7B7FF26F03BFA2F4A88
:10BDE0002F49C3B22F4813706362FEF7ADFF26F0F0
:10BDF00031FA2D4A2D49C3B22D48A3601370FEF7C6
:10BE0000A3FF26F027FA2B4A2B49C3B22B48137005
:10BE1000F365FEF799FF26F01DFA294AC3B24FF4E5
:10BE2000DA7013703B60FEF775FA284601234FF471
:10BE300096722449FEF730FB0123E0624FF41F7233
:10BE400028462149FEF728FB002320624FF43D726B
:10BE50001E492846FEF720FB26F0D6F91C4BE06170
:10BE600019683846542220F0B7FE1A4B304619683C
:10BE7000602220F0B1FE184B204619686C22BDE804
:10BE8000F84020F0A9BE00BF4082030014790300EF
:10BE9000E898FF1F5C96FF1F5894FF1F1C98FF1F18
:10BEA0002879030080740300C49AFF1F34790300CB
:10BEB000D47403005494FF1F1C76030018820300FF
:10BEC000C497FF1F9C740300707403008C740300FC
:10BED0002487FF1F9887FF1F8487FF1F2DE9F04FDE
:10BEE000D74BD84DD84CDFF808A4DFF80894D3F826
:10BEF000D8306869D54ED64F6A68D6498AF80000AE
:10BF000085B0204603932B7889F800309DF80C30DB
:10BF100032703B70FEF718FF26F076F9CE498AF8AA
:10BF20000000034620466B61FEF70EFF26F06CF919
:10BF30002B686860C94989F800302046FEF704FF85
:10BF400026F062F9C649DFF8B083DFF8B0A30346F4
:10BF5000C44833706B60FEF7F7FE26F055F9B84A17
:10BF6000C14E034668203B70C2F8D830FEF7D2F9C4
:10BF700000234FF46272BD49BD4F2046FEF78CFA94
:10BF800026F042F90023A8604FF46C72B9492046AC
:10BF9000FEF782FA26F038F9002328629C22B6497F
:10BFA0002046FEF779FA26F02FF901232863B42200
:10BFB0002046B249FEF770FA0023E8622C22B0490D
:10BFC0002046FEF769FA26F01FF900236862202256
:10BFD000AC492046FEF760FA26F016F90023E86027
:10BFE0004FF40C72A8492046FEF756FA26F00CF9D9
:10BFF0000023A8624FF4FE72A4492046FEF74CFAD3
:10C0000026F002F900232861C022A1492046FEF74C
:10C0100043FA26F0F9F80023C8F800004FF40F7235
:10C020009C492046FEF738FA26F0EEF801234FF43B
:10C03000B072C8F8040098492046FEF72DFA012195
:10C040008146F5F799FC50460C2122F027FE484620
:10C0500025F054FA4FF0020902460B46CDF8009045
:10C06000304623F009FA304623F0A8F91B218B480B
:10C0700022F014FE00230A22D8F80810304623F0DC
:10C08000B1F9304623F09AF91B21854822F006FECB
:10C09000D8F80C0025F032FACDF8009002460B4695
:10C0A000304623F0E9F9304623F088F90023A02236
:10C0B0007C492046FEF7F0F926F0A6F80023386008
:10C0C0004FF4317278492046FEF7E6F926F09CF8E5
:10C0D00001234FF4B472786074492046FEF7DCF90E
:10C0E00049468346F5F748FC50460C2122F0D6FD20
:10C0F000584625F003FACDF8009002460B4630462C
:10C1000023F0BAF9304623F059F91B216848DFF8CB
:10C11000F0B1DFF8F0A122F0C1FD00230A22B968D6
:10C12000304623F05FF9304623F048F91B2161487F
:10C1300022F0B4FDF86825F0E1F9CDF80090024650
:10C140000B46304623F098F9304623F037F90023A8
:10C15000982259492046FEF79FF926F055F8574A8C
:10C160005749106000234FF414722046FEF794F9EB
:10C1700026F04AF8514A5349506001234FF4117296
:10C180002046FEF789F90321F5F7F6FB00234FF46B
:10C19000D6724D492046FEF77FF926F035F8002388
:10C1A000CBF800004FF4137248492046FEF774F9AB
:10C1B00026F02AF80123CBF804004FF42872204619
:10C1C0004349FEF769F90421F5F7D6FB00234FF444
:10C1D000DC7240492046FEF75FF926F015F800238F
:10C1E000CAF800004FF406723B492046FEF754F9A6
:10C1F00026F00AF80123CAF804004FF42A722046F8
:10C200003649FEF749F90521F5F7B6FB344B2846C8
:10C210001968342220F0E0FC324B404619681022A5
:10C2200020F0DAFC304B38461968102220F0D4FC9C
:10C230002E4B22481968102220F0CEFC64E000BF8B
:10C24000BC96FF1FB498FF1F0C8203005494FF1F7D
:10C25000C497FF1FF87503001C7603003C790300A8
:10C2600044790300547903006488FF1F4475030078
:10C27000EC92FF1F60750300B4770300CC770300D6
:10C28000C47603009C760300D0760300A8760300F2
:10C29000607903007879030088790300A0790300AE
:10C2A000BC790300D8790300F0790300007A030019
:10C2B000087A0300247A0300407A03000C93FF1FDE
:10C2C000587A0300687A0300707A0300887A0300C2
:10C2D000987A0300A07A0300B87A0300C87A0300B2
:10C2E0006487FF1F4087FF1F4487FF1F4887FF1F8A
:10C2F0001C98FF1FC49AFF1FB49AFF1F9079030078
:10C30000C89AFF1FD89AFF1F0A4B58461968102277
:10C3100020F062FC084B50461968102220F05CFCAB
:10C32000064B07481968E42205B0BDE8F04F20F03D
:10C3300053BC00BF4C87FF1F5087FF1FD895FF1FBE
:10C34000BC96FF1F2DE9F04F954C964FDFF8C49235
:10C35000DFF8C4826369A16D934E944DD7F8DC2059
:10C3600089F800308BB0D7F8E03088F8001090489A
:10C3700090492B703270FEF7E7FC824625F044FFAF
:10C380006061504625F066FF8B4989F800008848B7
:10C39000DFF830A2FEF7D8FC834625F035FFA06514
:10C3A000584625F057FF854988F800008448FEF775
:10C3B000CBFC834625F028FFC7F8DC00584625F063
:10C3C00049FFDAF80030059305993070DAF800304B
:10C3D0000493049B7B4A5B1A0E2BF7D97A49784861
:10C3E0000192FEF7B1FC834625F00EFFC7F8E0008E
:10C3F000584625F02FFF28700020FDF78BFF019A8B
:10C4000013680393039ADAF800300293029B9B1A95
:10C410000E2BF8D906A86D4923F070FA002106A862
:10C42000F5F778FC06A823F029FAD7F8E00025F004
:10C43000B7FC0021F5F77AFF654B06A8196823F0D1
:10C440005DFA06A80021F5F765FC06A823F016FAA8
:10C4500000234FF45A725F495548FEF71DF825F046
:10C46000D3FE002320604FF464725B495048FEF70E
:10C4700013F825F0C9FE236AE269A769A06257494B
:10C4800033704B4894F8243088F800202B7089F8DA
:10C490000070FEF759FC25F0B7FE514903464448A9
:10C4A000A36189F80030FEF74FFC25F0ADFE4D4941
:10C4B00003463F48E36188F80030FEF745FC25F06D
:10C4C000A3FE494903463A4823623370FEF73CFC19
:10C4D00025F09AFE0346082063622B70FDF71AFFD1
:10C4E00000234FF46E7241493148FDF7D5FF25F026
:10C4F0008BFE002360604FF473723D492C48FDF7BA
:10C50000CBFF25F081FE0023E0624FF478723949B9
:10C510002748FDF7C1FF25F077FE0023A0604FF408
:10C520007B7235492248FDF7B7FF25F06DFE0023E9
:10C5300020634FF47E7231491D48FDF7ADFF25F0B1
:10C5400063FE0023E0604FF47F722D491848FDF729
:10C55000A3FF25F059FE002360634FF4657229495B
:10C560001348FDF799FF25F04FFE002320614FF49B
:10C57000667225490E48FDF78FFF25F045FE234BD7
:10C58000A06319680648782220F026FB204B054856
:10C590001968E42220F020FB0BB0BDE8F08F00BF4B
:10C5A000E095FF1FBC96FF1F5494FF1FC497FF1F09
:10C5B000D07A0300F87503001C760300D87A0300D4
:10C5C000547903007CA0FF1FE47A0300F07A030093
:10C5D000A487FF1F447503006075030034760300D1
:10C5E000487603005C7603007076030084760300CF
:10C5F000B476030090760300BC7603009C760300BB
:10C60000C4760300A8760300D07603008C87FF1F52
:10C61000D895FF1F1C98FF1FC49AFF1F2DE9F043F8
:10C62000C649C748C74C87B0FEF78EFB4FF07E5116
:10C63000054625F0BFFD002800F02782012384F87D
:10C64000A030284625F006FEBF4FC0493870BC48D0
:10C65000FEF77AFB4FF07E51054625F0ABFD002832
:10C6600000F01082012384F89C30284625F0F2FD6A
:10C67000B74DB8492870B248DFF86483DFF8C49238
:10C68000FEF762FB25F0E6FDB3490346AC4863655F
:10C6900088F80030FEF758FB4FF07E51064625F033
:10C6A00089FD002800F0EB81012389F89D30304698
:10C6B00025F0D0FDA94E30704FF4E670FDF72AFE4C
:10C6C000A7499F48FEF740FB4FF07E5125F072FDD1
:10C6D000002800F0D081012084F8C8000346A14959
:10C6E00097483370FEF730FB4FF07E5125F062FD26
:10C6F000002800F0BC81012084F89E000346B02091
:10C700002B70FDF707FE98498D48FEF71DFB4FF093
:10C710007E51814625F04EFD002800F0A5810123C1
:10C7200084F89F30484625F095FD90493070904838
:10C73000FEF70AFB25F068FD8E4903468048C4F8E1
:10C74000D43088F80030FEF7FFFA25F05DFD8A4905
:10C7500003467B4863632B70FEF7F6FA25F054FD21
:10C7600003464FF4D070C4F8CC303B70FDF7D2FDD7
:10C7700082497348FEF7E8FA25F06CFD8049307075
:10C780006F48FEF7E1FA25F065FD7E4988F8000064
:10C790006B48FEF7D9FA25F05DFD7B4928706848A3
:10C7A000FEF7D2FA25F056FD3870FC20FDF7B2FDF9
:10C7B00000234FF4847275496148FDF76DFE002334
:10C7C000C82273495E48FDF767FE25F01DFD002372
:10C7D0002060F4226F495A48FDF75EFE25F014FDF3
:10C7E000012360604FF486726B495548FDF754FE93
:10C7F0000023A060C42269495148FDF74DFE25F091
:10C8000003FD0023E0604FF4EA7265494C48FDF7F0
:10C8100043FE25F0F9FC4FF40072012320616149C9
:10C820004748FDF739FE6049606102A823F066F8C9
:10C8300002A80021F5F76EFA02A823F01FF85B4B5F
:10C8400002A8196823F05AF802A80021F5F762FA45
:10C85000002502A823F012F82B464FF40D7254491C
:10C860003748C4F8B850FDF717FE25F0CDFC2B462D
:10C8700020624FF4F2724F493148FDF70DFE25F06A
:10C88000C3FC012360624FF4F4724B492C48FDF75E
:10C8900003FE2B46A0624FF40E7248492848FDF76C
:10C8A000FBFD25F0B1FC2B46C4F8BC00CC2244496A
:10C8B0002348FDF7F1FD25F0A7FC0123C4F8C000D3
:10C8C000D82240491E48FDF7E7FD2B46C4F8C400B6
:10C8D0005C223D491A48FDF7DFFD25F095FC2B460B
:10C8E000A0634FF4087239491548FDF7D5FD25F0CE
:10C8F0008BFC0123E0634FF4097235491048FDF7C2
:10C90000CBFD012320644FF4CC7232490C48FDF773
:10C91000C3FD012360644FF42C722F490848FDF7D2
:10C92000BBFD2B46A06460222C490548FDF7B4FDF1
:10C9300025F06AFC2B46A06554E000BF0C7B030089
:10C9400054790300BC96FF1FC497FF1F187B030098
:10C950005494FF1F2C7B0300407B03001C98FF1F97
:10C960004C7B03005C7B0300687B0300747B03004B
:10C970007C7B0300847B0300987B0300AC7B03007B
:10C98000C07B0300D47B0300E87B0300FC7B030037
:10C99000107C0300247C0300387C03004C7C0300E3
:10C9A0005C7C03006C7C0300807C0300A487FF1F79
:10C9B0008C7C03009C7C0300AC7C0300C07C0300E7
:10C9C000D07C0300E47C0300F87C0300087D0300B6
:10C9D000187D0300287D03003C7D0300487D030093
:10C9E000C49AFF1F4FF4CA7229492A48FDF754FD23
:10C9F00025F00AFC01234FF4BE72E0652649254864
:10CA0000FDF74AFD1F212066244822F047F9206ED9
:10CA100024F074FD022502460B460095204822F0C2
:10CA20002BFD1F4822F0CAFC3F211E4822F036F998
:10CA30001B4822F0C3FC01234FF416721A49154813
:10CA4000FDF72AFD012360664FF42672174911484D
:10CA5000FDF722FD164BA06619681648E42220F067
:10CA6000BBF807B0BDE8F08384F89F005AE684F86D
:10CA70009E00034643E684F8C80003462FE689F883
:10CA80009D0014E684F89C00EFE584F8A000D8E54A
:10CA9000587D030054790300687D0300787D03000E
:10CAA0006488FF1F987D0300D87D0300EC7D0300A0
:10CAB000D895FF1FBC96FF1F2DE9F04F8049814894
:10CAC000814D824EDFF85892DFF85882804F814CBA
:10CAD00091B0FEF739F925F097FB7F490346794875
:10CAE000EB643370FEF730F925F08EFB7B4903468B
:10CAF00074482B6589F80030FEF726F925F084FB91
:10CB0000774903466F48C5F8D03088F80030FEF703
:10CB10001BF925F079FB03464FF41070C5F8B430CB
:10CB20003B70FDF7F7FB6F496648FEF70DF9236888
:10CB30000F930F99824623680E930E9B654A5B1AEA
:10CB4000632BF8D95046039225F05EFB039AA86147
:10CB500013680D930D9923680C930C9B5D4A5B1A27
:10CB6000632BF8D95046039225F074FB5E49307070
:10CB70005448FEF7E9F825F047FB5C490346514865
:10CB8000EB6189F80030FEF7DFF825F03DFB5849EE
:10CB900003464C48EB6288F80030FEF7D5F825F0E4
:10CBA00033FB03464FF4D4702B633B70FDF7B2FBAD
:10CBB000039A13680B930B9A23680A930A9BDFF876
:10CBC00014B19B1A632BF7D94A493E48FEF7BCF8CB
:10CBD00038218246484822F061F8504624F08EFC05
:10CBE0004FF0020E0B460246CDF800E0434822F01B
:10CBF00043FC424822F0E2FBDBF80030099309993C
:10CC000023680893089B334A5B1A632BF8D9504674
:10CC1000039225F0F9FA039AE866136807930799D7
:10CC200023680693069B2B4A5B1A632BF8D913687B
:10CC30000593059A307023680493049B9B1A632B19
:10CC4000F9D92F212E482F4C22F028F80A22002350
:10CC500031782A4822F0C6FB284822F0AFFB2A4947
:10CC60001848FEF771F825F0CFFA284903462848FE
:10CC70002B6789F80030FEF767F825F0C5FA2549DB
:10CC80000346234888F80030A361FEF75DF825F0DD
:10CC9000BBFA03464FF4B870E3613B70FDF73AFB13
:10CCA0001D4B09481968E4221FF096FF1B4B2046D4
:10CCB000196834221FF090FF11B0BDE8F08F00BF5B
:10CCC000F87D03007C7B0300BC96FF1F1C98FF1FB0
:10CCD000C497FF1F7CA0FF1F007E0300087E030097
:10CCE000107E03001C7E0300247E03002C7E0300C4
:10CCF000347E03003C7E0300447E03006488FF1FF3
:10CD0000807E0300B498FF1FB07E03005C760300B2
:10CD10000C82030070760300D895FF1F6487FF1F05
:10CD2000C49AFF1F5494FF1FF0B50023A3B001A8BD
:10CD30001A46AE491FF02CFB0C9C002C33D0236804
:10CD4000AB4A1B6B934228D1236D002B00F0D2819C
:10CD50002368A84FDB6ABB4240F06582A06D18B122
:10CD600025F0BCFC0023A365236D002B00F07E8220
:10CD700004F118001EF072F90C9D6C68013C6C60A7
:10CD8000002C00F0D0819C4E00230C939DF81E30A7
:10CD9000012B0DD144F202230FE02046984710B139
:10CDA0000C9C002CD4D19DF81E30934E012BF1D059
:10CDB000022B40F2022318BF00230EA801AA8F49BC
:10CDC0001EF036FA209B002B00F0B8805C2022F089
:10CDD000B3FA04468A4B9DF83C00109A89492360B7
:10CDE00000259DF844302073A160226112A92375AB
:10CDF000656004F118001EF003F96368824AA565B6
:10CE00000133636012A8A2600E961EF027F96368D2
:10CE10000C9D01336360002D00F071816F68013F4C
:10CE20006F60002F00F0FC800C94002C00F09380C9
:10CE300063685D1E6560002D00F029810C9C002C4C
:10CE400000F0898023686A4D1B6BAB4240F059812A
:10CE5000236D002B00F0628100238DF81F302368C2
:10CE60001B6BAB4240F09581236D002B00F09B8142
:10CE70002368604FDB6ABB4240F0D881A06D18B1D7
:10CE800025F02CFC0023A365236D002B00F0F88116
:10CE900004F118001EF0E2F80C9D6C68013C6C6017
:10CEA000002C00F0858100230C93FFF7B7FBFDF702
:10CEB000BDFEFFF701FEFFF745FAFEF7EDF9FFF7BC
:10CEC0000DF8FEF76BFEFEF75FFBFDF739FEFDF791
:10CED0005DFEFDF703FEFEF777FFFEF7EDFC4B4925
:10CEE0004B4C0EA822F00AFD00210EA8F4F712FF09
:10CEF0000EA822F0C3FC21680EA822F0FFFC00213E
:10CF00000EA8F4F707FF0EA822F0B8FC41490EA8BE
:10CF100022F0F4FC00210EA8F4F7FCFE0EA822F08B
:10CF2000ADFC21680EA822F0E9FC00210EA8F4F760
:10CF3000F1FE0EA822F0A2FC37493DE0219C002C16
:10CF40007FF444AF12A80E961EF088F80C9D002DB9
:10CF50007FF464AF0C95012330498DF81F300EA883
:10CF600022F0CCFC2A4C00210EA8F4F7D3FE0EA828
:10CF700022F084FC21680EA822F0C0FC00210EA83B
:10CF8000F4F7C8FE0EA822F079FC22490EA822F080
:10CF9000B5FC00210EA8F4F7BDFE0EA822F06EFC31
:10CFA00021680EA822F0AAFC00210EA8F4F7B2FE18
:10CFB0000EA822F063FC15490EA822F09FFC002168
:10CFC0000EA8F4F7A7FE0EA822F058FC21680EA8C0
:10CFD00022F094FC00210EA8F4F79CFE0EA822F08B
:10CFE0004DFC01A81FF000FA23B0F0BD2093FF1FF5
:10CFF000750400006D05000094620300749BFF1F20
:10D000000863030070620300B862030044850300F4
:10D01000A487FF1FCC890300B87E03001C740300A3
:10D020002B68A34ADB6A934240F0F480A86D10B1EC
:10D0300025F054FBAF652B6D002B00F00D8105F141
:10D0400018001EF00BF80C9D002D3FF4EDAE2B6880
:10D05000984A5B68934240F0E380A86D964B2B6042
:10D0600018B125F03BFB0023AB652B6D05F11807CC
:10D07000002B00F0F68038461DF0F0FFAE60384619
:10D080001DF0ECFF28465C2122F05AF9CCE623681B
:10D09000874ADB6A934240F0C080A06D10B125F052
:10D0A0001DFBA565236D002B00F0C38004F1180063
:10D0B0001DF0D4FF23687F4A5B68934240F0C9802B
:10D0C000A06D7D4B236018B125F008FB0023A365FC
:10D0D000236D04F11805002B00F0CD8028461DF0CB
:10D0E000BDFFA66028461DF0B9FF20465C2122F056
:10D0F00027F9A3E6636D002B7FF42AAE53E60C9468
:10D1000097E62046984700283FF425AF0C9C002363
:10D110008DF81F30002C3FF4C8AEA0E6636D002BE5
:10D120007FF49AAE17E72B68DB6ABB4240F0AD8014
:10D13000A86D10B125F0D2FAAC652B6D002B00F074
:10D14000AD8005F118001DF089FF0C9C002C3FF408
:10D150001AAE2368574A5B68934240F09C80A06DEA
:10D16000554B236018B125F0B9FA0023A365236D50
:10D1700004F11805002B68D028461DF06FFF4F4EB4
:10D18000A66028461DF06AFF20465C2122F0D8F8F0
:10D19000FAE52046984700283FF487AE0C9C002C07
:10D1A0003FF483AE64E6636D002B7FF461AE7CE6F2
:10D1B0002B68DB6ABB426BD1A86D10B125F08EFAEB
:10D1C000AC652B6D002B3CD005F118001DF046FF1F
:10D1D0000C9C002C3FF467AE2368364A5B68934290
:10D1E0002CD1A06D344B236018B125F077FA0023C1
:10D1F000A365236D04F11805002B54D028461DF0BB
:10D200002DFFA66028461DF029FF20465C2122F054
:10D2100097F848E62846984715E72046984749E793
:10D220002846984700E620469847A5E520469847B7
:10D2300032E6636D002B7FF439AF3BE72046984719
:10D2400031E66B6D002BBFD1C2E7636D002B93D12C
:10D2500095E720469847F1E56B6D002B7FF4EFAE24
:10D26000F1E66B6D002B7FF406AF07E7636D002BD3
:10D270007FF47EAD80E5636D002B7FF42FAF30E748
:10D28000636D002B7FF404AE06E6284698475CE702
:10D29000284698479CE72046984774E56B6D002B1D
:10D2A0007FF44FAF51E7636D002BA7D1A9E700BF13
:10D2B0006D050000590D000008630300946203002F
:10D2C00070B5D8B004461D4930A822F017FB1B49A1
:10D2D00034A822F013FB1A4938A822F00FFB194991
:10D2E0003CA822F00BFB184940A822F007FB174985
:10D2F00044A822F003FB164948A822F0FFFA15497A
:10D300004CA822F0FBFA50A8134922F0F7FA0122A8
:10D31000124B94421A7000F099810B2C00F07C8320
:10D32000023C082C20D8DFE814F01B005D016201EC
:10D330001F0067016C01710176015801AC94030074
:10D34000C47E0300CC890300D47E0300EC87030075
:10D35000E47E0300D8870300406403005594FF1F58
:10D36000AF4930A822F036FB54AD38A934A822F0DA
:10D3700021FB34A9284622F0D5FA00212846F4F7EB
:10D38000C9FC284622F07AFA50A9284622F0CAFAA7
:10D39000A44C28460021F4F7BDFC284622F06EFA82
:10D3A00023682D932D9A23682C932C9B9D4E9B1ABA
:10D3B0000E2BF8D930A9284622F0B4FA3CA9284609
:10D3C00022F068FB014634A822F0F4FA284622F045
:10D3D00055FA3CA9944821F0CBFF934821F0EEFF89
:10D3E0003CA9284622F09EFA00212846F4F792FC38
:10D3F000284622F043FA50A9284622F093FA002149
:10D400002846F4F787FC284622F038FA33682B9335
:10D410002B9A23682A932A9B824E9B1A0E2BF8D9AB
:10D4200040A934A822F0C6FA40A97F4821F0A0FF05
:10D430007D4821F0C3FF40A9284622F073FA00215D
:10D440002846F4F767FC284622F018FA50A9284627
:10D4500022F068FA00212846F4F75CFC284622F006
:10D460000DFA33682993299A23682893289B6D4ED7
:10D470009B1A092BF8D944A934A822F09BFA44A995
:10D48000694821F075FF684821F098FF44A92846B3
:10D4900022F048FA00212846F4F73CFC284622F006
:10D4A000EDF950A9284622F03DFA00212846F4F76C
:10D4B00031FC284622F0E2F933682793279A236843
:10D4C0002693269B574E9B1A0E2BF8D948A934A8B1
:10D4D00022F070FA34A9544821F04AFF524821F052
:10D4E0006DFF48A9284622F01DFA00212846F4F7CE
:10D4F00011FC284622F0C2F950A9284622F012FA5F
:10D5000000212846F4F706FC284622F0B7F93368D4
:10D510002593259A23682493249B9B1A0E2BF9D9D3
:10D520004CA934A822F046FA34A93F4821F020FF44
:10D530003D4821F043FF4CA9284622F0F3F9002191
:10D540002846F4F7E7FB284622F098F950A9284628
:10D5500022F0E8F900212846F4F7DCFB284622F007
:10D560008DF923682F932F9A23682E932E9B9B1A55
:10D57000092BF9D92D49284622F0C0F90021284667
:10D58000F4F7C8FB284622F079F950A9284622F082
:10D59000C9F900212846F4F7BDFB284622F06EF9B0
:10D5A00050A822F06BF94CA822F068F948A822F0A4
:10D5B00065F944A822F062F940A822F05FF93CA87E
:10D5C00022F05CF938A822F059F934A822F056F973
:10D5D00030A822F053F958B070BD154930A822F098
:10D5E000F9F9C1E6134930A822F0F4F9BCE6124972
:10D5F00030A822F0EFF9B7E6104930A822F0EAF996
:10D60000B2E60F4930A822F0E5F9ADE60D4930A8A1
:10D6100022F0E0F9A8E60C4930A822F0DBF9A3E6F5
:10D62000548203007CA0FF1F6488FF1F5C820300FC
:10D630004882030008820300148203002082030052
:10D640002C820300348203003C82030054ADCE4997
:10D65000CE4C284622F052F900212846F4F75AFB16
:10D66000284622F00BF950A9284622F05BF92846FB
:10D670000021F4F74FFB284622F000F923681193AC
:10D68000119A23681093109BC04E9B1A092BF8D94E
:10D69000BF49284622F032F900212846F4F73AFB28
:10D6A000284622F0EBF850A9284622F03BF9002149
:10D6B0002846F4F72FFB284622F0E0F8B549284623
:10D6C00022F01CF900212846F4F724FB284622F01A
:10D6D000D5F850A9284622F025F900212846F4F76C
:10D6E00019FB284622F0CAF833680F930F9A236873
:10D6F0000E930E9BA54E9B1A092BF8D9A6492846D6
:10D7000022F0FCF800212846F4F704FB284622F01A
:10D71000B5F850A9284622F005F900212846F4F76B
:10D72000F9FA284622F0AAF89C49284622F0E6F8A1
:10D7300000212846F4F7EEFA284622F09FF850A977
:10D74000284622F0EFF800212846F4F7E3FA2846AD
:10D7500022F094F833680D930D9A23680C930C9B78
:10D760008A4E9B1A092BF8D98D49284622F0C6F813
:10D7700000212846F4F7CEFA284622F07FF850A977
:10D78000284622F0CFF800212846F4F7C3FA2846AD
:10D7900022F074F88349284622F0B0F80021284688
:10D7A000F4F7B8FA284622F069F850A9284622F082
:10D7B000B9F800212846F4F7ADFA284622F05EF8C1
:10D7C00033680B930B9A23680A930A9B6F4E9B1A3C
:10D7D000092BF8D97449284622F090F800212846F0
:10D7E000F4F798FA284622F049F850A9284622F082
:10D7F00099F800212846F4F78DFA284622F03EF8E1
:10D800006A49284622F07AF800212846F4F782FA7D
:10D81000284622F033F850A9284622F083F8002148
:10D820002846F4F777FA284622F028F83368099357
:10D83000099A23680893089B544E9B1A092BF8D920
:10D840005B49284622F05AF800212846F4F762FA8C
:10D85000284622F013F850A9284622F063F8002148
:10D860002846F4F757FA284622F008F85149284686
:10D8700022F044F800212846F4F74CFA284621F01B
:10D88000FDFF50A9284622F04DF800212846F4F764
:10D8900041FA284621F0F2FF33680793079A23687C
:10D8A0000693069B394E9B1A092BF8D94249284604
:10D8B00022F024F800212846F4F72CFA284621F01B
:10D8C000DDFF50A9284622F02DF800212846F4F764
:10D8D00021FA284621F0D2FF3849284622F00EF8D6
:10D8E00000212846F4F716FA284621F0C7FF50A970
:10D8F000284622F017F800212846F4F70BFA2846AC
:10D9000021F0BCFF33680593059A23680493049BB8
:10D910001E4E9B1A092BF8D92949284621F0EEFF03
:10D9200000212846F4F7F6F9284621F0A7FF50A970
:10D93000284621F0F7FF00212846F4F7EBF92846A6
:10D9400021F09CFF1F49284621F0D8FF00212846DE
:10D95000F4F7E0F9284621F091FF50A9284621F07C
:10D96000E1FF00212846F4F7D5F9284621F086FF8B
:10D9700033680393039A23680293029B034E9B1A16
:10D98000092BF8D920E000BFF47E03007CA0FF1F24
:10D990000C7F0300207F0300387F03004C7F0300CF
:10D9A000647F0300787F0300907F0300A47F03005F
:10D9B000BC7F0300D07F0300E87F0300FC7F0300EF
:10D9C00014800300288003001149284621F096FFA7
:10D9D00000212846F4F79EF9284621F04FFF50A970
:10D9E000284621F09FFF00212846F4F793F92846A6
:10D9F00021F044FF33680193019A23680093009B50
:10DA00009B1A092BF9D90349284621F077FF96E59F
:10DA1000408003005480030054ADCE49CE4C2846CC
:10DA200021F06CFF00212846F4F774F9284621F014
:10DA300025FF50A9284621F075FF28460021F4F75C
:10DA400069F9284621F01AFF23682393239A236853
:10DA50002293229BC04E9B1A092BF8D9BF49284616
:10DA600021F04CFF00212846F4F754F9284621F014
:10DA700005FF50A9284621F055FF00212846F4F75C
:10DA800049F9284621F0FAFEB549284621F036FF2B
:10DA900000212846F4F73EF9284621F0EFFE50A970
:10DAA000284621F03FFF00212846F4F733F92846A5
:10DAB00021F0E4FE33682193219A23682093209B70
:10DAC000A54E9B1A092BF8D9A649284621F016FF26
:10DAD00000212846F4F71EF9284621F0CFFE50A970
:10DAE000284621F01FFF00212846F4F713F92846A5
:10DAF00021F0C4FE9C49284621F000FF0021284661
:10DB0000F4F708F9284621F0B9FE50A9284621F07B
:10DB100009FF00212846F4F7FDF8284621F0AEFE63
:10DB200033681F931F9A23681E931E9B8A4E9B1A6D
:10DB3000092BF8D98D49284621F0E0FE002128461E
:10DB4000F4F7E8F8284621F099FE50A9284621F07C
:10DB5000E9FE00212846F4F7DDF8284621F08EFE84
:10DB60008349284621F0CAFE00212846F4F7D2F85E
:10DB7000284621F083FE50A9284621F0D3FE00213B
:10DB80002846F4F7C7F8284621F078FE33681D933D
:10DB90001D9A23681C931C9B6F4E9B1A092BF8D966
:10DBA0007449284621F0AAFE00212846F4F7B2F86D
:10DBB000284621F063FE50A9284621F0B3FE00213B
:10DBC0002846F4F7A7F8284621F058FE6A49284667
:10DBD00021F094FE00212846F4F79CF8284621F015
:10DBE0004DFE50A9284621F09DFE00212846F4F75D
:10DBF00091F8284621F042FE33681B931B9A236854
:10DC00001A931A9B544E9B1A092BF8D95B49284644
:10DC100021F074FE00212846F4F77CF8284621F014
:10DC20002DFE50A9284621F07DFE00212846F4F75C
:10DC300071F8284621F022FE5149284621F05EFE67
:10DC400000212846F4F766F8284621F017FE50A96F
:10DC5000284621F067FE00212846F4F75BF82846A5
:10DC600021F00CFE33681993199A23681893189BB6
:10DC7000394E9B1A092BF8D94249284621F03EFE1D
:10DC800000212846F4F746F8284621F0F7FD50A970
:10DC9000284621F047FE00212846F4F73BF82846A5
:10DCA00021F0ECFD3849284621F028FE00212846C5
:10DCB000F4F730F8284621F0E1FD50A9284621F07C
:10DCC00031FE00212846F4F725F8284621F0D6FD3C
:10DCD00033681793179A23681693169B1E4E9B1A48
:10DCE000092BF8D92949284621F008FE00212846A9
:10DCF000F4F710F8284621F0C1FD50A9284621F07C
:10DD000011FE00212846F4F705F8284621F0B6FD5B
:10DD10001F49284621F0F2FD00212846F3F7FAFFBB
:10DD2000284621F0ABFD50A9284621F0FBFD00213B
:10DD30002846F3F7EFFF284621F0A0FD336815933E
:10DD4000159A23681493149B034E9B1A092BF8D938
:10DD500020E000BF688003007CA0FF1F84800300D8
:10DD60009C800300B8800300D0800300EC80030097
:10DD700004810300208103003881030054810300E3
:10DD80006C8103008481030098810300B08103004B
:10DD9000C48103001249284621F0B0FD0021284625
:10DDA000F3F7B8FF284621F069FD50A9284621F075
:10DDB000B9FD00212846F3F7ADFF284621F05EFDAE
:10DDC00033681393139A23681293129B9B1A092B9F
:10DDD000F9D90449284621F091FDFFF7B0BB00BFF7
:10DDE000DC810300F081030030B5A9B004460D4684
:10DDF00008A87D4921F082FD7B490CA821F07EFD19
:10DE00007A4910A821F07AFD794914A821F076FD0D
:10DE1000784918A821F072FD77491CA821F06EFD01
:10DE200020A8764921F06AFD0122754B94421A70B0
:10DE300063D00B2C4AD0012D00F08980013545D1EB
:10DE400010A90CA821F0B6FD0CA96E4824AC21F055
:10DE50008FFA6C4821F0B2FA0CA9204621F062FD3D
:10DE600000212046F3F756FF204621F007FD20A9A8
:10DE7000204621F057FD00212046F3F74BFF2046B6
:10DE800021F0FCFC604A136805930599136804931C
:10DE9000049B5B1A092BF9D914A90CA821F08AFD5F
:10DEA0000CA9204621F03EFD00212046F3F732FF69
:10DEB000204621F0E3FC20A9204621F033FD204636
:10DEC0000021F3F727FF204621F0D8FC20A821F0FD
:10DED000D5FC1CA821F0D2FC18A821F0CFFC14A876
:10DEE00021F0CCFC10A821F0C9FC0CA821F0C6FC44
:10DEF00008A821F0C3FC29B030BD95424ED00135B1
:10DF0000E4D124AC4149204621F0F8FC0021204610
:10DF1000F3F700FF204621F0B1FC20A9204621F0B4
:10DF200001FD00212046F3F7F5FE204621F0A6FC76
:10DF3000354A13680193019913680093009B5B1A9B
:10DF4000092BF9D93249204621F0D8FCACE724ACA2
:10DF500018A90CA821F02EFD0CA9204621F0E2FC06
:10DF600000212046F3F7D6FE204621F087FC20A9A9
:10DF7000204621F0D7FC00212046F3F7CBFE2046B7
:10DF800021F07CFC204A13680793079913680693D5
:10DF9000069B5B1A092BF9D91CA97EE724AC1D4905
:10DFA000204621F0ABFC00212046F3F7B3FE2046CB
:10DFB00021F064FC20A9204621F0B4FC0021204679
:10DFC000F3F7A8FE204621F059FC0F4A136803938B
:10DFD000039913680293029B5B1A092BF9D90E4926
:10DFE000204621F08BFC5FE7AC940300D47E030055
:10DFF000EC870300E47E0300D8870300406403003D
:10E000006C9BFF1F6488FF1F7CA0FF1F207F030005
:10E01000387F03004C7F0300647F030090F890304A
:10E0200010B504461BB906E001201EF075FFA36879
:10E03000002BF9D110BDF2F735FBF8E738B583684E
:10E04000F3B1816D826F4B68D0F8AC40D21A82EA8E
:10E05000E273A3EBE273A34213DBD0F8B020934248
:10E0600017DA1A190025C2672346C0F8B0504A686B
:10E070000C6804FB0323CB60CA684B689A420BD040
:10E0800038BD00225C00C0F8B020C0F8AC20C467E6
:10E09000EDE7C26FD31AEAE704460C3021F0FAF834
:10E0A0000023206AA3601EF03BF9606ABDE8384097
:10E0B0001EF036B910B50446FFF7C0FFA3682BB1B8
:10E0C00001201EF029FFA368002BF9D110BD00BF6D
:10E0D000F8B5044600230D46606101211E4F1F4E16
:10E0E000A3608020E36084F82830E365236684F829
:10E0F0006430A36666602074E16627602846164691
:10E1000023F04EFE164923F0A3FE164923F0A0FE8D
:10E110004FF0745123F09CFE4FF07C5123F090FDA2
:10E1200024F072F8A061304623F03AFE0C4923F047
:10E130008FFE0C4923F08CFE4FF0745123F088FEC3
:10E140004FF07C5123F07CFD24F05EF82667E061FF
:10E1500065672046F8BD00BF706303006463030079
:10E16000BD3786354054094C38B590F86430114AB3
:10E170000260044600F10C0553B1284621F08AF8EC
:10E180000023206AA3601EF0CBF8606A1EF0C8F876
:10E19000094B6360284621F07DF80023A360206AC4
:10E1A0001EF0BEF8606A1EF0BBF8284621F072F837
:10E1B000204638BD706303006463030010B5034B51
:10E1C00003600446FFF7D0FF204610BDA86303009C
:10E1D00010B5054B03600446FFF7C6FF2046B82183
:10E1E00021F0AEF8204610BDA863030010B5034B24
:10E1F00003600446FFF7B8FF204610BD8C630300A0
:10E2000010B5054B03600446FFF7AEFF204694218E
:10E2100021F096F8204610BD8C63030010B504462B
:10E22000FFF7A2FF2046782121F08AF8204610BD92
:10E23000884231D02DE9F04700F1040841451646E7
:10E240008A46814617D0D9F80010D8F80000B047A8
:10E2500098B9D8F80050444601E023686360274627
:10E26000284654F8041DB0470028F6D13D6008F157
:10E270000408C245E7D1BDE8F087C9EB080293085E
:10E28000D8F8004005D0C2F104004044494624F0CB
:10E2900081FDC9F80040EAE7704700BF2DE9F84367
:10E2A0000B1A432B1CDD00F14008894641461746F6
:10E2B000FFF7BEFFC14515D0D8F80050444601E035
:10E2C000236863602646284654F8041DB847002892
:10E2D000F6D108F10408C1453560EDD1BDE8F883F9
:10E2E000FFF7A6FFBDE8F8832DE9F04F561E06EBB9
:10E2F000D67683B07610B14201928846054699469B
:10E300000C9F5CDA8A4600E0DA460AF101034FEA24
:10E31000430B0BF18041013955F8330055F82110BA
:10E3200005EBC304B84718B10BF1FF3B05EB8B04B9
:10E33000236845F82A30B345E6DB019BDA0707D4AA
:10E34000019BA3F1020A0AEBDA7ABBEB6A0F06D053
:10E35000C34514DCC4F8009003B0BDE8F08F0BF1A6
:10E36000010B4FEA4B0B0BF18043013B0BF1FF3BE1
:10E3700055F823302360C34505EB8B04EADD0BF130
:10E38000FF3606EBD6767610494655F82600B84794
:10E39000731E03EBD37305EB86045B1030B905EBFA
:10E3A0008B04C4F8009003B0BDE8F08F55F8262028
:10E3B00045F82B20B045CDDAB3461E46E4E7019B75
:10E3C000DB0700EB8104C5D48B46B9E72DE9F04F9C
:10E3D0000C1A432C85B040F3898005468946924645
:10E3E0001E46002A61D0031D0393E410686855F8A7
:10E3F0002410B0470AF1FF3A59F8041C002834D021
:10E4000055F82400B047002837D02B6855F8242051
:10E410002A6045F8243068682968039FCB46B846CF
:10E42000B04780B9ABF1040421682868A346043CD6
:10E43000B0470028F8D15F4509D23A68DBF80010F0
:10E440003960CBF8002057F8040F2968E7E7494600
:10E450003346524638467C1BFFF7B8FF432C45DD58
:10E46000BAF1000F22D0B946BFE76868B04798B14B
:10E4700095E8030029606860CFE759F8041C6868D4
:10E48000B0470028F4D02B6859F8042C2A6049F8CA
:10E49000043C68682968C0E759F8041C55F8240052
:10E4A000B0472B680028B1D0EEE78846A410A71E1D
:10E4B0007F1005EB870900E0013F59F80439009609
:10E4C000224639462846FFF70FFF002FF4D158F8AF
:10E4D000043D2A680096C5EB0804C8F80020002116
:10E4E000A2102846FFF700FF072CF0DC05B0BDE8BE
:10E4F000F08F00BF836833B15E4B1B6813B10121FD
:10E500000220184770472DE9F04700F12C074FEA29
:10E51000810907EB0906B74215468846044610D024
:10E520004FEAA902B2FA82F2C2F11F02520031464A
:10E530003846514BFFF74AFF4F4A31463846FFF7FE
:10E54000ADFEE06AA0658269002A00F0888082EA58
:10E55000E273A3EBE273B8F1010F4FF00002036125
:10E56000826012DD09F1280EA6443A4652F8041FD3
:10E570008B6983EAE37CACEBE37CC1F810C00369F0
:10E580007245C3EB4C034B61F0D1B7426ED0406A89
:10E5900004F1300306E01A68526A904203F1040362
:10E5A00028BF10469E42F6D106460023271D84F858
:10E5B000903084F8283038461DF09EFE20623846A0
:10E5C0001DF09AFE60621DF06BFE616904F10800A7
:10E5D0001DF01CFEA36D276F98695B6823F0E4FBB8
:10E5E000C4F88000304623F0DBFB0646384623F0B3
:10E5F000D7FB0146304623F02BFC204923F0DCFCFE
:10E600000023C4F88400E36772B6D4F88430C4F8F9
:10E61000883062B672B6D4F88010284623F018FC11
:10E62000E16FA06723F0D0FDD8B1D4F88830C4F8EA
:10E630008C3062B6124A236AE06900211160DB0067
:10E64000516803F1804303F5603301440D201961E3
:10E650001060DA68502122F08002DA60D960BDE8EB
:10E66000F087D4F8883003F10043E0E7E36A5E6A9C
:10E670009BE700BF44A0FF1F9904000000247449D9
:10E68000008003402DE9F04FA94DD5F8D830D3B024
:10E69000A3F10A021D2A00905FD9A64CA64B22685E
:10E6A0000A9200210A9A197023680993099B9B1A00
:10E6B000092BF9D9A149A24FA24EDFF8D0922DA87B
:10E6C00021F01CF900212DA8F3F724FB2DA821F03F
:10E6D000D5F89D4B2DA8196821F010F900212DA81F
:10E6E000F3F718FB2DA821F0C9F8984B4FF001085B
:10E6F00041F2883205212DA8C3F80080FFF7E8FC1D
:10E70000BB6D0293184600233360914E91493360EC
:10E71000914A924E0B60136033609149914A924E38
:10E720000B6013608DF844313360904BCDF820813D
:10E730000621052219608E4BC9F800202D93D5F8CB
:10E740001CB0D5F818A0042800F20A85DFE810F004
:10E750002401650137014E010A00D8B200211EF0E4
:10E760009DFB9AE7814A786A13234FF01208C2F89A
:10E770000080C9F80030039323F016FB7D4923F095
:10E7800067FB3A69D5F870B0D5F86CA0BB6B019007
:10E790000098069302FB00F2039B04924146764ADE
:10E7A000029E16607548764A016013605FFA8BF12D
:10E7B0005FFA8AF31E4608460291012103931EF078
:10E7C0006DFB304601211EF069FB684BD9F8002033
:10E7D00019680DF1740840461DF024FC00231E93B7
:10E7E00023680C930C9A23680B930B9B514E9B1A36
:10E7F000042BF8D9049940461DF056FC06991DF0EB
:10E8000047FC01221146B86DF3F7A0FABB6D002B4F
:10E8100040F01A84DFF87891D9F87420012A00F0CA
:10E820003284479952A800EB8100864640F8688CF4
:10E830004FF07E524EF8643C01212DA84793FFF71C
:10E8400059FE33681093109A23680F930F9B9B1AFD
:10E85000042BF9D900238DF8443172B64D990198F3
:10E8600023F0F6FA4C994B9023F0AEFC002800F010
:10E8700018834F9B509362B62F9B424EDFF8148152
:10E8800093B31EF029FF002840F300833068F3F7AC
:10E89000CDFDC0B26E2888F8000000F0DD826F2840
:10E8A00000F09382532800F06782ABF10A031D2B1E
:10E8B00040F2C480AAF10A031D2B40F2EE80D5F885
:10E8C000D000DFF86C90A0F10A031D2B40F21581F7
:10E8D00023681893189A23681793179B9B1A092B80
:10E8E000F9D92F9B002BCCD1274CB86D1E9B184A11
:10E8F000002840F0D182134910600B605A42174B38
:10E900001A6001220021F3F721FA2468022C00F09A
:10E91000D0820B2C40F02182BB6D042B00F21D82B3
:10E92000DFE813F0B801810163014501270100BF51
:10E93000BC96FF1F7CA0FF1F5594FF1F7882030029
:10E94000BC94FF1F1C93FF1FA487FF1F9C9AFF1FEF
:10E950005499FF1FDC95FF1FF09AFF1FA893FF1F1C
:10E96000B493FF1FB893FF1FAC93FF1F8887FF1F4F
:10E970008C6303000AD7233C7487FF1F3C87FF1F6B
:10E980005487FF1F8087FF1F6C87FF1F2887FF1F8B
:10E99000E095FF1F8595FF1FB24A786902234FF06B
:10E9A0000308C2F80080C9F80030039323F0FCF993
:10E9B000AD4923F04DFA3A680190BB6AE8E6A94AEE
:10E9C000F86914234FF01508C2F80080C9F8003028
:10E9D000039323F0E9F9A44923F03AFABA680190C5
:10E9E000D5F830B0D5F82CA03B6BD1E69D4A386AFB
:10E9F00017234FF01008C2F80080C9F800300393C5
:10EA000023F0D2F9984923F023FAFA680190D5F857
:10EA100050B0D5F84CA07B6BBAE6B86923F0C4F9C6
:10EA2000914923F015FAFA6A7B680692009A0190E0
:10EA300003FB02F3049306210523B0E602981EF0BF
:10EA400033FAD5F8D43098423FF434AF009B012B11
:10EA50007FF430AF00238DF8443172B600214D9819
:10EA600023F0F6F94C994B9023F0AEFB002800F010
:10EA700073834F9B509362B630A820F00BFC7B4C05
:10EA8000359800232F931DF04BFC36981DF048FC61
:10EA900020680121FFF7A8F927E703981EF004FA80
:10EAA000D5F8D43098423FF40AAF009B01337FF48D
:10EAB00006AF00238DF8443172B600214D9823F043
:10EAC000C7F94C994B9023F07FFB002800F040835E
:10EAD0004F9B509362B630A820F0DCFB634C359816
:10EAE00000232F931DF01CFC36981DF019FC2068A4
:10EAF0004FF0FF31FFF778F9F7E6C0B21EF0D4F916
:10EB0000D9F8D43098423FF4E3AE30A8002420F086
:10EB1000C1FB35982F941DF003FC36981DF000FCC6
:10EB2000224621462046F3F711F9224621460120CC
:10EB3000F3F70CF9224621460220F3F707F92246A3
:10EB400021460320F3F702F9224621460420F3F779
:10EB5000FDF8464B1868FEF7B3FBD9F8D800A0F1D2
:10EB60000A031D2B00F20081C0B201211EF096F9AC
:10EB7000FAE0D5F8CC30012B00F0EF803C4919A821
:10EB800020F0BCFE002119A8F3F7C4F819A820F062
:10EB900075FE384919A820F0B1FE002119A8F3F735
:10EBA000B9F819A820F06AFE19A83349ABE0D5F8E6
:10EBB000CC30012B00F0D180304919A820F09EFE06
:10EBC000002119A8F3F7A6F819A820F057FE294943
:10EBD00019A820F093FE002119A8F3F79BF819A8B3
:10EBE00020F04CFE19A826498DE0D5F8CC30012B39
:10EBF00000F0B380234919A820F080FE002119A855
:10EC0000F3F788F819A820F039FE1A4919A820F05E
:10EC100075FE002119A8F3F77DF819A820F02EFE43
:10EC200019A819496FE0D5F8CC30012B00F0958078
:10EC3000164919A820F062FE002119A8F3F76AF816
:10EC400019A820F01BFE0B4919A820F057FE00213F
:10EC500019A8F3F75FF819A820F010FE19A80C49BD
:10EC600051E000BF8887FF1F0AD7233C6C87FF1F36
:10EC7000008403004064030018840300D083030071
:10EC8000E8830300A0830300B883030070830300BC
:10EC900088830300D5F8CC30012B5ED0AE4919A88B
:10ECA00020F02CFE002119A8F3F734F819A820F061
:10ECB000E5FDAA4919A820F021FE002119A8F3F7C3
:10ECC00029F819A820F0DAFD19A8A5491BE0D5F804
:10ECD000CC30012B41D0A34919A820F00FFE002110
:10ECE00019A8F3F717F819A820F0C8FD9B4919A82F
:10ECF00020F004FE002119A8F3F70CF819A820F061
:10ED0000BDFD994919A820F0F9FD002119A8F3F7D4
:10ED100001F819A820F0B2FD944919A820F0EEFDE1
:10ED2000002119A8F2F7F6FF19A820F0A7FD9049D5
:10ED300019A820F0E3FD002119A8F2F7EBFF19A8AC
:10ED400020F09CFD8B4919A820F0D8FD19A80021BE
:10ED5000F2F7E0FF19A820F091FDD5F8D800A0F156
:10ED60000A031D2B7FF600AF834B2D932DA8FFF7D1
:10ED7000FBF953B0BDE8F08F00238DF8443172B633
:10ED800000214D9823F064F84C994B9023F01CFA25
:10ED9000002800F08A804F9B509362B62368169338
:10EDA000169A23681593159B744E9B1A042BF8D959
:10EDB0002DA8FFF733F933681493149A236813933B
:10EDC000139B9B1A632BF9D98EE53068F2F7FCFA96
:10EDD00022F098FEBB6D013B032B0AD8DFE803F05D
:10EDE00028302002786222F0DFFF654923F030F8F6
:10EDF0000190644B6448196878221DF0EDFE0023F1
:10EE00008DF8443172B64D99019823F021F84C9950
:10EE10004B9023F0D9F9D8B14F9B509362B644E59B
:10EE2000386222F0C1FF564923F012F80190E0E762
:10EE3000B86122F0B9FF524923F00AF80190D8E7EF
:10EE4000F86122F0B1FF4E4923F002F80190D0E7BB
:10EE50004F9B03F10043E0E73068F2F7B5FA22F088
:10EE600051FE786122F0A0FF454922F0F1FF454BA9
:10EE7000019019688146782243481DF0ADFE0023B9
:10EE80008DF8443172B64D994846BEE7F1F702FC61
:10EE900000287FF70AADF9E413603C4A5B42136037
:10EEA0002FE54F9B03F10043E4E44F9B03F1004344
:10EEB00072E7374B5A6F012A00F03E81BB6D042B7D
:10EEC0003FF64BAF01A252F823F000BFCFEC000099
:10EED000E1EF0000A5EF00001DEF0000E1EE0000F3
:10EEE000D5F8CC30012B3FF438AF2A4919A820F0CF
:10EEF00005FD002119A8F2F70DFF19A820F0BEFCAE
:10EF0000164919A820F0FAFC002119A8F2F702FF0F
:10EF100019A820F0B3FC19A81F49F4E6D5F8CC30A5
:10EF2000012B3FF41AAF1D4919A820F0E7FC00217E
:10EF300019A8F2F7EFFE19A820F0A0FC074919A8BC
:10EF400020F0DCFC002119A8F2F7E4FE19A820F05B
:10EF500095FC19A81249D6E63084030040640300EA
:10EF600048840300488303005C8303004866030071
:10EF7000BC820300C88203008C6303007CA0FF1FD7
:10EF80000AD7233C5C87FF1FBC94FF1FA893FF1F79
:10EF9000E095FF1F2083030034830300F882030001
:10EFA0000C830300D5F8CC30012B3FF4D6AE714969
:10EFB00019A820F0A3FC002119A8F2F7ABFE19A8AC
:10EFC00020F05CFC6C4919A820F098FC002119A8DD
:10EFD000F2F7A0FE19A820F051FC19A8674992E6A3
:10EFE000D5F8CC30012B3FF4B8AE654919A820F014
:10EFF00085FC002119A8F2F78DFE19A820F03EFC2F
:10F000005D4919A820F07AFC002119A8F2F782FEC8
:10F0100019A820F033FC5A4919A820F06FFC0021F0
:10F0200019A8F2F777FE19A820F028FC524919A870
:10F0300020F064FC002119A8F2F76CFE19A820F05A
:10F040001DFC19A84F495EE6479B52A903F10B002E
:10F0500001EB800001EB8301002341F8688C4FF045
:10F060007E5240F8903C01212DA84793FFF742FAC9
:10F0700033681293129A23681193119B9B1A042BE5
:10F08000F9D9FFF7E7BBDFF818C10693DFF814E101
:10F090003D49049807920323CCF800304FF0100C40
:10F0A000CEF800C04FF0170EC1F800E022F07CFE51
:10F0B000D9F87010DFF8DC9022F0CAFE334922F054
:10F0C000C7FE22F01BFA20F0E1FE079ACDE9040109
:10F0D00011460320F2F73AFE069BC9F80430DDE939
:10F0E000040122F00FFD014648461CF0DDFF284BCD
:10F0F000996A1CF0CDFF33680E930E9A23680D9326
:10F100000D9B9B1A042BF9D9479B52A903F10C06BE
:10F1100001EB830001EB8606002340F8688C40F881
:10F12000649C4FF07E5246F8903C02212DA84793F4
:10F13000FFF7E0F9FFF7A0BB00210320F2F706FE7E
:10F14000144B154A5B681460144A5B421360B5E6C1
:10F150004F9B03F10043BCE44F9B03F1004389E460
:10F160000023002206930493019205230621FFF752
:10F1700016BB00BFD082030040640300E48203009A
:10F1800094820300A8820300B487FF1F0AD7233CA0
:10F190005C96FF1F8895FF1F9C9AFF1FAC93FF1F73
:10F1A0007887FF1FB087FF1F2DE9F04F434ED6F839
:10F1B000D830ADF5697DA3F10A041D2C00900691AD
:10F1C000154641F2BC8241F2883205219EA8FEF725
:10F1D0007FFF00273A4B9E934FF0010841F288329F
:10F1E0000521C3A8CDF8E4828DF80873354CDFF80B
:10F1F000ECA0FEF76DFF324BCDF87883022203219D
:10F200004EA8C3938DF89C731CF00CFFB169226863
:10F210002D4B019106210992CAF800102B491F704D
:10F22000099AD6F81C8005230B6023680893089B75
:10F230009B1A092BF9D926498EA820F05FFB0021E3
:10F240008EA8F2F767FD8EA820F018FB214B8EA840
:10F25000196820F053FB8EA80021F2F75BFD8EA801
:10F2600020F00CFB002D41F370824FF000090125C6
:10F27000052206215EA81CF0D5FE142215216EA8D9
:10F280001CF0D0FE144F172210217EA81CF0CAFEDD
:10F29000132212218EA81CF0C5FEBB6D0022591E40
:10F2A0005F926F927F928F924F92032901F2828236
:10F2B000DFE811F0AA0183015C011600BC96FF1F74
:10F2C0008C6303007CA0FF1F5594FF1F2887FF1F3E
:10F2D00078820300A487FF1FE095FF1F8887FF1F28
:10F2E000786A22F061FDBB6B39690293009B019043
:10F2F00001FB03F1924BD6F870B0D6F86C80122265
:10F3000013201860CAF800208EA800228F921CF0EB
:10F31000CBFE029B19461CF0BBFE23681193119A89
:10F3200023681093109B9B1A042BF9D9BB6D844A58
:10F330008449D2F800C0DAF80000DFF820E2086063
:10F340005FFA88F25FFA8BF102927F4A03910846D6
:10F3500001211360CEF800C01DF0A0FD029801212C
:10F360001DF09CFD236813937B6907933B6804930E
:10F37000139ABB6A059323681293129BDFF8E0A1EE
:10F380009B1A042BF7D9049A069B03FB02F3194638
:10F390004EA806931CF088FE05991CF079FE7A6F42
:10F3A0006A4B0221012A196001F00D82002D41F003
:10F3B000378101230693B9F1000F41F05781644A68
:10F3C000644B12681B681DB9B9F1000F01F0F2809F
:10F3D000D6F8D000DFF88CA1A0F10A031D2B40F273
:10F3E0006F8723682393239A23682293229B9B1A77
:10F3F000042BF9D91EF070F9002840F3B287DFF82A
:10F4000068A1DAF80000F3F711F8534AC0B2A0F18E
:10F4100042031070902B00F22781DFE813F01C01EB
:10F4200025012501250125012501250125012501AC
:10F43000250125012501250125012501250125019C
:10F44000CC04250125012501250125012501F4050F
:10F45000AF052501250125012501250125012501EE
:10F46000A3042501250125012501250125012501EB
:10F470005704F2032501ED02CA02250125012501E9
:10F48000250125012501250125012501250125014C
:10F49000250125012501250125012501250125013C
:10F4A000250125012501250125012501250125012C
:10F4B000250125012501250125012501250125011C
:10F4C000250125012501250125012501250125010C
:10F4D00025012501250125012501250125012501FC
:10F4E000250125014101AF03250125012501250144
:10F4F00014035803250125012501250125012501B6
:10F5000025012501250125012501250125012501CB
:10F5100025012501250125012501250125012501BB
:10F52000250125011C0125012501250125012501B4
:10F530002501250125012501250125013706400565
:10F540002887FF1FB087FF1F7887FF1F9C9AFF1F28
:10F5500090F00F40D0F00F408595FF1FB487FF1F3C
:10F560007CA0FF1FBC96FF1F8087FF1F386A22F018
:10F570001BFC7B6BF9680293009B019001FB03F17C
:10F58000444BD6F850B0D6F84C80102217201860A3
:10F59000CAF800207EA800227F921CF085FD029B05
:10F5A00019461CF075FD23680F930F9A23680E937C
:10F5B0000E9B9B1A042BF9D9B8E6F86922F0F4FBEC
:10F5C0003B6BB9680293009B019001FB03F1314B47
:10F5D000D6F830B0D6F82C80152214201860CAF85E
:10F5E00000206EA800226F921CF05EFD029B19465F
:10F5F0001CF04EFD23680D930D9A23680C930C9B11
:10F600009B1A042BF9D991E6B86922F0CDFBFB6A6D
:10F6100079680293009B019001FB03F11D4BD6F822
:10F620001CB0D6F81880062205201860CAF8002001
:10F630005EA800225F921CF037FD029B19461CF069
:10F6400027FD23680B930B9A23680A930A9B9B1A46
:10F65000042BF9D96AE6F2F7F7FE0F4BB865196883
:10F660000E4878221DF0B8FA55B1ABF10A031D2BF4
:10F6700071D9A8F10A031D2B4FF0010540F2EB8070
:10F6800023684993499A23684893489B9B1A042B03
:10F69000F9D998E62887FF1F8C87FF1FE095FF1F89
:10F6A000DDF814A3BAF1000FDED1F86922F07CFB7B
:10F6B000C84922F0CDFBB968019049426EA81CF000
:10F6C000F3FC012211460220F2F740FBDD9BCDF84E
:10F6D00074A3E8A901EB830003466EAD40F8685CB3
:10F6E0004FF07E520121C3A843F864ACFEF702FF3D
:10F6F0008DF89CA372B60021E39822F0A9FBE29951
:10F70000E19022F061FD002801F03E82E59BE69346
:10F7100062B623683793379A23683693369B9B1AD1
:10F72000042BF9D900238DF89C3372B6E399019824
:10F7300022F08EFBE299E19022F046FD002801F0D4
:10F74000F581E59BE69362B64FF0FF330093ABF192
:10F750000A031D2B8DD803981DF0A6FBD6F8D430D4
:10F76000984286D0009B012B83D100238DF89C33D7
:10F7700072B60021E39822F06BFBE299E19022F04F
:10F7800023FD002800F01187E59BE69362B6C6A82A
:10F790001FF080FD0025CB98C5951CF0C1FDCC98CD
:10F7A0001CF0BEFDD6F8B430002B40F07286D6F8BF
:10F7B000CC30012B0DF5947A00F0E986864950464D
:10F7C00020F09CF800215046F2F7A4FA504620F0B1
:10F7D00055F88249504620F091F800215046F2F742
:10F7E00099FA504620F04AF87D49504620F086F8B4
:10F7F00000215046F2F78EFA504620F03FF8794942
:10F80000504620F07BF800215046F2F783FA50462C
:10F8100020F034F87449504620F070F8002150462A
:10F82000F2F778FA504620F029F87049504620F057
:10F8300065F800215046F2F76DFA504620F01EF8A8
:10F8400001210846FEF7D0FAA8F10A031D2B4FF05C
:10F8500000053FF615AF02981DF026FBD6F8D43010
:10F8600098423FF40DAF009B01337FF409AF0023B2
:10F870008DF89C3372B60021E39822F0E9FAE29900
:10F88000E19022F0A1FC002800F0FE85E59BE693C4
:10F8900062B6C6A81FF0FEFC0025CB98C5951CF0EB
:10F8A0003FFDCC981CF03CFDD6F8B430002B40F066
:10F8B0005F85D6F8CC30012B0DF5947A00F0D68513
:10F8C0004549504620F01AF800215046F2F722FA36
:10F8D00050461FF0D3FF4149504620F00FF8002159
:10F8E0005046F2F717FA50461FF0C8FF3C49504601
:10F8F00020F004F800215046F2F70CFA50461FF0B1
:10F90000BDFF384950461FF0F9FF00215046F2F77D
:10F9100001FA50461FF0B2FF334950461FF0EEFF88
:10F9200000215046F2F7F6F950461FF0A7FF2F4985
:10F9300050461FF0E3FF00215046F2F7EBF9504626
:10F940001FF09CFF2A4950461FF0D8FF0021504667
:10F95000F2F7E0F950461FF091FF204950461FF0A2
:10F96000CDFF00215046F2F7D5F950461FF086FF33
:10F9700023684793479A23684693469B9B1A092B13
:10F98000F9D91C4950461FF0B9FF00215046F2F743
:10F99000C1F950461FF072FF104950461FF0AEFFEC
:10F9A00000215046F2F7B6F950461FF067FF0025D8
:10F9B00066E6DAF80000F1F707FD22F0A3F8BA6D69
:10F9C000013A032A00F23584DFE812F0550472048C
:10F9D0004D042C040AD7233CB08403004064030088
:10F9E000C484030048660300BC820300C88203008D
:10F9F000207F0300387F0300DAF80000F1F7E4FC11
:10FA000022F080F8AE4B82461968AE48C7F814A0C1
:10FA100078221DF0E1F800238DF8083372B65046C5
:10FA200022F0C2F9A84922F013FABE9922F010FA86
:10FA3000BD99BC9022F0C8FB002800F01286C09B44
:10FA4000C19362B610E6DDF814A3BAF1000F7FF49B
:10FA50000BAE386A22F0A8F99B4922F0F9F9F9684F
:10FA6000019049427EA81CF01FFB01221146032091
:10FA7000F2F76CF9DD9BCDF874A3E8A901EB8300E4
:10FA800003467EAD40F8685C4FF07E520121C3A86A
:10FA900043F864ACFEF72EFD8DF89CA372B60021EE
:10FAA000E39822F0D5F9E299E19022F08DFB00284D
:10FAB00001F06580E59BE69362B623683B933B9A31
:10FAC00023683A933A9B9B1A042BF9D92AE6DDF86E
:10FAD00014A3BAF1000F7FF4C7AD386A22F064F9BD
:10FAE000794922F0B5F9F96801907EA81CF0DCFA9A
:10FAF000012211460320F2F729F9DD9BCDF874A30A
:10FB0000E8A901EB830003467EAD40F8685C4FF046
:10FB10007E520121C3A843F864ACFEF7EBFC8DF8DC
:10FB20009CA372B60021E39822F092F9E299E19049
:10FB300022F04AFB002801F0D380E59BE69362B6F1
:10FB400023683D933D9A23683C933C9B9B1A042B6E
:10FB5000F9D900238DF89C3372B6E399019822F00D
:10FB600077F9E299E19022F02FFB002800F0E3877B
:10FB7000E59BE69362B60123009376E5DDF814A3D6
:10FB8000BAF1000F7FF470ADF86922F00DF94E491B
:10FB900022F05EF9B96801906EA81CF085FA012286
:10FBA00011460220F2F7D2F8DD9BCDF874A3E8A944
:10FBB00001EB830003466EAD40F8685C4FF07E5267
:10FBC0000121C3A843F864ACFEF794FC8DF89CA314
:10FBD00072B60021E39822F03BF9E299E19022F01D
:10FBE000F3FA002800F0DA87E59BE69362B6236813
:10FBF0003993399A23683893389B9B1A042BF9D987
:10FC0000A7E7DDF880A2BAF1000F7FF42DAD786987
:10FC100022F0CAF8049B2C49C3F1000922F018F91C
:10FC2000494607904EA81CF03FFA01221146504663
:10FC3000F2F78CF87A6F012A01F00A80B89ACDF8B1
:10FC4000E0A29EAB03EB820108464EABCB624FF0C5
:10FC50007E52C0F830A001219EA8FEF74BFC002385
:10FC60008DF8083372B60021BE9822F0F1F8BD99E4
:10FC7000BC9022F0A9FA002800F0E587C09BC19350
:10FC800062B623683593359A23683493349B9B1A64
:10FC9000042BF9D900238DF8083372B60798BE9962
:10FCA00022F0D6F8BD99BC9022F08EFA002800F020
:10FCB0005787C09BC19362B64FF00109D4E400BFDF
:10FCC0008C87FF1FE095FF1F0AD7233CDDF880A239
:10FCD000BAF1000F7FF4C8AC786922F065F8A0494A
:10FCE00022F0B6F8049981464EA81CF0DDF90122F5
:10FCF00011465046F2F72AF87A6F012A00F05D8724
:10FD0000B89ACDF8E0A29EAB03EB820108464EAB59
:10FD1000CB624FF07E52C0F830A001219EA8FEF7C2
:10FD2000E9FB00238DF8083372B60021BE9822F05B
:10FD30008FF8BD99BC9022F047FA002800F0338775
:10FD4000C09BC19362B623683193319A2368309384
:10FD5000309B9B1A042BF9D900238DF8083372B617
:10FD600048469CE700238DF89C3372B60021E39847
:10FD700022F06EF8E299E19022F026FA002800F0D5
:10FD80006784E59BE69362B623682B932B9A2368DE
:10FD90002A932A9B9B1A042BF9D9C3A8FEF73EF994
:10FDA000BB6D013B032B00F2C381DFE813F02F0290
:10FDB00016023502BC0100238DF8083372B600210B
:10FDC000BE9822F045F8BD99BC9022F0FDF90028BC
:10FDD00000F03984C09BC19362B623682593259AAD
:10FDE00023682493249B9B1A042BF9D99EA8FEF721
:10FDF00015F97A6F012A00F0588600210846012281
:10FE0000F1F7A4FFD6F8CC300DF5947A012B5046CB
:10FE100000F0C28453491FF071FD00215046F1F7F4
:10FE200079FF50461FF02AFD4F4950461FF066FDEE
:10FE300000215046F1F76EFF50461FF01FFD4B4961
:10FE400050461FF05BFD00215046F1F763FF50461E
:10FE50001FF014FD464950461FF050FD002150464A
:10FE6000F1F758FF50461FF009FD424950461FF078
:10FE700045FD00215046F1F74DFF50461FF0FEFCB6
:10FE80003D4950461FF03AFD50460021F1F742FF30
:10FE900050461FF0F3FC4FF00009FFF7E5BBDDF81B
:10FEA00014A3BAF1000F7FF4DFAB736D786A012BF6
:10FEB0000CBF4FF0FF3301231D46009321F074FF68
:10FEC000274921F0C5FF3969019001FB05F18EA892
:10FED0001CF0EAF8012211460420F1F737FFDD9B00
:10FEE000CDF874A3E8A901EB830003468EAD40F87A
:10FEF000685C4FF07E520121C3A843F864ACFEF762
:10FF0000F9FA8DF89CA372B60021E39821F0A0FFC6
:10FF1000E299E19022F058F9002800F02B86E59B49
:10FF2000E69362B623684193419A23684093409BCD
:10FF30009B1A042BF9D900238DF89C3372B6E399F0
:10FF4000019821F085FFE299E19022F03DF9002827
:10FF500000F0B185E59BE69362B6FFF786BB00BF74
:10FF60000AD7233C748403004064030088840300A0
:10FF700048660300BC820300C8820300DDF814A3B6
:10FF8000BAF1000F7FF470ABB86921F00DFFBE49E4
:10FF900021F05EFF7968019049425EA81CF084F868
:10FFA000012211461046F1F7D1FEDD9BCDF874A376
:10FFB000E8A901EB830003465EAD40F8685C4FF0B2
:10FFC0007E520121C3A843F864ACFEF793FA8DF882
:10FFD0009CA372B60021E39821F03AFFE299E190E8
:10FFE00022F0F2F8002800F0D485E59BE69362B693
:10FFF00023682993299A23682893289B9B1A042B0A
:020000021000EC
:10000000F9D9FFF78FBBDDF814A3BAF1000F7FF425
:100010002BABB86921F0C8FE9B4921F019FF796824
:1000200001905EA81CF040F8012211461046F1F73D
:100030008DFEDD9BCDF874A3E8A901EB8300034698
:100040005EAD40F8685C4FF07E520121C3A843F8D2
:1000500064ACFEF74FFA8DF89CA372B60021E398CA
:1000600021F0F6FEE299E19022F0AEF8002800F0CF
:100070009F85E59BE69362B623682793279A2368BA
:100080002693269B9B1A042BF9D962E5DDF814A36D
:10009000BAF1000F7FF4E8AA736D786A012B0CBFE8
:1000A00001234FF0FF331D46009321F07DFE76497A
:1000B00021F0CEFE3969019001FB05F18EA81BF0FD
:1000C000F3FF012211460420F1F740FEDD9BCDF83D
:1000D00074A3E8A901EB830003468EAD40F8685C89
:1000E0004FF07E520121C3A843F864ACFEF702FA38
:1000F0008DF89CA372B60021E39821F0A9FEE29945
:10010000E19022F061F8002800F02F85E59BE6934E
:1001100062B623683F933F9A23683E933E9B9B1AA7
:10012000042BF9D907E7012200210420F1F70EFE84
:10013000D6F8CC300DF5947A012B504659D053495E
:100140001FF0DCFB00215046F1F7E4FD50461FF0A4
:1001500095FB4F4950461FF0D1FB00215046F1F767
:10016000D9FD50461FF08AFB4A4950461FF0C6FB96
:1001700000215046F1F7CEFD50461FF07FFB464967
:1001800050461FF0BBFB00215046F1F7C3FD50461F
:100190001FF074FB414950461FF0B0FB0021504650
:1001A000F1F7B8FD50461FF069FB3D4950461FF07E
:1001B000A5FB50460021F1F7ADFD50461FF05EFB58
:1001C00023682D932D9A23682C932C9B9B1AB3F5AF
:1001D0007A7FF8D30025FFF753BA022001220021CD
:1001E000F1F7B4FDD6F8CC300DF5947A012B5046DA
:1001F000A5D12C491FF082FB00215046F1F78AFD62
:1002000050461FF03BFB50462149D0E701221046E3
:100210000021F1F79BFD8BE7012200210320F1F77C
:1002200095FD85E7786221F0BFFD174921F010FEAA
:1002300001901D4B1D48196878221CF0CDFC00234D
:100240008DF89C3372B6E399019821F001FEE29992
:10025000E19021F0B9FF002800F0FF81E59BE693D3
:1002600062B6FFF701BA386221F09EFD064921F01F
:10027000EFFD0190DDE7B86121F096FD024921F024
:10028000E7FD0190D5E700BF0AD7233CB084030007
:1002900040640300C484030048660300BC8203007A
:1002A000C88203009C8403008C87FF1FE095FF1F1A
:1002B000F86121F079FDCD4921F0CAFD0190B8E740
:1002C000C0B21CF0F1FDDAF8D43098423FF489A8AE
:1002D000A1A800241EF0DEFFA698A0941CF020F830
:1002E000A7981CF01DF8C6A81EF0D4FFCB98C594A3
:1002F0001CF016F8CC981CF013F8BD4B01252246D3
:10030000214620461D70F1F721FD22462146284650
:10031000F1F71CFD224621460220F1F717FD224687
:1003200021460320F1F712FD224621460420F1F771
:100330000DFD2846FCF7C4FFDAF8D800A0F10A0347
:100340001D2B40F2C783AB4BC393C3A8FDF70CFF33
:10035000A84B9E939EA8FDF707FF0DF5697DBDE8AC
:10036000F08FF0F797F90028FFF67EA9FFF747B85E
:100370008DF8085372B60021BE9821F069FDBD9931
:10038000BC9021F021FF002800F05581C09BC19353
:1003900062B623684593459A23684493449B9B1A0D
:1003A000042BF9D9A1A81EF075FF0025A698A095E9
:1003B0001BF0B6FFA7981BF0B3FF7A6F012A00F07D
:1003C0008483002108460122F1F7C0FCD6F8CC3026
:1003D0000DF5947A012B504600F0D18186491FF02B
:1003E0008DFA00215046F1F795FC50461FF046FA71
:1003F000824950461FF082FA00215046F1F78AFCEC
:1004000050461FF03BFA7E4950461FF077FA002114
:100410005046F1F77FFC50461FF030FA79495046BC
:100420001FF06CFA00215046F1F774FC50461FF0A3
:1004300025FA754950461FF061FA00215046F1F740
:1004400069FC50461FF01AFA704950461FF056FAE0
:1004500050460021F1F75EFC50461FF00FFAD6F827
:10046000CC30012B4FF000097FF42AAA684950468E
:100470001FF044FA00215046F1F74CFC50461FF0A3
:10048000FDF95E49FFF754BAE59B03F10043FFF71E
:10049000FEB98DF8085372B60021BE9821F0D8FC41
:1004A000BD99BC9021F090FE002800F0C880C09B50
:1004B000C19362B623684393439A23684293429B55
:1004C0009B1A042BF9D9A1A81EF0E4FE0025A698DA
:1004D000A0951BF025FFA7981BF022FF7A6F012A39
:1004E00000F0EE82002108460122F1F72FFCD6F839
:1004F000CC300DF5947A012B504600F033813E4903
:100500001FF0FCF900215046F1F704FC50461FF0A3
:10051000B5F93A4950461FF0F1F900215046F1F77C
:10052000F9FB50461FF0AAF9354950461FF0E6F98D
:1005300000215046F1F7EEFB50461FF09FF931497C
:1005400050461FF0DBF900215046F1F7E3FB50461F
:100550001FF094F92C4950461FF0D0F90021504665
:10056000F1F7D8FB50461FF089F9284950461FF093
:10057000C5F950460021F1F7CDFB50461FF07EF93A
:10058000D6F8CC30012B4FF000097FF417A9204991
:1005900050461FF0B3F900215046F1F7BBFB50461F
:1005A0001FF06CF91549FFF741B9E59B03F10043D2
:1005B000FFF7EBB87F9B069B002B00F0B480154C37
:1005C0007A6F1548154B4F9D21680560012A196007
:1005D00000F08582D6F8D800A0F10A031D2B3FF663
:1005E000B2AEC0B201211CF059FCACE60AD7233CE4
:1005F000989AFF1F8C630300748403004064030017
:100600008884030048660300BC820300C88203009C
:100610009C8403005499FF1F1898FF1FF499FF1F33
:10062000BB6D013B032B00F26083DFE813F03D015B
:1006300075010501C701C09B03F10043A7E6C09BFC
:1006400003F1004334E7C09B03F10043FFF7C3BB52
:10065000E59B03F10043FFF795BBE59B03F10043E6
:10066000FDE5C09B03F10043FFF7EAB90122114603
:100670000020F1F76BFB23681F931F9A23681E93DA
:100680001E9B9B1A042BF9D97A6F012A00F02F8246
:10069000B89B9EA903F10B0001EB800001EB8301E5
:1006A0004FF0000E4EABCB624FF07E52C0F804E02C
:1006B00001219EA8CDF8E0E2FDF71CFF00238DF894
:1006C000083372B60021BE9821F0C2FBBD99BC90E0
:1006D00021F07AFD002874D1C09B03F10043C1933F
:1006E00062B623682193219A23682093209B9B1A4A
:1006F000092BF9D900238DF8083372B6079821F039
:1007000053FBA24921F0A4FBBE9921F0A1FBBD99A6
:10071000BC9021F059FD002800F0C381C09BC1931B
:1007200062B6FEF74CBEBB6D994C013B032B3FF606
:1007300047AFDFE813F0AA01A2019A019201D8B2F3
:1007400000211CF0ABFBFEF73EBD9249924A934B51
:1007500000250D600321116002221A604FF001098B
:10076000FEF786BD8E491FF0C9F800215046F1F70B
:10077000D1FA50461FF082F850468A49F7E6884978
:100780001FF0BCF800215046F1F7C4FA50461FF0A4
:1007900075F85046834959E681491FF0AFF80021AA
:1007A0005046F1F7B7FA50461FF068F850467D49B9
:1007B000FFF768BB0022C346DDF804800192FEF714
:1007C000B6BDC09B8BE7DFF8F0E1774A7749069822
:1007D0004FF0030CCEF800C0C3F800C04FF0100E6D
:1007E00017231360C1F800E000217F9121F0DCFAAB
:1007F0006F4B196821F02CFB6E4B06906349186F04
:1008000021F026FB069B0146184621F021FB21F032
:10081000FBFC01467EA81BF047FC05991BF038FC49
:10082000DAF800301593159A23681493149B9B1AD9
:10083000042BF9D9FEF7BABD012211460320F1F7C6
:1008400085FADD9BE8A903F10B0E01EB8E0E01EB9F
:1008500083034FF0000A7EA843F8680C4FF07E52E5
:100860000121C3A84EF890ACCDF874A3FDF742FE69
:100870008DF89CA372B60021E39821F0E9FAE29981
:10088000E19021F0A1FC002800F05E81E59BE69359
:1008900062B623681B931B9A23681A931A9B9B1AB0
:1008A000092BF9D9386AC0E0012211461046F1F748
:1008B0004DFADD9BE8A903F10B0E01EB8E0E01EB67
:1008C00083034FF0000A5EA843F8680C4FF07E5295
:1008D0000121C3A84EF890ACCDF874A3FDF70AFE31
:1008E0008DF89CA372B60021E39821F0B1FAE29949
:1008F000E19021F069FC002800F02A81E59BE69355
:1009000062B623681793179A23681693169B9B1A4F
:10091000092BF9D9B86988E0012211460220F1F7C4
:1009200015FA00238DF89C3372B60021E39821F06C
:100930008FFAE299E19021F047FC002800F00C8149
:10094000E59BE69362B6DD9BE8A803F10B0100EBA3
:10095000810100EB83034FF0000E6EA843F8680C92
:100960004FF07E5241F890ECC3A80121CDF874E31A
:10097000FDF7C0FD23681993199A23681893189BF3
:100980009B1A092BF9D9F8694FE000BF0AD7233C1D
:100990005499FF1F7487FF1F3C87FF1F5487FF1F59
:1009A0006084030040640300A887FF1F6087FF1F67
:1009B000849AFF1FE095FF1F3087FF1F0122114619
:1009C0000420F1F7C3F9DD9BE8A903F10B0E01EB5D
:1009D0008E0E01EB83034FF0000A8EA843F8680CDB
:1009E0004FF07E520121C3A84EF890ACCDF874A30D
:1009F000FDF780FD8DF89CA372B60021E39821F0ED
:100A000027FAE299E19021F0DFFB002800F09880BE
:100A1000E59BE69362B623681D931D9A23681C9399
:100A20001C9B9B1A092BF9D9786A21F0BDF9B149B1
:100A300021F00EFA00238DF89C3372B6E39921F071
:100A400007FAE299E19021F0BFFB30B3E59BE69312
:100A500062B600230693FEF7AEBC8F9B2360012293
:100A600000210420F1F772F9AAE57F9B236001229F
:100A700000210320F1F76AF9A2E56F9B23600122B0
:100A800000210220F1F762F99AE501225F9B2360C1
:100A900010460021F1F75AF992E5E59B03F1004376
:100AA000D5E7C09B03F1004339E600210320F1F7AD
:100AB0004DF9FFF7A2B9E59B03F10043FFF74BBAED
:100AC00029460320F1F742F90CE529460320F1F706
:100AD0003DF976E42946C0B21CF0E0F933E4002188
:100AE0000320F1F733F9844B7F9A1A6072E51146BF
:100AF0000320F1F72BF9B89B9EA901EB830E03F1BC
:100B00000C0001EB80004EAB7146CEF82C304FF05C
:100B1000000E7EAB0B634FF07E52C0F804E0022162
:100B20009EA8CDF8E0E2FDF7E5FCC7E5E59B03F103
:100B30000043FEF707BEE59B03F10043FFF719B83A
:100B4000E59B03F1004364E7E59B03F100439EE668
:100B5000E59B03F10043D2E6E59B03F10043F0E699
:100B6000C09B03F10043FFF7A5B8E59B03F10043E9
:100B7000FFF7CDBAE59B03F10043FFF7D1B9E59B41
:100B800003F10043FEF797BFE59B03F10043FEF737
:100B9000BEBDE59B03F10043FFF728BAE59B03F1D7
:100BA0000043FFF722B8C09B03F10043FFF7C9B829
:100BB000E59B03F10043FFF75DBA0498CDF8FCA173
:100BC00021F0F2F84D4B196821F042F94C4B49499C
:100BD0008246186F21F03CF90146504621F038F961
:100BE00021F012FB01467EA81BF05EFA05991BF06E
:100BF0004FFA23682F932F9A23682E932E9B9B1ACC
:100C0000042BF9D9012211460320F1F79FF8B89B74
:100C10009EA901EB83010DF51E7E03F10C000EEB86
:100C200080004EABCB624FF0000E7EAB0B634FF0FB
:100C30007E52C0F804E002219EA8CDF8E0E2FDF764
:100C400059FCFFF76EB8C09B03F10043FFF717B8DC
:100C50004846CDF8FCA121F0A7F8284B196821F0EF
:100C6000F7F8274B23498146186F21F0F1F8014628
:100C7000484621F0EDF800F1004021F0C5FA0146A8
:100C80007EA81BF011FA05991BF002FA2368339332
:100C9000339A23683293329B9B1A042BF9D9012291
:100CA00011460320F1F752F8B89B9EA901EB83018E
:100CB0000DF51E7E03F10C000EEB80004EABCB62F7
:100CC0004FF0000E7EAB0B634FF07E52C0F804E095
:100CD00002219EA8CDF8E0E2FDF70CFCFEF7BFBFB5
:100CE000E59B03F10043FEF729BF00230693FEF7BF
:100CF00062BB00BF0AD7233CF49AFF1F849AFF1FF0
:100D0000E095FF1F2DE9F04F00F12C054FEA810817
:100D100087B005EB080A554504468946029200F063
:100D20003E814FEAA802B2FA82F2C2F11F025200DB
:100D3000B04B51462846FDF749FBAE4A514628467E
:100D4000FDF7ACFAE76AA765B9F1010F40F3358109
:100D5000D7F810B02846012250F8041F0B69013261
:100D6000CBEB430391454B61F6DC3B6AFE69009394
:100D7000554500F02B81E06A04F13003456A1A46BC
:100D800006E01168496A8D4202F1040228BF0D464F
:100D90009245F6D182690DE01968896982EAE270AC
:100DA00081EAE17EA0EBE270AEEBE17E04338645A2
:100DB000B8BF0A469A45EFD110460028B8BF404256
:100DC00020F0F2FF029921F043F821F043FABBF141
:100DD000000F00F0DA80002800F0D780B869002802
:100DE000B8BF404220F0E0FFB9F1000F824640F367
:100DF000EA80584620F0D8FF08F1280783464FF0D4
:100E00000008274404F12809029459F8044F206986
:100E100020F0CAFF594621F0CFF8514621F018F8CA
:100E20000590A0690028B8BF404220F0BDFF059A98
:100E30000146104621F0C0F84146044621F0C4F9AD
:100E400000B1A046B945E0D1029C4146504621F090
:100E5000B3F821F0FFF94FF0000A271D804684F80F
:100E600028A038461BF048FA206238461BF044FAA6
:100E700060621BF015FA616904F108001BF0C6F905
:100E8000A36D5F68DB68A767DF1B009BC4F88880E1
:100E900008FB08F203FB03F0934606FB06F34FF052
:100EA000000CCDE902BC9B46009BC4F88430DDE910
:100EB0000223002FB8BF7F424FF0000C0021C4E98D
:100EC0002823B0EB0B0261EB0C03C4E926016D0093
:100ED000104619465A466346C4E92423E767534639
:100EE000C4F8A850C4F880602A46CDE900BC21F0BF
:100EF000D1F9C01941EBE771CB0FC01841F10001E6
:100F00005FEA61094FEA3008D04541DB47453FDBE6
:100F1000DDE900BCDDE90201B0EB0B0061EB0C0187
:100F20002A46534621F0B6F9804540F39A80C0EB3B
:100F30004803C4F8B030C4F8AC00A368002E00F039
:100F40008A80002B75D01A682B498A4240D82B4AD8
:100F5000B2FBF6F61E60226A2949E46900200325E7
:100F60000126DE60AA4098609D60086002F180431F
:100F70004A6803F5603322440D201A610860DA687C
:100F8000502122F08002DA60D96007B0BDE8F08F0E
:100F900019201BF0C1FF19201BF0BEFFF8E7C76A3C
:100FA000876501293FF7D4AE3B6AFE69D7F810B0D8
:100FB00000933B465D6A9869FFE63B6AFE690093D1
:100FC000D7F810B0D7E64FF000083EE7E36AF1E744
:100FD00059680A48B0FBF6F6521A964212D3B21A72
:100FE0000025012003219D60D8601A6099601E6071
:100FF000B1E700BF890400007F32020000512502E2
:1010000000800340606902680321002701259F607A
:101010001268DD601E6099609047A368002B9AD12A
:10102000174A1268002A96D0284602219047A368E2
:1010300091E71349134A0D68B2FBF6F61DB1022180
:101040000120A847A3680020012103229860D960ED
:101050001E609A607FE74BB19A6822F002029A60A4
:1010600079E7C4F8B080C4F8AC8066E7044B1B682D
:1010700023B1022101209847A368EDE73346EBE74F
:1010800044A0FF1F005125022DE9F04FFDB041F2B1
:1010900088320191804605214EA8FDF719F80024F9
:1010A000984B4E93052206210EA869941AF0BAFFB8
:1010B000142215211EA81AF0B5FF934D17221021F6
:1010C0002EA81AF0AFFF3EA8132212211AF0AAFF91
:1010D0008E4BD5F8D8001C70A0F10A031D2BEE69C9
:1010E000AF693AD98A4C8B4B226805920021059A48
:1010F000197023680493049B9B1A092BF9D986491C
:101100000AA81EF0FBFB00210AA8F0F703FE0AA8BC
:101110001EF0B4FB814B0AA819681EF0EFFB08F122
:10112000FF330AA800210393F0F7F4FD0AA81EF08C
:10113000A5FB039B0D2B00F23C83DFE813F00101BC
:101140006401C90135023A033A033A033A033A0308
:101150003A03B9025B02140313002146C0B21BF02C
:101160009DFEBFE701222B6F029311460420EF6E14
:10117000DFF89491F0F7EAFD6B6D002B40F03385BA
:10118000D9F85C30D9F85800DFF8AC8100FB03F0E7
:1011900020F006FED9F8601020F05AFE6049824621
:1011A000D9F8680020F054FE0146D8F8500020F02D
:1011B00003FF0146504620F04BFE20F09FF9D8F87F
:1011C00030308246D8F828004FF0000900FB03F0C9
:1011D0008B46CDF8FC9020F0E3FD524920F038FE1C
:1011E00021F012F801463EA81AF05EFFD8F82C1044
:1011F0001AF04EFF8046019820F06EF952465B4689
:1012000020F0D0F920F07EFC014640461AF08AFF1B
:10121000689BCDF8A0917CA903F10B0E01EB8E0E1B
:1012200001EB83033EAE43F88C6C4FF07E520121FC
:101230004EA84EF8B49CFFF765FDDDF808A0DFF876
:10124000C890DFF8F880FBB25FFA8AFB1E4658466A
:10125000012102931BF022FE304601211BF01EFEED
:101260005646509B002B00F0C482A6F10A031D2BAA
:1012700040F2A182A7F10A031D2B40F22384D5F886
:10128000D000DFF884A0A0F10A031D2B07D8C0B25C
:101290001BF00AFED9F8D430984240F066841CF066
:1012A0001BFA002840F31B84D8F80000F1F7BEF8C1
:1012B0001D4BC0B2532818701AD1509B002B00F060
:1012C0001A841A4A1B681A49B1FBF3F3F92B13600D
:1012D00000F20C8451A81DF0DDFF002356985093B6
:1012E0001BF01EF857981BF01BF8124B01221A70C6
:1012F00023680993099A23680893089B9B1A012B7A
:10130000F9D9AEE7A8630300BC96FF1F6C9BFF1FD3
:101310007CA0FF1F5594FF1F78820300A487FF1F46
:10132000DB0FC9400AD7233C8595FF1F3093FF1F71
:1013300000512502989AFF1F5894FF1F8087FF1FB6
:101340000122EB69AF69114610461E46F0F7FEFC1C
:1013500023680793079A23680693069B9B1A052B1D
:10136000F9D92B69E868029600FB03F020F018FD1C
:10137000DFF8348369698146D8F8340020F01CFE18
:101380000146484620F064FD20F0B8F8D8F80C304B
:101390008246D8F8040000FB03F08B4620F000FDE5
:1013A000BF4920F055FD20F02FFF01460EA81AF08E
:1013B0007BFED8F808100EA81AF06AFE019820F0FB
:1013C0008BF852465B4620F0EDF820F09BFB01467F
:1013D0000EA81AF0A7FE689B7CA903F10B0E01EB87
:1013E0008E0E01EB83034FF0000C0EAE43F88C6CB5
:1013F0004FF07E5201214EA84EF8B4CCCDF8A0C1DA
:10140000FFF780FC19E701222B6B029311460220A3
:10141000EF6ADFF89892F0F799FCD5F8B830002B16
:1014200040F01A84D9F82430D9F82000DFF8788207
:1014300000FB03F020F0B4FCD9F828108246D8F85D
:10144000380020F0B9FD0146504620F001FD20F0A3
:1014500055F8D8F818308246D8F810004FF0000937
:1014600000FB03F08B46CDF87C9020F099FC8C4972
:1014700020F0EEFC20F0C8FE01461EA81AF014FE73
:10148000D8F814101AF004FE8046019820F024F8D1
:1014900052465B4620F086F820F034FB0146404679
:1014A0001AF040FE689BCDF8A0917CA903F10B0EC9
:1014B00001EB8E0E01EB83031EAE43F88C6C4FF0F4
:1014C0007E5201214EA84EF8B49CFFF71BFCB4E6F7
:1014D00001222B6D029311460320EF6CDFF8CC91B3
:1014E000F0F734FC6B6B002B40F09A83D9F83C305A
:1014F000D9F83800DFF8B08100FB03F020F050FC91
:10150000D9F8401020F0A4FC66498246D9F848007A
:1015100020F09EFC0146D8F83C0020F04DFD01462D
:10152000504620F095FC1FF0E9FFD8F824308246A1
:10153000D8F81C004FF0000900FB03F08B46CDF8F3
:10154000BC9020F02DFC564920F082FC20F05CFE7F
:1015500001462EA81AF0A8FDD8F820101AF098FD20
:10156000804601981FF0B8FF52465B4620F01AF8FB
:1015700020F0C8FA014640461AF0D4FD689BCDF829
:10158000A0917CA903F10B0E01EB8E0E01EB8303FE
:101590002EAE43F88C6C4FF07E5201214EA84EF8CF
:1015A000B49CFFF7AFFB48E601222B6F0293114674
:1015B0000420EF6EDFF8F490F0F7C8FB6B6D002BA2
:1015C00040F02083D9F85C30D9F85800DFF8D88093
:1015D00000FB03F020F0E4FBD9F8601020F038FCA9
:1015E00030498246D9F8680020F032FC0146D8F82C
:1015F0004000DCE501222B6B029311460220EF6ACA
:10160000DFF8A890F0F7A2FBD5F8B830002B40F037
:101610001583D9F82430D9F82000DFF88C8000FB3E
:1016200003F020F0BDFBD9F828108246D8F8480016
:1016300020F0C2FC0146504620F00AFC1FF05EFF7D
:10164000D8F818308246D8F810004FF0000900FB97
:1016500003F08B46CDF87C9020F0A2FB104920F0DF
:10166000F7FB20F0D1FD01461EA81AF01DFDD8F8A9
:1016700014101AF00DFD804601981FF02DFF524600
:101680005B461FF08FFF20F03DFA014640461AF0FE
:1016900049FD012211460220F0F758FB02E700BF86
:1016A0000AD7233CDB0FC9405894FF1FBC96FF1F8D
:1016B000012211461046EB690293AF69DFF850939F
:1016C000F0F744FB2B69E8684FF0000800FB03F0DB
:1016D000CDF83C8020F064FB69698246D9F844006B
:1016E00020F06AFC0146504620F0B2FB1FF006FFD6
:1016F000D9F80C308246D9F8040000FB03F08B4681
:1017000020F04EFBAF4920F0A3FB20F07DFD014609
:101710000EA81AF0C9FCD9F808101AF0B9FC8146D5
:1017200001981FF0D9FE52465B461FF03BFF20F0A8
:10173000E9F9014648461AF0F5FC689BCDF8A0810E
:101740007CA903F10B0E01EB8E0E01EB83030EAEB1
:1017500043F88C6C4FF07E5201214EA84EF8B48CA9
:10176000FFF7D0FA69E501222B6D029311460320A1
:10177000EF6CDFF8A092F0F7E9FA6B6B002B40F00A
:101780007A82D9F83C30D9F83800DFF8848200FB3F
:1017900003F020F005FBD9F8401020F059FB8A49EE
:1017A0008246D9F8480020F053FB0146D8F84C0097
:1017B000B3E6029641E558461BF076FBD5F8D430E7
:1017C00098423FF457AD019B002B7FF753AD51A8D2
:1017D0001DF060FD0023569850931AF0A1FD579814
:1017E0001AF09EFD794B0199012204201A70FCF732
:1017F000FBFA774B1C78002C00F0888175490AA809
:101800001EF07CF800210AA8F0F784FA0AA81EF05E
:1018100035F8714B0AA819681EF070F800210AA863
:10182000F0F778FA0AA81EF029F86C490AA81EF009
:1018300065F800210AA8F0F76DFA0AA81EF01EF854
:10184000654B0AA819681EF059F800210AA8F0F79C
:1018500061FA0AA81EF012F8039B0D2B00F23081EA
:10186000DFE813F00401DA00A4000E002E012E01BF
:101870002E012E012E012E010401DA00A4000E001B
:1018800057483F9B574C03600122002104202360EE
:10189000F0F75CFA544A23681068544903440AA8D4
:1018A00013601EF02BF800210AA8F0F733FA0AA8FB
:1018B0001DF0E4FF484B0AA819681EF01FF800212C
:1018C0000AA8F0F727FA0AA81DF0D8FF48490AA885
:1018D0001EF014F800210AA8F0F71CFA0AA81DF05F
:1018E000CDFF3D4B0AA819681EF008F800210AA890
:1018F000F0F710FA0AA81DF0C1FFD5F8CC30012B83
:1019000000F064813B490AA81DF0F8FF00210AA8F5
:10191000F0F700FA0AA81DF0B1FF37490AA81DF038
:10192000EDFF00210AA8F0F7F5F90AA81DF0A6FFBF
:1019300032490AA81DF0E2FF00210AA8F0F7EAF9EF
:101940000AA81DF09BFF2E490AA81DF0D7FF002111
:101950000AA8F0F7DFF90AA81DF090FF29490AA8A4
:101960001DF0CCFF00210AA8F0F7D4F90AA81DF059
:1019700085FF25490AA81DF0C1FF00210AA8F0F73C
:10198000C9F90AA81DF07AFFD5F8D800A0F10A031A
:101990001D2B03D8C0B201211BF080FA1B4B4E93C4
:1019A0004EA8FCF7E1FB7DB0BDE8F08F0C4A2F9B01
:1019B0000C4C13600021012203202360F0F7C6F9CC
:1019C00068E700BF0AD7233CDB0FC940989AFF1F86
:1019D0006C9BFF1F00850300A487FF1F1485030075
:1019E000DC95FF1F5499FF1FB894FF1F3C8503002F
:1019F0005085030078850300406403008C85030054
:101A000048660300BC820300C8820300A863030089
:101A10005894FF1FBC96FF1F9E499F4C0AA81DF0BB
:101A20006DFF00210AA8F0F775F90AA81DF026FF3E
:101A30002220F0F7C9FC994B00211868F0F776FCDA
:101A4000974B0AA819681DF059FF00210AA8F0F762
:101A500061F90AA81DF012FF924A1F9B1360002132
:101A6000012202202360F0F771F913E789498A4CBB
:101A70000AA81DF043FF00210AA8F0F74BF90AA8B5
:101A80001DF0FCFE2220F0F79FFC874B0021186818
:101A9000F0F74CFC824B0AA819681DF02FFF0021BB
:101AA0000AA8F0F737F90AA81DF0E8FE7D4A0F9B57
:101AB00013600122104600212360F0F747F9E9E6A0
:101AC000754CE7E602981BF0EFF9D5F8D430984250
:101AD0003FF4D5AB019B002BBFF6D1AB77E6EEF719
:101AE000D9FD0028FFF604ACFFF7DEBB4EA8FCF7DB
:101AF000E1FAFFF7FABB6D4B1B68002B3FF4E1AB3B
:101B0000022101209847509BFFF7DBBB68490AA8D8
:101B10001DF0F4FE21460AA8F0F7FCF80AA81DF013
:101B2000ADFE644B0AA819681DF0E8FE21460AA81C
:101B3000F0F7F0F80AA81DF0A1FE5F490AA81DF011
:101B4000DDFE21460AA8F0F7E5F80AA81DF096FE8A
:101B5000584B0AA819681DF0D1FE0AA82146F0F7D3
:101B6000D9F80AA81DF08AFE48E651A800241DF005
:101B700091FB56985094514E1AF0D2FB57981AF098
:101B8000CFFB01252246214620463570F0F7DEF8CE
:101B9000224621462846F0F7D9F82246214602205F
:101BA000F0F7D4F8224621460320F0F7CFF80420BE
:101BB000FBF786FBDAF8D800A0F10A031D2B3FF6ED
:101BC000EDAE2946C0B21BF069F9E7E63C490AA828
:101BD0001DF094FE00210AA8F0F79CF80AA81DF059
:101BE0004DFE3849C6E6D9F85C30D9F85800DFF820
:101BF000D88000FB03F020F0D3F8D9F864108246B7
:101C0000FFF7D3BAD9F85C30D9F85800DFF8B880BC
